:020000040800F2
:100000000000012015240008A1160008A31600080E
:10001000A5160008A7160008A91600080000000091
:10002000000000000000000000000000AB16000807
:10003000AD16000800000000AF160008B116000859
:100040006524000865240008B5160008652400082A
:100050006524000865240008C1160008C7160008BA
:10006000652400086524000865240008652400084C
:10007000652400086524000865240008CD160008E2
:10008000652400086524000865240008652400082C
:100090000000000065240008D91600086524000847
:1000A000652400086524000865240008652400080C
:1000B00065240008652400086524000865240008FC
:1000C00065240008652400086524000865240008EC
:1000D00065240008E116000865240008652400086E
:1000E0006524000865240008ED1600086524000852
:1000F00065240008000000000000000065240008DE
:100100006524000865240008F91600086524000825
:10011000652400086524000865240008652400089B
:10012000652400086524000865240008652400088B
:080130006524000865240008A5
:1001380010B5054C237833B9044B13B10448AFF319
:1001480000800123237010BD08010020000000007A
:1001580028F0000808B5034B1BB103490348AFF367
:10016800008008BD000000000C01002028F00008F5
:10017800034613F8012B002AFBD1181A01387047DF
:1001880081F0004102E000BF83F0004330B54FEA40
:1001980041044FEA430594EA050F08BF90EA020FAD
:1001A8001FBF54EA000C55EA020C7FEA645C7FEA40
:1001B800655C00F0E2804FEA5454D4EB5555B8BF63
:1001C8006D420CDD2C4480EA020281EA030382EAD4
:1001D800000083EA010180EA020281EA0303362D66
:1001E80088BF30BD11F0004F4FEA01314FF4801C39
:1001F8004CEA113102D0404261EB410113F0004F4B
:100208004FEA03334CEA133302D0524263EB430301
:1002180094EA050F00F0A780A4F10104D5F1200E9F
:100228000DDB02FA0EFC22FA05F2801841F10001FA
:1002380003FA0EF2801843FA05F359410EE0A5F1CE
:1002480020050EF1200E012A03FA0EFC28BF4CF0FF
:10025800020C43FA05F3C01851EBE37101F00045B5
:1002680007D54FF0000EDCF1000C7EEB00006EEBC2
:100278000101B1F5801F1BD3B1F5001F0CD349084C
:100288005FEA30004FEA3C0C04F101044FEA4452A3
:1002980012F5800F80F09A80BCF1004F08BF5FEA2A
:1002A800500C50F1000041EB045141EA050130BD0A
:1002B8005FEA4C0C404141EB0101013C28BFB1F51C
:1002C800801FE9D291F0000F04BF01460020B1FA67
:1002D80081F308BF2033A3F10B03B3F120020CDA3A
:1002E8000C3208DD02F1140CC2F10C0201FA0CF018
:1002F80021FA02F10CE002F11402D8BFC2F1200C7D
:1003080001FA02F120FA0CFCDCBF41EA0C01904032
:10031800E41AA2BF01EB0451294330BD6FEA04047B
:100328001F3C1CDA0C340EDC04F11404C4F1200266
:1003380020FA04F001FA02F340EA030021FA04F378
:1003480045EA030130BDC4F10C04C4F1200220FACF
:1003580002F001FA04F340EA0300294630BD21FA0D
:1003680004F0294630BD94F0000F83F4801306BFD3
:1003780081F480110134013D4EE77FEA645C18BFC7
:100388007FEA655C29D094EA050F08BF90EA020F5E
:1003980005D054EA000C04BF1946104630BD91EA56
:1003A800030F1EBF0021002030BD5FEA545C05D159
:1003B8004000494128BF41F0004130BD14F5800498
:1003C8003CBF01F5801130BD01F0004545F0FE410C
:1003D80041F470014FF0000030BD7FEA645C1ABF41
:1003E800194610467FEA655C1CBF0B46024650EA78
:1003F800013406BF52EA033591EA030F41F40021A4
:1004080030BD00BF90F0000F04BF0021704730B529
:100418004FF4806404F132044FF000054FF00001FE
:1004280050E700BF90F0000F04BF0021704730B5BF
:100438004FF4806404F1320410F0004548BF404294
:100448004FF000013EE700BF42004FEAE2014FEAE9
:1004580031014FEA02701FBF12F07F4393F07F4FC4
:1004680081F06051704732F07F4208BF704793F0C7
:100478007F4F04BF41F40021704730B54FF46074DA
:1004880001F0004521F000411CE700BF50EA0102DD
:1004980008BF704730B54FF000050AE050EA010286
:1004A80008BF704730B511F0004502D5404261EBF6
:1004B80041014FF4806404F132045FEA915C3FF437
:1004C800D8AE4FF003025FEADC0C18BF03325FEAD4
:1004D800DC0C18BF033202EBDC02C2F1200300FA85
:1004E80003FC20FA02F001FA03FE40EA0E0021FAAA
:1004F80002F11444BDE600BF4FF0FF3C06E000BF28
:100508004FF0010C02E000BF4FF0010C4DF804CD94
:100518004FEA410C7FEA6C5C4FEA430C18BF7FEA54
:100528006C5C1BD001B050EA410C0CBF52EA430C82
:1005380091EA030F02BF90EA020F0020704710F102
:10054800000F91EA030F58BF994208BF90422CBF91
:10055800D8176FEAE37040F0010070474FEA410C8A
:100568007FEA6C5C02D150EA013C07D14FEA430CA8
:100578007FEA6C5CD6D152EA033CD3D05DF8040B19
:10058800704700BF8446104662468C46194663464B
:1005980000E000BF01B5FFF7B7FF002848BF10F122
:1005A800000F01BD4DF808EDFFF7F4FF0CBF012067
:1005B80000205DF808FB00BF4DF808EDFFF7EAFFE3
:1005C80034BF012000205DF808FB00BF4DF808ED9E
:1005D800FFF7E0FF94BF012000205DF808FB00BF93
:1005E8004DF808EDFFF7CEFF94BF012000205DF81D
:1005F80008FB00BF4DF808EDFFF7C4FF34BF01202A
:1006080000205DF808FB00BF4FEA410212F5001216
:1006180015D211D56FF47873B3EB625212D94FEA41
:10062800C12343F0004343EA505311F0004F23FA2B
:1006380002F018BF404270474FF00000704750EA80
:10064800013005D111F0004008BF6FF0004070473D
:100658004FF00000704700BF80F0004002E000BF8C
:1006680081F0004142001FBF5FEA410392EA030F95
:100678007FEA226C7FEA236C6AD04FEA1262D2EBDF
:100688001363C1BFD218414048404140B8BF5B42E4
:10069800192B88BF704710F0004F40F4000020F07D
:1006A8007F4018BF404211F0004F41F4000121F093
:1006B8007F4118BF494292EA030F3FD0A2F10102DD
:1006C80041FA03FC10EB0C00C3F1200301FA03F11B
:1006D80000F0004302D5494260EB4000B0F5000F3E
:1006E80013D3B0F1807F06D340084FEA310102F1FD
:1006F8000102FE2A51D2B1F1004F40EBC25008BFAF
:1007080020F0010040EA03007047490040EB000078
:10071800013A28BFB0F5000FEDD2B0FA80FCACF179
:10072800080CB2EB0C0200FA0CF0AABF00EBC250A6
:1007380052421843BCBFD0401843704792F0000F94
:1007480081F4000106BF80F400000132013BB5E7E7
:100758004FEA41037FEA226C18BF7FEA236C21D05D
:1007680092EA030F04D092F0000F08BF08467047C2
:1007780090EA010F1CBF0020704712F07F4F04D190
:10078800400028BF40F00040704712F100723CBFA3
:1007980000F50000704700F0004343F0FE4040F4CD
:1007A800000070477FEA226216BF08467FEA23638B
:1007B8000146420206BF5FEA412390EA010F40F476
:1007C800800070474FF0000304E000BF10F00043C2
:1007D80048BF40425FEA000C08BF704743F09643A9
:1007E80001464FF000001CE050EA010208BF7047C4
:1007F8004FF000030AE000BF50EA010208BF70474B
:1008080011F0004302D5404261EB41015FEA010C5F
:1008180002BF84460146002043F0B64308BFA3F157
:100828008053A3F50003BCFA8CF2083AA3EBC25339
:1008380010DB01FA02FC634400FA02FCC2F1200258
:10084800BCF1004F20FA02F243EB020008BF20F08F
:100858000100704702F1200201FA02FCC2F12002F5
:1008680050EA4C0021FA02F243EB020008BF20EAEA
:10087800DC7070474FF0FF0C1CEAD0521EBF1CEA18
:10088800D15392EA0C0F93EA0C0F6FD01A4480EA06
:10089800010C400218BF5FEA41211ED04FF00063EF
:1008A80043EA501043EA5111A0FB01310CF000401B
:1008B800B1F5000F3EBF490041EAD3715B0040EA41
:1008C800010062F17F02FD2A1DD8B3F1004F40EB11
:1008D800C25008BF20F00100704790F0000F0CF0E4
:1008E800004C08BF49024CEA502040EA51207F3AA8
:1008F800C2BFD2F1FF0340EAC250704740F4000083
:100908004FF00003013A5DDC12F1190FDCBF00F073
:1009180000407047C2F10002410021FA02F1C2F121
:10092800200200FA02FC5FEA310040F1000053EABD
:100938004C0308BF20EADC70704792F0000F00F00B
:10094800004C02BF400010F4000F013AF9D040EA11
:100958000C0093F0000F01F0004C02BF490011F4A5
:10096800000F013BF9D041EA0C018FE70CEAD153A3
:1009780092EA0C0F18BF93EA0C0F0AD030F0004C23
:1009880018BF31F0004CD8D180EA010000F00040D7
:10099800704790F0000F17BF90F0004F084691F095
:1009A800000F91F0004F14D092EA0C0F01D14202CF
:1009B8000FD193EA0C0F03D14B0218BF084608D198
:1009C80080EA010000F0004040F0FE4040F40000E2
:1009D800704740F0FE4040F4400070474FF0FF0C75
:1009E8001CEAD0521EBF1CEAD15392EA0C0F93EABC
:1009F8000C0F69D0A2EB030280EA010C49024FEA0E
:100A0800402037D04FF0805343EA111143EA1013C6
:100A18000CF000408B4238BF5B0042F17D024FF47E
:100A2800000C8B4224BF5B1A40EA0C00B3EB510F59
:100A380024BFA3EB510340EA5C00B3EB910F24BF42
:100A4800A3EB910340EA9C00B3EBD10F24BFA3EBC7
:100A5800D10340EADC001B0118BF5FEA1C1CE0D18F
:100A6800FD2A3FF650AF8B4240EBC25008BF20F042
:100A7800010070470CF0004C4CEA50207F32C2BF96
:100A8800D2F1FF0340EAC250704740F400004FF033
:100A98000003013A37E792F0000F00F0004C02BF64
:100AA800400010F4000F013AF9D040EA0C0093F02E
:100AB800000F01F0004C02BF490011F4000F013B88
:100AC800F9D041EA0C0195E70CEAD15392EA0C0FF0
:100AD80008D142027FF47DAF93EA0C0F7FF470AF28
:100AE800084676E793EA0C0F04D14B023FF44CAF6B
:100AF80008466EE730F0004C18BF31F0004CCAD100
:100B080030F000427FF45CAF31F000437FF43CAF3B
:100B18005FE700BF4FEA4002B2F1FE4F0FD34FF03C
:100B28009E03B3EB12620DD94FEA002343F0004352
:100B380010F0004F23FA02F018BF404270474FF000
:100B48000000704712F1610F01D1420205D110F087
:100B5800004008BF6FF0004070474FF0000070473A
:100B680042000ED2B2F1FE4F0BD34FF09E03B3EB0F
:100B7800126209D44FEA002343F0004323FA02F03B
:100B880070474FF00000704712F1610F01D1420227
:100B980002D14FF0FF3070474FF00000704700BFA0
:100BA80053B94AB9002908BF00281CBF4FF0FF31CC
:100BB8004FF0FF3000F06AB9ADF1080C6DE904CED2
:100BC80000F006F8DDF804E0DDE9022304B0704720
:100BD8002DE9F047089D0C46002B4ED194468C45D4
:100BE8008646B2FA82F262D94AB1C2F12003914034
:100BF80020FA03F30CFA02FC194300FA02FE4FEA4A
:100C08001C471FFA8CF6B1FBF7F44FEA1E4307FBAB
:100C1800141143EA014304FB06F199420AD91CEB7B
:100C2800030304F1FF3080F01281994240F20F81F2
:100C3800023C6344591A1FFA8EF3B1FBF7F007FB25
:100C4800101143EA014300FB06F69E420AD91CEB49
:100C5800030300F1FF3180F0FC809E4240F2F980EE
:100C6800634402389B1B40EA044000211DB1D34075
:100C78000022C5E90032BDE8F0878B4205D90DB1E5
:100C8800C5E9000100210846F5E7B3FA83F1002918
:100C980046D1A34202D39042C0F0F080861A64EB9A
:100CA80003030120002DE6D0C5E90063E3E7002A2D
:100CB80040F09080A1EB0C044FEA1C481FFA8CF717
:100CC8000121B4FBF8F64FEA1E4308FB164443EA39
:100CD800044307FB06F0984208D91CEB030306F10E
:100CE800FF3402D2984200F2CD8026461C1A1FFA21
:100CF8008EF3B4FBF8F008FB104443EA044300FB0E
:100D080007F79F4208D91CEB030300F1FF3402D216
:100D18009F4200F2B0802046DB1B40EA0640A5E770
:100D2800C1F120068B4022FA06F71F4320FA06FC81
:100D380004FA01F343EA0C03F44000FA01F8380C12
:100D48004FEA1349B4FBF0FE1FFA87FC00FB1E4470
:100D580049EA04440EFB0CF9A14502FA01F20AD94A
:100D68003C190EF1FF3A80F08480A14540F2818061
:100D7800AEF1020E3C44A4EB09041FFA83F9B4FB5C
:100D8800F0F300FB134449EA044403FB0CFCA445BC
:100D980007D93C1903F1FF3067D2A44565D9023B56
:100DA8003C4443EA0E40A0FB0293A4EB0C049C4293
:100DB800CE469C4651D34ED055B1B8EB0E0364EBEA
:100DC8000C0404FA06F6CB401E43CC40C5E9006487
:100DD800002150E7C2F1200320FA03F10CFA02FCCB
:100DE80024FA03F394400C434FEA1C4800FA02FE2D
:100DF8001FFA8CF7B3FBF8F008FB1031230C43EA19
:100E0800014300FB07F1994208D91CEB030300F1E9
:100E1800FF362CD299422AD9023863445B1AA4B20D
:100E2800B3FBF8F108FB113344EA034401FB07F371
:100E3800A34208D91CEB040401F1FF3613D2A342E4
:100E480011D902396444E41A41EA004139E70446F9
:100E5800F0E6084606E7C845AED2B9EB020E63EBEA
:100E6800070C0138A8E73146EDE7034699E7304615
:100E7800D4E7D6467FE7634402384DE70646234663
:100E880008460FE7023E634430E700BF704700BFE3
:100E98001348144A08B54FF00043C0E90023042260
:100EA800426101220023C2614FF480510722C0E948
:100EB8000233C0E90933C0E90C1203610383837666
:100EC80080F8203080F82C30826380F83C30C3648E
:100ED80001F000FB18B1BDE8084000F01FBB08BDD9
:100EE80024010020002401400268084B9A4282B085
:100EF8000AD14FF0B0431A6E42F400721A661B6EA4
:100F080003F400730193019B02B070470024014071
:100F18000268054B9A4201BF4FF0B042136E23F4AA
:100F280000731366704700BF0024014030B585B0D8
:100F380000240546CDE901440394FFF7A9FF1448AE
:100F480001F05CFE08B100F0E9FA1148039401A928
:100F5800CDE9015401F01CFC08B100F0DFFA0C489F
:100F680001F076FD08B100F0D9FA4FF0FF310848DA
:100F780001F0B0FB064801F023FE054801F004FC2F
:100F88000446034801F0C6FD204605B030BD00BF49
:100F980024010020014B024A1A60704724010020F6
:100FA8000024014008B50948FFF7C0FF68B1084BA5
:100FB800B3F8AA304FF6FF72934216BF40F6E442E8
:100FC800044B5343B3FBF0F398B208BD002000B4C0
:100FD8000075FF1FD8084C0013B50023ADF8063084
:100FE800FFF7E0FF04461948FFF7A0FF184BB3F8D6
:100FF800C820B3F8A8108A4204FB00F018D040F6C5
:10100800E443B0FBF3F364205B1A4343521A93FBA7
:10101800F2F31E331BB2ADF80630BDF806305BB2F2
:101028001B02ADF80630BDF8060000B202B010BDD4
:101038004FF47A7240F6FF73B0FBF3F35343A3F512
:101048003923A3F50C6340F6C412E0E7001000B0A2
:101058000075FF1F4FF0B04307B59A6C42F00402C9
:101068009A649A6C02F004020192019A9A6C42F016
:1010780001029A649B6C03F0010300930022022191
:101088000F20009B01F058FE0F2003B05DF804EB21
:1010980001F084BE08B502F0C5F810B16FF0040085
:1010A80008BD064B9A6942F040429A614CF2FA3206
:1010B8001A6102F0C9F80028F2D0EFE700400058A2
:1010C800F0B585B000230D4600930646A8B3FFF798
:1010D800E1FF044670BB02F0A5F888BB1A481B4A1A
:1010E80002230193D0F8E01506F1784302EA812142
:1010F800B3FBF1F701FB1733DB0A0293D0F8E005E5
:1011080005F178410139314402EA8022B1FBF2F05D
:1011180002FB1011C3EBD1230133694601A80393E5
:1011280002F012F920B1022814BF6FF00104012463
:1011380002F08AF8204605B0F0BD6FF00504F9E723
:101148006FF00404F6E700BF0070FF1F00FCFF0308
:10115800014B186000207047880100202DE9F04FEE
:10116800B0F1006F89B006460F469046C0F0C080C7
:10117800DFF89091644DD9F8E03505EA832303F14F
:101188000063013B984200F2B380002900F0B3806D
:1011980040EA02035B0740F0AE80FFF77BFF04469E
:1011A80090BB02F03FF8002840F0A880D9F8E0157D
:1011B800009705EA812106F17842B2FBF1F301FBC1
:1011C800132208F17843013B3344B3FBF1F001FBF0
:1011D8001033DB0A01334FEAD22AA3EBD222012AC9
:1011E800039388BFC6F30A050AF58037C6F10803DA
:1011F8008CBFC5F500654546FF02B3460693039BC1
:101208009A4505D302F020F8204609B0BDE8F08FD2
:10121800A6F10803069A1A4495421CD8009B049527
:101228000193CDF814B04FF00009059B09EB0301B9
:10123800049B99453DD3009BAB442B44A8EB050583
:10124800B5F5006F009328BF4FF400650AF1010A55
:1012580007F50067D3E753F8081F5A68B2F1FF3F54
:1012680008BFB1F1FF3FD5D0284B186810B96FF00F
:101278000504C7E727B14FF4006239460DF0F6F9C7
:10128800DFF888900099D9F80030CBF30A001844A9
:10129800AAB20DF0EBF94FF400613846FFF710FFE2
:1012A80000BBD9F8003001934FF40063059704930D
:1012B800B9E7019B07914B4402930120D3E900232E
:1012C80001F0FCFF88B90799019BD1E9000259F8A0
:1012D8000310029B5B689A4208BF884205D109F156
:1012E8000809A2E76FF001048CE76FF0030489E7AF
:1012F8004FF0FF3488E76FF0050485E76FF00404CA
:1013080082E700BF0070FF1F00FCFF038801002078
:10131800B1F1006F70B510D30B4BD3F8E0650B4BF0
:1013280003EA862303F10063013B994205D838B1EB
:1013380092B20DF09BF9002070BD4FF0FF30FBE733
:101348006FF00500F8E700BF0070FF1F00FCFF0307
:10135800B0F1006F10B40DD3084BD3F8E045084B3B
:1013680003EA842303F10063013B984202D810BCCE
:10137800FFF7A6BE4FF0FF3010BC70470070FF1F8C
:1013880000FCFF034FF0B04382B0DA6C0243DA642A
:10139800DB6C03400193019B02B0704730B502201B
:1013A80087B000242C4DCDE90444FFF7EBFF04205F
:1013B800FFF7E8FF0120FFF7E5FF01A94FF6FF72ED
:1013C80003232846CDE90123039402F00BF801A971
:1013D800224802F007F801A94FF0904002F002F805
:1013E8004FF0B0432846DA6C22F00102DA64DA6C76
:1013F80022F00202DA64DA6C22F00402DA644FF4B2
:101408003A41224602F00EF90220FFF7BBFF1421F1
:101418000123CDE90113CDE9030001A9284601F014
:10142800E1FF22462146062001F086FC062001F055
:10143800B5FC22462146072001F07EFC072001F07A
:10144800ADFC22462146162001F076FC162001F05C
:10145800A5FC07B030BD00BF0004004800080048E4
:1014680000B59BB04822002108A80DF02BFD1822DA
:10147800002102A80DF026FD02F0EEF84FF0B04270
:101488000120D2F8903023F01803C2F89030D2F837
:10149800003423F4C06343F40073C2F80034D2F874
:1014A800003403F4C0630193019B24230893812330
:1014B8000B930023CDE91003B02208A8CDE912232D
:1014C80002F054FA08B172B6FEE74F23CDE90230B4
:1014D800CDE90400CDE90600022102A802F0E0FCF3
:1014E80008B172B6FEE71BB05DF804FB08B500F062
:1014F800B7FFFFF7B5FFFFF751FF064803F0EEFB14
:1015080000F058FC04480122102102F08BF800F08A
:1015180058FCFCE73C0200200004004872B6FEE7D5
:1015280000B58DB02C22002101A80DF0CBFC174886
:10153800174B03601F2383604FF080420023C0E9EC
:101548000433C0E9072383614FF48073436202F0D8
:101558004DFF08B1FFF7E2FF0C4803F073F808B13C
:10156800FFF7DCFF4FF0005300220793074808926B
:101578004FF4807301A9029206920B9302F096FF32
:1015880008B1FFF7CBFF0DB05DF804FB8C0100201C
:101598000028004010B5044690B03822002102A867
:1015A8000DF090FC2268194B9A422CD14FF48033ED
:1015B800029302A84FF480730F9302F095FD08B1CF
:1015C800FFF7ACFF4FF0B0430220D3F8902042F46D
:1015D8000042C3F890209A6D42F480629A659B6D30
:1015E800002203F4806311460193019B01F0A4FBE0
:1015F800022001F0D3FB00222A20114601F09CFBB7
:101608002A2001F0CBFB10B010BD00BF002800401D
:1016180008B500F03BFF034B07229A61BDE808407C
:1016280002F042B80004005800F037BF08B50F4870
:1016380003F054FB00F07CFB4FF6FF714FF0904035
:1016480001F07CFF0A484FF6FF7101F077FF094867
:101658004FF6FF7101F072FF00F018FF064B0120F2
:10166800C3F88800BDE8084002F060B83C020020DA
:1016780000040048000800480004005808B500F0BD
:1016880005FFBDE808400121002001F0EDBF00F092
:1016980004BF00F002BF7047FEE7FEE7FEE7FEE783
:1016A800FEE770477047704770470000014802F036
:1016B800EFBF00BF8C010020012001F0C1BF022054
:1016C80001F0BEBF014801F03FBD00BFDC010020B2
:1016D800402001F0B5BF0000014803F0BBBB00BFCC
:1016E8003C020020014802F007BE00BF8C01002028
:1016F800014803F0F6B900BFC4010020054808B549
:101708000823036003F00AF818B1BDE80840FFF7A2
:1017180005BF08BDC40100204FF0B04307B55A6E9D
:1017280042F001025A665B6E002203F00103019346
:1017380011463220019B01F0FFFA322003B05DF818
:1017480004EB01F02BBB00000CB407B5054A05AB50
:10175800102101930DF094FA03B05DF804EB02B088
:10176800704700BFCCF0000830B585B0044602A829
:101778000D460DF0B1F8BDF90C30064A0093102162
:10178800029B2046FFF7E0FF2046FEF7F1FC288089
:1017980005B030BDCCF000084FF0B04210B59368EA
:1017A80023F4004393600DF01FF90D4B01241C70C6
:1017B8000CF0ECFD0B480CF003FE0B4B4FF4004211
:1017C8001A6100200CF002FEFFF7E4FB00F0B4F809
:1017D8000CF0F6FE21462046BDE810400CF010BF84
:1017E800D001002071170008004000580CF01EBFFF
:1017F80008B5FFF7D7FB40F6B83398420CD8B0F5D8
:10180800E16F0BD3FE23A0F5E16058434FF49663D4
:10181800B0FBF3F0C0B208BDFE20FCE70020FAE7F9
:101828007FB5684600F06CF80198FFF773F900B2CD
:1018380007B05DF804FB0000194A38B5D2F88035C6
:10184800591C044619D100F02FFE054600F038FE59
:10185800054400F02FFE2B0EE3712B0CA3712B0A0D
:101868006371030EE370C0F30742C0F307232571C9
:10187800C0B2A2706370207038BD190AC37181713B
:10188800190C1B0E41710371D2F88435C370D2F85C
:101898008405C0F30722C0F30743000EE9E700BF41
:1018A8000070FF1F38B5094BD3F88035036001334A
:1018B800054609D100F0F8FD044600F0FBFD444060
:1018C80000F0FEFD44402C6038BD00BF0070FF1FD3
:1018D800012102200CF07EBE002102200CF07ABE0D
:1018E80000207047024B187808B100F05DB87047C7
:1018F800D001002082B00190019802B000F0F0B849
:1019080010B50446FFF768FB074BA36040F30F20B0
:10191800FEF75CFF054B064A2360064B6060C4E98E
:101928000323002010BD00BF0000484200007A4495
:101938000D093E00AB03050000207047014B1868F5
:10194800704700BFD40100200320704708B5014646
:101958004FF47A7200238002890DFFF721F908BD40
:101968004FF47A73A0FB0303800A40EA8350704760
:10197800034B98689A689042FBD1C043704700BFF8
:101988000028004008B5FFF7F3FF014B186008BDB9
:10199800D401002008B5FFF7EBFF024B1B68C01A03
:1019A80008BD00BFD4010020024B187808B1FFF72A
:1019B800DFBF7047D801002010B5074B074C012244
:1019C800DA654FF48071204602F05CFC4FF0FF337B
:1019D8002363002010BD00BF002800408C010020B8
:1019E80002460021014802F064BE00BF8C010020BD
:1019F80002460121014802F05CBE00BF8C010020B4
:101A080010B58CB02C220021044601A80DF05AFA1A
:101A1800FFF7D2FF0C4B0D481B681C4400230893AA
:101A280006934FF00053E443079301224FF4807369
:101A380001A902940B9302F039FD08B1FFF76EFD7E
:101A480000200CB010BD00BFD40100208C01002084
:101A580038B50546FFF78CFF02210446074802F017
:101A68002FFEC4F309024FF47A71A2FB0121920AF6
:101A7800A30A2A8043EA805038BD00BF8C010020A9
:101A88000148002102F01CBE8C0100200148012100
:101A980002F016BE8C010020F8B50F4D2E78CEB995
:101AA8000E4C4FF0FF372763FFF73AFDFFF784FF2F
:101AB8004FF48071204602F0E5FB2046276302F0D0
:101AC800A3FD32462046022102F0F3FDFFF75AFF3C
:101AD80001232B700020F8BDD80100208C010020C4
:101AE800014610B54FF47A7200238002890DFFF782
:101AF80057F80146FFF73CFF0446FFF739FF031B81
:101B08008B4200D310BD00BFF7E70DF075B8000099
:101B180010B5064C0221204602F0D2FD0221421CDB
:101B28002046BDE8104002F0C4BD00BF8C01002073
:101B38001348144A08B54FF4E133C0E900230023E1
:101B48000C22C0E90233C0E90523C0E90733C0E924
:101B58000933036103F063FF08B1FFF7DFFC0848AE
:101B6800002104F0D4F808B1FFF7D8FC044804F0C9
:101B7800AEF818B1BDE80840FFF7D0BC08BD00BFFB
:101B88003C0200200044004070B596B0064614227E
:101B9800002103A80DF096F93822002108A80DF0BD
:101BA80091F932682C4B9A4254D10223089308A821
:101BB8002A4B0A9302F098FA08B1FFF7AFFC4FF0EE
:101BC800B04300259A6D42F400329A659A6D02F48A
:101BD80000320292029ADA6C42F00102DA64DB6C9B
:101BE80003F0010301930422019B0223CDE903239F
:101BF8000324072303A94FF09040CDE90554079328
:101C080001F0F0FB082303A94FF09040CDE903341D
:101C1800CDE90555124C01F0E5FB12492562142364
:101C2800C4E900131023C4E9023520468023C4E91F
:101C38000435C4E9065501F011F908B1FFF76EFC47
:101C48002520F46700220221A66201F075F82520FC
:101C580001F0A4F816B070BD0044004004000C0068
:101C6800DC0100205800024002680C4B9A4210B573
:101C7800044612D14FF0B0420C21936D23F4003387
:101C880093654FF0904001F059FCE06F01F058F96E
:101C9800BDE81040252001F08FB810BD0044004079
:101CA80008B50A460146024803F038F8002008BD86
:101CB8003C02002013B5114B114C18604FF400136F
:101CC800009302AB13E90600204603F0A4FF236843
:101CD800DA69D103FCD4DA695202FCD59A6808485B
:101CE80042F480029A6003F0DCFF064904480122AE
:101CF80003F04AFF002002B010BD00BFD002002050
:101D08003C020020D802002008B5074B1860FFF7F6
:101D1800A1F9FFF70DFF054AD2F8803043F00063C0
:101D2800C2F88030002008BDD40200200008005806
:101D380008B54FF0B04308489A6B42F400329A63F2
:101D48009A6B22F400329A63FFF78EFF0F2001F09E
:101D580033F8002008BD00BF3C0200200268044B95
:101D68009A4203D1034B00201B681847704700BFF5
:101D780000440040D402002002680B4B9A4210B580
:101D880004460FD1094B1B682BB1D0F8902012B92B
:101D980007480121984720460549BDE8104001221F
:101DA80003F0F2BE10BD00BF00440040D002002086
:101DB800D802002008B5FFF7EFFCBDE8084000F0A6
:101DC80013BA4FF0FF300CF095BC7047704770475E
:101DD800014BD870704700BF0C000020014B1874ED
:101DE800704700BF0C000020024800224FF4004159
:101DF80001F018BC00040048024800224FF40071AA
:101E080001F010BC00040048002101200CF03ABC8D
:101E180008B50E4B1B78022B03D1002108200CF0CB
:101E280031FC0B4800224FF4004101F0FBFB08484D
:101E380000224FF4007101F0F5FBBDE808400448AA
:101E480000224FF4006101F0EDBB00BF70000020DC
:101E58000004004810B54EF66023084C002818BF4F
:101E68000346074823600CF027FE216804480CF05D
:101E7800ABFEBDE8104002480CF06CBE0800002024
:101E8800300400200A460149FFF742BA00F003086F
:101E980038B5154801224FF4004101F0C3FB124840
:101EA80001224FF4007101F0BDFB0F4801224FF4ED
:101EB800006101F0B7FB0D480CF0FEFD04F088FB53
:101EC80060B90B4C0B480125257004F015FA2078F1
:101ED800294603F069FF05480CF03CFEBDE8384090
:101EE80005480CF037BE00BF00040048300400204D
:101EF800700000200C0000201804002004F006BC2C
:101F08002DE9F04387B0FFF773FC054604F046F867
:101F1800074690B1002447480CF0CEFD464B454893
:101F28001B689C42214638BF19460CF04DFE4148BB
:101F38000CF010FE07B0BDE8F083404C6846FFF790
:101F4800DFFC0223029823703D49FEF793FCFEF75D
:101F580007FE86B20198FEF7DDFD3A490FFA80F8D0
:101F68000098FEF787FC3649FEF738FDFEF7F8FDC6
:101F7800354A636812781A706368C0F307225A708A
:101F880063689870636883F803806368320A1A711B
:101F980063685E712D4E3378082B01D0012B2DD844
:101FA8006268002393716268D371626828B200EB9B
:101FB80040001372537200EB4010FE23B0FBF3F0A5
:101FC8000B2390726370224C637A63B103F0D2FFE3
:101FD800012808D120460CF06FFD1E4800224FF45E
:101FE800006101F01FFBF1781448002203F0ECFFB8
:101FF80006308FD103F0B8FF04468CE7DDE903858E
:10200800D4F80490FFF7F4FB89F8060063684FEAF8
:102018002842DA7163684FEA28221A722A149A72DF
:102028002A1283F80980DA721D735F739F730F2376
:10203800C8E700BF3004002008000020000000208E
:10204800000020410000C842240300200C000020AA
:10205800DC0200200004004802484FF4006101F04F
:10206800E6BA00BF0004004808B560B1037853B170
:10207800054801224FF4007101F0D4FABDE8084088
:1020880002480CF067BD08BD000400480C0300209E
:1020980008B504F0A6FA80B903F06CFF01280CD14A
:1020A800BFF34F8F0549064BCA6802F4E062134339
:1020B800CB60BFF34F8F00BFFDE708BD00ED00E028
:1020C8000400FA0510B568B190F9064054B90648FD
:1020D8000CF0F2FC22460548BDE810404FF40061C0
:1020E80001F0A0BA10BD00BFDC02002000040048C7
:1020F80038B504460D4681B3184801224FF4004113
:1021080001F090FA16480CF025FD2B782BB324B378
:10211800636822780BB3022A0ED0032A1DD1627895
:10212800012A1AD11878012802D0022800D0A0B9B3
:10213800BDE8384004F012B86278012A0DD11B7846
:10214800084903F001030B7003B91A46BDE838408B
:1021580002484FF4006101F065BA38BD0004004838
:10216800F40200202403002038B504460D46074831
:102178004FF40061FFF7ECF830B92A4621460348CE
:10218800BDE83840FEF7EABF38BD00BF00F00308DD
:102198004FF0B04313B5DA6C104C42F00202DA6427
:1021A800DB6C03F002030122019320461021019BFE
:1021B80001F038FA002102200CF064FA4FF4FA60BA
:1021C800FFF798FB20460022102101F02BFA044863
:1021D80002B0BDE810400CF0BDBC00BF00040048D0
:1021E80030040020704700001FB5002403A92046D2
:1021F800039404F0DBF903A9012004F0D7F92C4B70
:102208002C48009422464FF4FA710CF0F7FB2A4B45
:102218002A48009422464FF4FA710CF0EFFB284B41
:102228002848009401224FF4FA710CF0E7FB20468D
:10223800FEF78EFF08B1FFF771F9234B00940022D7
:102248004FF4FA6121480CF0D9FB214A0021012002
:102258000CF0D4FA1F4A002102200CF0CFFA1E4AD3
:10226800002104200CF0CAFA1C4A002108200CF0B6
:10227800C5FA00F04FF81A491A4804F04DF91A48FF
:1022880004F03AF80F480CF065FC184B0021187858
:1022980003F08AFD16490094164B09681648002277
:1022A8000CF0ACFB14480CF055FC04B010BD00BF9A
:1022B800011E00080C030020F11D0008F402002094
:1022C80061200008DC020020191E00081804002004
:1022D80005610008091F0008051F0008991E00086D
:1022E80000000301240000200C00002070000020E2
:1022F800080000209921000830040020022804D09A
:10230800402806D10021042001E0002108200CF01B
:10231800B9B97047034B0022C3E902220122C3E97D
:1023280000227047480400200048704748040020F5
:102338004FF0B04382B0DA6C0243DA64DB6C0340DE
:102348000193019B02B070472DE9F04186B000244B
:102358000220154D0594FFF7EBFF0420FFF7E8FF77
:10236800124F03944FF4807601230DEB0001CDE961
:1023780001632846032304934FF4005801F032F810
:1023880001A93846CDF8048001F02CF822464146D0
:10239800384601F047F928462246314601F042F90D
:1023A800204606B0BDE8F081000400480008004857
:1023B800032810B50ED8012810D868B902460B4872
:1023C8004FF4807101F02EF9002209484FF40051B2
:1023D80001F028F9002010BD0122F0E7002203488F
:1023E8004FF4807101F01EF90122EEE70004004865
:1023F80000080048022070470020704701207047FD
:10240800002814BF16200F20704700000D4885468D
:1024180000F025F80C480D490D4A002302E0D45875
:10242800C4500433C4188C42F9D30A4A0A4C002316
:1024380001E013600432A242FBD30CF04BFDFFF71E
:1024480055F8FEE7000001200000002008010020E8
:10245800F4FB000808010020B8210020FEE77047BF
:1024680010B5032000F056FC01F070FA064B186016
:102478000F20FFF735FA044618B9FFF70CF9204684
:1024880010BD0124FBE700BF740000204FF0E022DC
:10249800136923F00203136170474FF0E0221369B8
:1024A80043F0020313617047014BD3F8900570475E
:1024B8000070FF1F014BD3F8940570470070FF1F91
:1024C800014BD3F8980570470070FF1F8068C0F370
:1024D80080007047F7B5002301930446002800F0F8
:1024E800E980856D25B9FEF7FFFCE56584F8545051
:1024F80023689A68D00040F1A1809A68D10000F161
:10250800B480A26D42F01002A265E26D42F00102B1
:10251800E26501251846FFF7D9FFA26D02F0100207
:10252800024340F0C980A26D206922F4817242F012
:102538000202A2659A68D2075DD4226BA67E94F83F
:102548002CC0003A18BF01221703D4E902120A432B
:10255800217E42EA8132617E42EAC13242EA463253
:10256800002842EA4C02B4BF20F000414FF40011A9
:102578003A430A4394F82010012903D1002E76D15A
:1025880042F48032616A21B1A66A01F4E0713143F4
:102598000A43D968E66C21F4FE3121F4FF71114336
:1025A800D96094F83C206168012A01F0404C4CEA5B
:1025B800060609D1D4E910273A433243A66C3243C0
:1025C80042EA0C0242F001061F693E4A3A40324391
:1025D8001A6121F00042B2F1804F0CD0B1F1004FE6
:1025E80009D0394ED6F8082701F4701122F4701278
:1025F8000A43C6F808275A69666BA16B22F00702DE
:1026080032435A615A6922F0700242EA01125A6151
:10261800002835D19A6A62F00F029A625B6903F06A
:1026280007039E423CD10023E365A36D23F0030317
:1026380043F00103A365284603B0F0BD9A68234917
:1026480022F0104222F0170242F080529A60204A8B
:102658001268B2FBF1F2013252000192019A002A8B
:102668003FF44BAF019A013AF7E7002552E7A16D15
:1026780041F02001A165E16D41F00101E16581E7CB
:10268800B0F5001FCAD19A6AE269013A92006FF068
:102698000F0102F01C0201FA02F2216E0A43BCE7A4
:1026A800A36D23F0120343F01003A365E36D43F019
:1026B8000103E3650125BEE7A36D43F01003A3659D
:1026C800F8E700BF02FCFF1F00200140400D030097
:1026D80074000020F8B54569082D04460E460AD056
:1026E8000368DB68D80705D5A36D43F02003A3650D
:1026F8000120F8BD0425FFF7F5F8074623681A6896
:102708002A4220D0A26D42F40072A265DA6812F45F
:10271800406F14D1A27E92B91A6812070FD51846D5
:10272800FFF7D4FE20BB5A6822F00C025A60A26D53
:1027380022F4807222F0010242F00102A265227E98
:10274800FAB10020D5E7711CD9D0FFF7CBF8C01B30
:10275800B04201D8002ED1D123681B682B40CDD1BF
:10276800A26D84F8543042F00402A2650320C0E749
:10277800A26D42F02002A265E26D42F00102E2651C
:10278800DDE70C221A60DCE70368186C704700006C
:10279800F7B50023019390F85430012B044600F05C
:1027A800C08005680269012380F854302846FFF785
:1027B8008DFE002840F0AF80D1E90030022822F0D9
:1027C80004027ED0B2F1004FC3F3110E35D1AA6ACC
:1027D80042EA0E02AA628A68686902EA032222F0C3
:1027E8007C4222F0FF0220EA03210A43002B6A619F
:1027F8001DDA4D4A4D4DD2F80817AB4201F0E07092
:1028080043D10D0213D4D2F8083723F0E073034301
:1028180043F40003C2F80837454B1A68454BB2FB2E
:10282800F3F20C2302FB03330193019B53BB0020FB
:10283800002384F8543003B0F0BD226E00F01F0767
:102848004FF00F0C0CFA07FC6FEA0C0622EA0C0C8E
:10285800BEF1000F11D1C3F38462BA4042EA0C0200
:1028680022668008E26901309042B4D8A86AC3F3AE
:102878008362BA4006403243ACE793FAA3F2B2FA55
:1028880082F2EAE7019B013BCEE72B4DAB420BD12D
:10289800C901CCD4D2F8083723F0E073034343F0DE
:1028A8008073C2F80837C2E7244DAB42BFD14B0250
:1028B800BDD4D2F8083723F0E073034343F4800310
:1028C800EFE7B2F1004F01BFAA6AC3F311018A43CF
:1028D800AA62002BABDA154813498342D1F80827BE
:1028E80009D1D1F8083702F0A07223F0E0731A4337
:1028F800C1F808279BE71048834204D1D1F808376C
:1029080002F44002F1E70D48834290D1D1F808372C
:1029180002F0C072E9E7A26D42F02002A2651846F3
:1029280086E7022087E700BF00200140001000B0C2
:1029380074000020400D0300004000B8002000B4DF
:10294800026838B504461046FFF7C0FD08B90020F4
:1029580038BD9368990707D4936823F0004323F0A0
:10296800170343F010039360FEF7BCFF0546236886
:102978009B685B07EBD5FEF7B5FF401B0228F6D92D
:1029880023689B685A07F2D5A36D43F01003A3652B
:10299800E36D43F00103E3650120D9E773B5002334
:1029A800026801939368DD07044602D5002002B04F
:1029B80070BD9168214B194209D0A36D43F01003F3
:1029C800A365E36D43F00103E3650120EFE7936836
:1029D80023F0004323F0170343F001039360184BDF
:1029E800D3F8083718021CD4637E012BDED0FEF71B
:1029F80079FF144E054622681368DB07D6D493681E
:102A0800D9075FBF9368334043F001039360FEF733
:102A180069FF401B0228EED923681B68DA07EAD44D
:102A2800CBE7094B094A1B68B3FBF2F30133019367
:102A3800019B002BD8D0019B013BF8E717000080D1
:102A480000200140E8FFFF7F74000020400D0300D4
:102A580038B504460068FFF739FD054620BB94F8F1
:102A68005430012B20D0012384F854302046FFF73E
:102A780095FFB0B9A36D226823F4706323F00103B6
:102A880043F48073A3651C23E065136084F8540045
:102A9800936823F0004323F0170343F00403936083
:102AA80038BD84F85450FBE70220F9E7026838B5CE
:102AB800936891680446C80701D4002038BD990777
:102AC800FBD4936803F00503012B19D1936823F015
:102AD800004323F0170343F00203936003231360BA
:102AE800FEF700FF054623689B68DB07E5D5FEF780
:102AF800F9FE401B0228F6D923689B68DA07F2D54D
:102B0800A36D43F01003A365E36D43F00103E36590
:102B18000120D3E770B5044600284BD0836D43F0FD
:102B280002038365FFF70CFF054668B92046FFF7E7
:102B3800BDFF054608B90123A3652268936823F001
:102B4800104323F01703936023685A6822F46772CE
:102B580022F003025A6040F29F321A60D968164A7E
:102B68000A40DA601A6922F040421A615A6922F072
:102B780007025A611A6A02F0F0221A625A6A02F0CF
:102B8800F0225A62DA6A02F0F022DA629A6A0B4A92
:102B980000269E62D2F8083723F0FE73C2F8083781
:102BA8002046FEF7B5F9E6652666A66584F8546002
:102BB800284670BD0125FBE700023E830020014046
:102BC80010B590F85430012B044615D0012380F835
:102BD8005430FFF7B5FE58B92046FFF767FF38B9FC
:102BE800A36D23F4807323F0010343F00103A3656D
:102BF800002384F8543010BD0220FCE7F7B5002309
:102C0800019390F85430012B04467FD0012380F8BB
:102C18005430FFF74BFF23689A6812F0010205460B
:102C280007D0A36D43F01003A365002384F8543044
:102C38002DE0A16D364F21F4817141F00201A165AB
:102C4800DE68D96826F4FF4626F07C0621F40041A8
:102C5800360421F00301360CD96008209968394000
:102C680041F0004199609968002913DA019901310E
:102C780001910199B1F52E3FF5D3A36D23F012030D
:102C880043F01003A365002384F854300125284637
:102C980003B0F0BDD3F8B410013801F07F010A4445
:102CA800DCD199681A48014041F001019960D3F8D4
:102CB800B41021F07F0141EAD202C3F8B4209A6827
:102CC800024042F002029A60FEF70CFE07462368B3
:102CD8009A68D20708D4DA683243DA60A36D23F021
:102CE800030343F001039FE7FEF7FCFDC01B022826
:102CF800EDD923689B68D907E9D5A36D43F0100384
:102D0800A365E36D43F00103E365BFE70225BEE772
:102D1800E8FFFF7F0749CA6822F4E0620302120451
:102D280003F4E063120C134343F0BF6343F400332E
:102D3800CB60704700ED00E0164B30B5DC68C4F39B
:102D48000224C4F10703251D042B28BF0423062DE4
:102D58004FF0FF358CBF033C002405FA03F321EA4A
:102D68000303A54022EA0502A340002843EA020320
:102D7800ACBF00F16040084A4FEA0313B8BF00F047
:102D88000F00DBB2AABF00F56140135480F800338E
:102D980030BD00BF00ED00E014ED00E0002807DBC7
:102DA800044A4109012300F01F00834042F8213002
:102DB800704700BF00E100E000280CDB430906492A
:102DC80000F01F0020330122824041F82320BFF386
:102DD8004F8FBFF36F8F704700E100E070B5D0E907
:102DE80013456560446D14B1D0E916456560D0E9B6
:102DF800105404F01C060124B4406C60046863603D
:102E08008368102B0BBFA260A160E160E26070BD17
:102E18000268416CD3B210B5083B1424B3FBF4F339
:102E28000B4CA24288BF0B4A21F0030199BF01F164
:102E3800804202F50232521807338264064AC2649D
:102E480003F01F03012202FA03F3036510BD00BF5C
:102E5800070402401C0802408008024038B50028D8
:102E68005CD002682E4B9A424FF014014AD82D4B81
:102E78001344B3FBF1F32C499B00C0E91013022360
:102E880080F825301368056923F4FF4323F07003A5
:102E98001360D0E9024323432B43456911682B4350
:102EA80085692B43C5692B43056A2B430B43136084
:102EB800FFF7AEFFB4F5804F04BF002343604368BB
:102EC800816C03F07F020A60D0E91314013B032BE5
:102ED8004C601ED8154B1649816513449B0001218F
:102EE800013A01FA02F200214365C2651960114BEB
:102EF8005A6400230122C36380F8243080F8252017
:102F0800184638BD0C4B1344B3FBF1F30B499B0037
:102F1800B3E70023C0E91533C365EAE70120F0E70A
:102F280007040240F8FFFDBF000002403F82001086
:102F38004009024000090240F8FBFDBF00040240BE
:102F480038B5002841D00268136823F001031360E4
:102F58001F4B9A424FF0140130D81E4B1344B3FB59
:102F6800F1F31D499B00C0E91013012403F01C0371
:102F780004FA03F3002515604B60FFF749FF836CE3
:102F880041681D60D0E913325A604A1E032A06D8E8
:102F9800124B0B449B0094401D60114B5C64002352
:102FA800C363C0E91533C0E90B33C0E90D33C3650A
:102FB80080F8253080F82430184638BD094B134472
:102FC800B3FBF1F308499B00CDE70120F5E700BF0B
:102FD80007040240F8FFFDBF000002403F820010D6
:102FE80000090240F8FBFDBF0004024070B590F8EC
:102FF8002450012D04463BD090F825600125AE42AF
:1030080080F824504FF000062CD1022580F8255076
:103018000568C6632E6826F001062E60FFF7DEFEFF
:10302800036BBBB12B6843F00E032B60A36C1A68CB
:10303800D20342BF1A6842F480721A60636D1BB1F2
:103048001A6842F480721A602B6843F001032B60FF
:10305800002070BD2B6823F004032B602B6843F01D
:103068000A03E2E78023C36380F824602846F0E778
:103078000220EEE7034640B190F82520022A06D048
:103088000422C263002280F82420012070470268CD
:10309800806C116821F00E011160016821F48071C3
:1030A8000160116821F001011160D3E9100202F0FA
:1030B8001C0101228A404260D3E9132151605A6DF4
:1030C80032B1116821F480711160D3E91621516081
:1030D8000122002083F8252083F82400704708B5D2
:1030E80090F82530022B03D00423C363012008BDC8
:1030F80003681A6822F00E021A601A6822F00102A8
:103108001A60826C136823F480731360D0E910137B
:1031180003F01C02012393404B60D0E913325A603C
:10312800436D33B11A6822F480721A60D0E91632FE
:103138005A60012380F82530002380F82430836BFF
:1031480003B198470020D2E770B4426C046C03685E
:1031580026681D6802F01C020421914031420FD0FC
:1031680015F0040F0CD01A6892065EBF1A6822F098
:1031780004021A60036B6160002B33D070BC1847DF
:1031880002219140314217D015F0020F14D01A686D
:10319800940606D41A6822F00A021A60012280F8FE
:1031A8002520114A93428CBF104B114B59600023C4
:1031B80080F82430C36ADFE708219140314211D0FA
:1031C80029070FD5196821F00E011960012303FAA8
:1031D80002F26260C36380F82530002380F824304F
:1031E800436BC9E770BC704780000240000402408E
:1031F800000002400A4A536943F4802330B5536102
:10320800EFF3108472B60023CD58C5500433B3F5DC
:10321800807FF9D11369DB03FCD484F3108830BDB7
:1032280000400058064B5A69002ABFBF054A9A60F9
:1032380002F188329A60BABF5869C00F00207047FF
:103248000040005823016745044B5A6942F0004288
:103258005A615869C043C00F704700BF004000580A
:1032680070B50546FEF73EFB124E04463369D90396
:1032780013D43369DA0744BF012232614CF2FA32BF
:10328800134011D10B4E306910F480200BD0FEF79B
:1032980029FB001BA842F6D304E0FEF723FB001B22
:1032A800A842E3D3032070BD024A1361024A0120F9
:1032B8005360F8E700400058580400202DE9F04119
:1032C800184D98462B78012B06460C46174626D0F3
:1032D80001232B704FF47A7000236B60FFF7C0FF57
:1032E800A0B9012E16D1104A536943F00103536166
:1032F8002760BFF36F8FC4F804804FF47A70FFF72C
:10330800AFFF094A536923EA0603536100232B7070
:10331800BDE8F08139462046FFF76CFFEDE7022053
:10332800F6E700BF5804002000400058054A5369DA
:1033380023F47E7343EAC00040F4803040F002007A
:1033480050617047004000582DE9F041234F3B7809
:10335800012B054688463FD001233B704FF47A7015
:1033680000237B60FFF77CFF044688B92B68042B99
:1033780013D11B4A536943F4803343F00403536168
:103388004FF47A70FFF76CFF0446154B1A681B68F8
:1033980000233B702046BDE8F0814FF0FF33C8F8AA
:1033A80000306E68D5E901321344B3420AD9304679
:1033B800FFF7BCFF4FF47A70FFF752FF50B1C8F81F
:1033C80000600446064A536923F47E7323F002031F
:1033D8005361DAE70136E5E70224DBE75804002009
:1033E800004000582DE9F04F524C00234FF00F09D0
:1033F8000A6832FA03F501D1BDE8F08F012505FA14
:1034080003F818EA020200F08E804E68032706F0DF
:1034180003054FEA430E07FA0EFC6F1E012F6FEAF1
:103428000C0C32D8876807EA0C0ACF6807FA0EF73F
:1034380047EA0A078760476827EA0808C6F30017BB
:103448009F4047EA08074760C76807EA0C088F6883
:1034580007FA0EF747EA0807022DC76017D14FEAA7
:10346800D30800EB880803F0070AD8F820704FEA61
:103478008A0A09FA0AFB27EA0B0B0F6907FA0AF707
:1034880047EA0B07C8F8207001E0032DDCD1076874
:1034980005FA0EF507EA0C073D4316F4403F0560B0
:1034A80041D023F0030707F1804707F5803703F081
:1034B800030CBD684FEA8C0C4FF0070E0EFA0CFE99
:1034C800B0F1904F25EA0E0E2FD01B4DA8422ED0FA
:1034D80005F58065A84214BF0725022505FA0CF5F5
:1034E80045EA0E05BD602568D74316F4801F0CBF5A
:1034F8003D4015432560656816F4001F0CBF3D402C
:1035080015436560D4F8805016F4803F0CBF3D40E9
:103518001543C4F88050D4F88450B60354BF3D40D6
:103528001543C4F88450013362E70025D6E7012526
:10353800D4E700BF0008005800040048374A2DE9C6
:10354800F04F00234FF0010A4FF0070B4FF00F091F
:1035580031FA03F401D1BDE8F08F0AFA03FC1CEA42
:10356800010654D023F0030404F1804404F58034A8
:1035780003F00307A568BF000BFA07F8B0F1904FF6
:1035880008EA050E45D0264DA84244D005F58065C9
:10359800A8420CBF02250725BD40754517D1D2F8B2
:1035A800805025EA0605C2F88050D2F8845025EAF2
:1035B8000605C2F88450156825EA060515605568A1
:1035C80025EA06055560A56825EA0805A560056889
:1035D80003265C0006FA04F423FA06F6254300EBFA
:1035E8008606056003F00705376AAD0009FA05F598
:1035F80027EA05073762856825EA04058560456876
:1036080025EA0C054560C56825EA0404C460013351
:103618009EE70025C0E70125BEE700BF0008005867
:10362800000400480AB181617047816270474369AC
:1036380001EA030221EA030141EA0241816170477C
:10364800044AD168014208B502D0D060FEF756FEA0
:1036580008BD00BF00080058024A136843F480738D
:1036680013607047000400580D4B10B55B690C4699
:1036780028B99A0507D500F039F820B110BD9B0587
:1036880001D400F02BF8074A1369012C23F0040336
:10369800136101D130BFF1E740BF20BF20BFEDE784
:1036A8000004005800ED00E0064A136823F0070301
:1036B80043F003031360044A136943F004031361DE
:1036C80030BF70470004005800ED00E0024B186856
:1036D80000F4C060704700BF00040058024A136835
:1036E80043F4804313607047000400580C4A136881
:1036F80023F4804313600B4B1B6832214B430A4968
:10370800B3FBF1F35169890500D533B9536913F453
:10371800007F14BF032000207047013BF2E700BF81
:10372800000400587400002040420F000B4A136840
:1037380023F0070343F002031360094B1A690128B9
:1037480042F004021A6105D130BF1A6922F004025E
:103758001A61704740BF20BF20BFF6E70004005839
:1037680000ED00E04FF0B0431868C0F340407047E8
:103778004FF0B0431868C0F3400070474FF0B042B4
:10378800536823F47F4343EA0023536070474FF0A4
:10379800B0431868C0F34060704700007FB54FF031
:1037A800B0432C4AD3F80831C0F3031003F00F03D9
:1037B80052F82040284A52F82330B4FBF3F4FFF7BC
:1037C80085FF264B054693E80700B5F5007F04AB57
:1037D80003E9070010D0224B9C4218D303F5B70326
:1037E80003F67F539C4229D903F5741303F510633C
:1037F8009C4225D802230BE01A4B9C4207D91A4B4E
:103808009C421BD903F5370303F5D853F0E700238F
:1038180004AA02EB830353F80C4C144D2B6823F0D5
:10382800070323432B60FEF75DF806462B6803F079
:1038380007039C4206D1002004B070BD0123E7E7CE
:103848000024EAE7FEF74EF8801B0228EED9032091
:10385800F2E700BF28F1000888F1000840F00008EE
:10386800C0CF6A00BFEA21013F93340200400058EC
:103878004FF0B04310B59A68D96812F00C0205D021
:103888000C2A4AD101F00303012B51D14FF0B0416A
:103898002B480B6813F0080306D00B6813F00803D5
:1038A80037D1D1F8941007E00C68240756BFD1F837
:1038B80094300968C3F3032350F82330002A0CBF5F
:1038C800184600204FF0B0418A6802F00C020C2A1A
:1038D8001ED1CA6802F00302022A2ED0032A06D19A
:1038E8000B68184A13F4801F174B18BF13464FF084
:1038F800B042D068D168D268C0F306205843C1F3FB
:1039080002130133B0FBF3F0530F0133B0FBF3F0B4
:1039180010BD0B68C3F30313CEE7042A05D0082AA9
:1039280006D11B6813F4801305D006480023C9E7A5
:1039380000231846C6E70448C4E7024BD7E700BF90
:1039480028F100080024F4000048E80108B5FFF752
:103958008FFF4FF0B043044A9B68C3F3031352F838
:103968002330B0FBF3F008BD88F100082DE9F041E1
:103978000446002853D04FF0B0439D68DE680368C2
:103988009B0605F00C0506F0030668D5026A1DB112
:103998000C2D46D1012E44D1002A40D04FF0B0431F
:1039A800A16A1A68170756BFD3F894301B681B0919
:1039B80003F0F00399421FD90846FFF7EFFE0028ED
:1039C8002DD14FF0B042136843F008031360136819
:1039D800A16A23F0F0030B431360606AFFF7CEFE81
:1039E800FFF7B4FFAB4B1860AB4B1868FDF778FFD7
:1039F800002834D0BDE8F0814FF0B042136843F09E
:103A080008031360136823F0F0030B431360606A24
:103A1800FFF7B4FE0846FFF7C1FE0028E0D00120FA
:103A2800E8E74FF0B043002A54D01A6842F0010288
:103A38001A60FDF757FF0746FFF79AFE002842D0A5
:103A48004FF0B042136843F0080313601368A16A8B
:103A580023F0F0030B431360606AFFF78FFE2368BF
:103A6800D80748D42368990700F18C8023681E077B
:103A780040F1FA80A3694FF0B046002B00F0E180D6
:103A8800D6F89430E16903F01002914200F0C48046
:103A980003F00302022AC2D0D80740F1B380D6F857
:103AA800943023F00103C6F89430FDF71BFF074656
:103AB800D6F89430990740F1A580FDF713FFC31B92
:103AC800112BF5D904E0FDF70DFFC01B0228B3D96F
:103AD80003208FE71A6822F001021A60FDF702FF3F
:103AE8000746FFF745FE0028B9D0FDF7FBFEC01BCF
:103AF8000228F6D9ECE7082D03D00C2D05D1032EAA
:103B080003D16368002BADD189E74FF0B043A168BA
:103B18001A6822F480120A431A606268B2F5803F7C
:103B280010D11A6842F480321A60FDF7DBFE0746AE
:103B3800FFF718FE002895D1FDF7D4FEC01B6428B6
:103B4800F6D9C5E7B2F5041F04D11A6842F4001289
:103B58001A60E6E7196821F480311960196821F4C0
:103B680000111960002AE0D1FDF7BCFE0746FFF7F7
:103B7800F9FD00283FF476AFFDF7B4FEC01B6428BA
:103B8800F5D9A5E7042D236903D00C2D0ED1022EFB
:103B98000CD1002B3FF443AF4FF0B042616953683A
:103BA80023F0FE4343EA016353605FE74FF0B046FA
:103BB800BBB1336843F480733360FDF793FE074667
:103BC80033685A0505D4FDF78DFEC31B022BF7D9C0
:103BD8007EE77368626923F0FE4343EA0263736019
:103BE80044E7336823F480733360FDF77BFE0746B0
:103BF80033685B057FF53AAFFDF774FEC31B022BF4
:103C0800F6D965E74FF0B042E169D2F8943023F075
:103C180010030B43C2F894304FF0B047D7F89430F4
:103C280043F00103C7F89430FDF75CFE0646D7F869
:103C380094309A0718D4FDF755FE831B112BF6D93B
:103C480046E7D6F8943023F00103C6F89430FDF720
:103C580049FE0746D6F894309B0705D5FDF742FE86
:103C6800C31B112BF6D933E72368580754D50B4FDC
:103C78003B68D90514D4FFF7EFFCFDF733FE064681
:103C88003B68DA050CD4FDF72DFE831B022BF7D910
:103C98001EE700BF740000207800002000040058D0
:103CA800E3684FF0B046002B58D023F08003052B73
:103CB80002BFD6F8903043F00403C6F890304FF0B6
:103CC800B046FDF70FFED6F8903043F001030746E3
:103CD800C6F8903041F28838D6F890309B0705D462
:103CE800FDF700FEC31B4345F6D9F1E6E36823F070
:103CF8000403812B1BD1FDF7F5FDD6F8903043F076
:103D08008003C6F8903007464FF0B04641F2883835
:103D1800D6F89030180504D5E36A002B4AD1002064
:103D280068E6FDF7DFFDC01B4045F1D9D0E6FDF799
:103D3800D9FDD6F8903023F08003C6F890300746B6
:103D48004FF0B04641F28838D6F890301905E3D5DF
:103D5800FDF7C8FDC01B4045F6D9B9E6FDF7C2FD21
:103D6800D6F8903023F080030746C6F8903041F229
:103D78008838D6F890301A0516D4FDF7B3FDD6F872
:103D8800903023F00103C6F8903007464FF0B04852
:103D980041F28836D8F890309B07BDD5FDF7A2FDD3
:103DA800C31BB342F6D993E6FDF79CFDC01B404503
:103DB800DFD98DE60C2D4ED0022B4FF0B0431A6898
:103DC80022F080721A6033D1FDF78CFD0546FFF7AB
:103DD800DEFC38BBD4E90C314FF0B0420B43D0685D
:103DE8002D4901400B43E16B0B43216C0B43616C84
:103DF8000B43A16B43EA0123D360136843F080733C
:103E08001360D36843F08053D360FDF76BFD04461D
:103E1800FFF7BDFC002882D1FDF764FD001B0A28CE
:103E2800F6D955E6FDF75EFD401B0A28CFD94FE6C7
:103E3800FDF758FD0446FFF7AAFC30B94FF0B04231
:103E4800164BD1680B40D36069E7FDF74BFD001BAB
:103E58000A28F0D93CE6012B3FF4E1AD4FF0B0431E
:103E6800D868236B00F003029A427FF4D8AD626BE6
:103E780000F0700393427FF4D2ADA26B00F4FE43CE
:103E8800B3EB022F7FF4CBAD636C00F06040C01A37
:103E980018BF0120AEE500BF8C80C111FCFFFEEE0B
:103EA8002DE9F0410D46044610B90120BDE8F08126
:103EB800684E336803F007038B4216D323689A07CA
:103EC80027D54FF0B047A268BB6823F0F00313432F
:103ED800BB60FDF707FD0646BB68DB0319D4FDF799
:103EE80001FD831B022BF7D911E0336823F0070388
:103EF8000B433360FDF7F6FC0746336803F007030E
:103F0800AB42DBD0FDF7EEFCC01B0228F5D903203D
:103F1800CCE72368580617D54FF0B0476269D7F841
:103F2800083123F00F0343EA1213C7F80831FDF7ED
:103F3800D9FC0646D7F80831D90305D4FDF7D2FCD9
:103F4800831B022BF6D9E2E723685A0713D54FF0F3
:103F5800B047E268BB6823F4E0631343BB60FDF736
:103F6800C1FC0646BB689B0305D4FDF7BBFC831B5D
:103F7800022BF7D9CBE72368180714D54FF0B047C1
:103F88002269BB6823F4605343EAC203BB60FDF7B0
:103F9800A9FC0646BB68590305D4FDF7A3FC831B9F
:103FA800022BF7D9B3E72368DA070FD4294C236823
:103FB80003F00703AB4239D8FFF7C8FC264B18605B
:103FC800264BBDE8F0411868FDF78ABC6268022AF2
:103FD8001DD1FFF7C7FB00283FF467AF4FF0B0468D
:103FE80041F28838B36823F003031343B360FDF745
:103FF80079FC0746B368626803F00C03B3EB820FE1
:10400800D4D0FDF76FFCC01B4045F3D97FE7032AE6
:1040180002D1FFF7BCFBDEE712B9FFF7A9FBDAE72D
:104028004FF0B0431B685B05D8D43EE7236823F004
:1040380007032B432360FDF755FC0646236803F06E
:104048000703AB42B8D0FDF74DFC801B0228F5D919
:104058005DE700BF00400058740000207800002091
:1040680008B5FFF773FC4FF0B043044A9B68C3F3ED
:10407800022352F82330D84008BD00BF68F1000879
:1040880008B5FFF763FC4FF0B043044A9B68C3F3DD
:10409800C22352F82330D84008BD00BF68F1000899
:1040A8004FF0B043D3F89000C0F3400070474FF092
:1040B800B0410209D1F8883002F47F22000123EAD6
:1040C800020300F47F200343C1F8883070474FF0A3
:1040D800B041020CD1F88830120423EA020343EA03
:1040E8000040C1F8880070470368DA0370B50446D9
:1040F80039D5FFF7B1FAFDF7F5FB614E0546336890
:10410800DB0532D54FF0B043616BD3F8902002F451
:10411800407291421DD0D3F89010D3F8902042F409
:104128008032C3F89020D3F8902021F4407022F414
:1041380080328D07C3F89020C3F8900009D5FDF7A9
:10414800D1FB41F288360546FFF7AAFF012840F067
:1041580090804FF0B042616BD2F8903023F44073F6
:104168000B43C2F89030002605E0FDF7BBFB401B6F
:104178000228C4D903262568E8070AD54FF0B041BC
:104188006268D1F8883023EA124392B21343C1F827
:104198008830A9070AD54FF0B041A268D1F8883015
:1041A80023EA124392B21343C1F88830AA0609D50C
:1041B8004FF0B0422169D2F8883023F440630B43B2
:1041C800C2F88830AB0502D5206AFFF780FF680582
:1041D80002D5606AFFF77BFF290502D5A06AFFF7C1
:1041E80076FF6A0602D56069FFF761FF2B0602D5E4
:1041F800A069FFF75CFFE80502D5E069FFF757FF04
:10420800E90610D54FF0B042E168D2F8883023F4BF
:1042180040730B43C2F88830B1F5807F02BFD36882
:1042280043F08073D3602A040ED54FF0B042216B5F
:10423800D2F8883023F040430B43C2F8883019B9CC
:10424800D36843F08073D3606B0410D54FF0B0424D
:10425800E16AD2F8883023F040530B43B1F1005F94
:10426800C2F8883003D1D36843F48033D360304632
:1042780070BDFDF737FB401BB0427FF665AF79E7AD
:104288000004005830B590F82C30012B02464FF04E
:10429800020022D0174B82F82D00CA24012582F88B
:1042A8002C505C6253245C62B1F5807F146B996971
:1042B80014D121F488519961596C24F0010421F03A
:1042C800004159641463DD650A4BFF2159620020DF
:1042D800012382F82D3082F82C0030BD21F40851DA
:1042E8009961D96C24F0020421F00041D964146367
:1042F800D865E9E70028004070B50B4E036B756D73
:104308001D40EA07044603D50123F365FDF7FDFBCD
:10431800AB0704D50223F365204600F0C9F9012351
:1043280084F82D3070BD00BF0028004038B50A4C15
:10433800E36823F02003E360FDF7D4FA0546E36859
:104348009B0601D5002038BDFDF7CCFA401BB0F51F
:104358007A7FF4D90320F6E700280040F8B5114D1C
:10436800EC6814F0400406461AD1EB6843F0800369
:10437800EB60FDF7B7FA23460746EC6814F04004F3
:1043880001D1032B01D11846F8BDFDF7ABFAC01BCC
:10439800B0F57A7F234684BF032386F82D30ECE7F7
:1043A8000023F0E70028004038B50F4CE36823F0FD
:1043B8008003E360A3699B06054606D4FFF7B6FFB2
:1043C80010B1032085F82D0038BDA36923F0200320
:1043D800A361FFF7ABFF10B1032085F82D00A36997
:1043E80043F02003A361EFE70028004038B50446F6
:1043F80000284BD090F82D3003F0FF021BB980F84D
:104408002C20FDF7C7F80223214D84F82D30EB68E6
:10441800DB0636D4CA236B6253236B622046FFF750
:104428009DFF10B1FF236B6238BDAB6923F08E632B
:1044380023F04003AB6121696368AA690B43134306
:10444800A2691343AB61D4E9022343EA02432B6117
:10445800D4E90931EA680B4322F4F8521343EB60BC
:104468002046FFF7A1FF0028DCD1D4E90713AA6989
:104478000B4322F06042134362691343AB61FF238D
:104488006B62012384F82D300020CDE70120CBE7B3
:10449800002800400023092803D840EA0310C0B2CE
:1044A80070470A380133C0B2F5E700002DE9F0473C
:1044B80090F82C30012B05464FF0020069D00123FB
:1044C80085F82C304E4B85F82D00DE6806F44076D2
:1044D800B6F5807F78D04C69087891F8019091F80A
:1044E80002A091F82470002A55D19B6913F040036B
:1044F80008BFCB70FFF7CEFF80464846FFF7CAFFDC
:1045080002465046FFF7C6FF81463846FFF7C2FF0E
:104518000B6ACF78234343EA875343EA090343EA04
:10452800084343EA022343EA0063354ACA2050623B
:10453800532050628C6A8869B4F5807F946945D1AC
:1045480024F4885494610124D465B6F5807F09BFAA
:10455800CB6913640343536418BF5064284B4A68FB
:104568001A672A6B42F001022A639A6942F4885258
:104578009A61244AD2F8803043F40033C2F880307C
:104588001F4BFF225A620020012385F82D3085F841
:104598002C00BDE8F087B4F1803F07D0B4F5000FD8
:1045A80004D09B6913F0400308BFCB700B6ACA782C
:1045B8001C4344EA0A0444EA004343EA092343EA61
:1045C800825343EA0763B0E70023AEE724F40854B4
:1045D80094610224D465B6F5807F09BFCB699364E2
:1045E8000343D36418BFD064054B4A685A672A6BE3
:1045F80042F002022A639A6942F40852B8E700BFFF
:10460800002800400008005890F82C20012A034692
:104618004FF0020012D00A4A83F82D00CA215162D5
:1046280053215162916941F020019161FF2151624A
:104638000020012283F82D2083F82C00704700BF4A
:104648000028004090F82C20012A03464FF0020071
:1046580019D00D4A83F82D00CA21516253215162A5
:1046680091690A4841F080019161D0F8801041F4C5
:104678008021C0F88010FF2151620020012283F8B8
:104688002D2083F82C0070470028004000080058AF
:10469800064B5A6D520610B5044603D54022DA651A
:1046A800FDF736FA012384F82D3010BD00280040AC
:1046B8007047890001F1804101F531410A60704776
:1046C800890001F1804101F5314108687047000017
:1046D800034AD2F8903043F40043C2F89030704750
:1046E80000040058034AD2F8903023F40043C2F87B
:1046F8009030704700040058074B1A6822F04002B7
:104708001A6040F441704FF4B85218605A601A6841
:1047180042F040021A6070470000015837B505465C
:1047280000284ED0837903F0FF046BB1032C0BD023
:10473800254B4FF400629A612868FFF7DDFF0024DB
:1047480001232B71AC602FE000236B712846FCF726
:10475800E3FF1E4AD2F8903043F48053C2F89030F9
:10476800002CE5D102234FF0B042AB71D2F894305F
:1047780023F40043C2F89430154B1B681C214B43AB
:10478800DB0C64214B430193019B93B90124AC607A
:10479800FFF79EFF0C4B9A6842F400629A604FF450
:1047A80000629A61002CC7D00123AB71204603B088
:1047B80030BD019B013B0193D2F894305B04E3D4F4
:1047C800E6E70124F2E700BF00040058000800589B
:1047D8007400002037B5174D2B6802461C20434350
:1047E800DB0C6420434314480193019B93B90120D7
:1047F8009060114C21732B681C214B43DB0C642106
:104808004B430193019B6BB9012090600A4BDB6815
:1048180003B030BD019B013B019383689C07E4D53D
:104828000020E6E7019B013B0193A368DB07E9D57C
:10483800ECE700BF740000200000015837B5184DA0
:104848002B6802461C204343DB0C64204343154875
:104858000193019BA3B901209060124CFF2323739D
:104868002B681C256B43DB0C64256B430193019B70
:1048780073B9012090600B4BDB680B7003B030BD3F
:10488800019B013B019383689C07E2D50020E4E784
:10489800019B013B0193A368DB07E8D5EBE700BF69
:1048A80074000020000001580E4B0F491B681822A5
:1048B800534382B01B0D6422534301934B69019A01
:1048C800C3F3800322B902238360012002B070473A
:1048D800019A013A01924A69920701D5002BEDD15C
:1048E8000020F3E7740000200004005807B503799E
:1048F800012B0FD10A4B1B68182253431B0C019341
:10490800FFF7F0FE019B013B0193019B002BF9D1BE
:10491800FFF7DEFE03B05DF804EBFFF7C5BF00BF8D
:1049280074000020F8B51E468379012B154604460D
:104938000F46DAB22DD14379012B2AD002234271D6
:104948008371FFF7D3FF0D212046FFF7CBFEFFF75A
:1049580041FF390A2046FFF73DFFF9B22046FFF72D
:1049680039FF2E44B5420ED12046FFF7B1FEFFF7BE
:104978009BFFA06801230038A3714FF0000318BF04
:1049880001206371F8BD15F8011B2046FFF722FFCF
:10499800E8E70220F6E7F8B51E468379012B1546AD
:1049A80004460F46DAB22FD14379012B2CD042713D
:1049B800FFF79CFF1D212046FFF794FEFFF70AFF33
:1049C800390A2046FFF706FFF9B22046FFF702FF33
:1049D80000212046FFF7FEFE2E44B5420ED12046A8
:1049E800FFF776FEFFF760FFA06801230038A37188
:1049F8004FF0000318BF01206371F8BD2946204617
:104A0800FFF71CFF0135E8E70220F6E7F8B51F4677
:104A18008379012B154604460E46DAB22CD1437928
:104A2800012B29D04271FFF761FF06F0EF03A3F1D4
:104A3800840253425341237131462046FFF752FE08
:104A4800FFF7C8FE2F44AF4210D1FFF741FE842E76
:104A580002D02046FFF728FFA06801230038A37181
:104A68004FF0000318BF01206371F8BD15F8011B52
:104A78002046FFF7AFFEE6E70220F6E7F8B51E4648
:104A88008379012B154604460F46DAB227D14379BC
:104A9800012B24D04271FFF729FF39462046FFF742
:104AA80021FEFFF797FE00212046FFF793FE2E44D4
:104AB800B5420ED12046FFF70BFEFFF7F5FEA068C2
:104AC80001230038A3714FF0000318BF0120637160
:104AD800F8BD29462046FFF7B1FE0135E8E7022078
:104AE800F6E737B50023ADF8043001AA02231221F6
:104AF8000546FFF7C3FFBDF80440022364BA01AAC4
:104B0800A4B219462846FFF781FFE20702D52846D6
:104B180009F03EFBA30702D5284609F03FFB6007D2
:104B280002D5284609F064FB210702D5284609F07A
:104B380065FBE20602D5284609F066FBA30602D506
:104B4800284609F04FFB600602D5284609F02CFBE1
:104B5800210606D514F4807118BF0121284609F0F2
:104B680029FBA20502D5284609F034FB630402D5C7
:104B7800284609F04FFB03B030BDF8B51E468379CF
:104B8800012B154604460F46DAB227D14379012B8B
:104B980024D04271FFF7AAFE0E212046FFF7A2FD9E
:104BA800FFF718FE39462046FFF714FE2E44B5429B
:104BB8000ED12046FFF78CFDFFF776FEA068012393
:104BC8000038A3714FF0000318BF01206371F8BDCE
:104BD80015F8011B2046FFF7FDFDE8E70220F6E780
:104BE800F8B51E468379012B154604460F46DAB2FE
:104BF8002BD14379012B28D04271FFF777FE1E2174
:104C08002046FFF76FFDFFF7E5FD39462046FFF721
:104C1800E1FD00212046FFF7DDFD2E44B5420ED10F
:104C28002046FFF755FDFFF73FFEA0680123003837
:104C3800A3714FF0000318BF01206371F8BD294626
:104C48002046FFF7FBFD0135E8E70220F6E702689A
:104C580052E8003F23F0C00342E80031026800290F
:104C6800F5D102F1080353E8003F23F4000302F1F1
:104C7800080C4CE800310029F3D12023C0F8883013
:104C88007047000010B5026852E8003F23F49073A3
:104C980042E8003102680029F5D10F4C02F10803FF
:104CA80053E8003F234002F1080C4CE8003100298A
:104CB800F4D1C36E012B07D152E8003F23F0100353
:104CC80042E800310029F7D12023C0F88C300023B6
:104CD800C366436710BD00BFFEFFFFEF38B505464A
:104CE800C8B12423C0F8883003681A68002422F069
:104CF80001021A601C605C609C60FCF7B5FFC5F897
:104D0800904085F88440C5F888402046C5F88C4016
:104D1800EC662C6738BD0120FCE70000F8B50446B6
:104D28001346D4F88850202D32D1F1B1EAB1E06FA2
:104D3800A4F85620A4F8542000262122C4F8906034
:104D48002165C4F88820226888B1124FC762124FC3
:104D58000763124F2832C0E90D76FEF747F930B1E4
:104D68001023C4F89030C4F888500120F8BD236897
:104D780040221A62226802F1080353E8003F43F018
:104D8800800302F1080141E800300028F3D1EDE783
:104D98000220EBE7A94D0008F14D0008FD4D000881
:104DA80008B50346806A1B681B6813F0200317D1F7
:104DB800A0F85630026802F1080353E8003F23F0D8
:104DC8008003083242E8003102680029F2D152E833
:104DD800003F43F0400342E800310029F7D108BD05
:104DE800FCF7BCFFFBE7704708B5806AFFF7FBFFDD
:104DF80008BD7047806A38B50468D0F88830D0F8A4
:104E08008C50A268120606D5212B04D10023A0F8E5
:104E18005630FFF71CFFA3685B0606D5222D04D188
:104E28000023A0F85E30FFF72DFFD0F8903043F054
:104E38001003C0F89030FFF7DCFF38BD08B5806A72
:104E48000023A0F85E30A0F85630FFF7D2FF08BD67
:104E5800704700000368D9691A682DE9F04140F6E7
:104E68000F0631429D68044610D18E0640F19780A6
:104E780002F0200605F080573E4300F09080436F13
:104E8800002B00F08580BDE8F0411847AB4EAC48D8
:104E98002E401040304300F08280CF0709D5D0055E
:104EA80007D501201862D4F8900040F00100C4F83A
:104EB80090008F0709D5E80707D502201862D4F8B3
:104EC800900040F00400C4F890004F0709D5E807A7
:104ED80007D504201862D4F8900040F00200C4F806
:104EE80090000F070BD502F02000304307D00820B0
:104EF8001862D4F8900040F00800C4F890000E053D
:104F08000AD5500108D54FF400601862D4F89030E3
:104F180043F02003C4F89030D4F89030002B37D0F9
:104F28008B0609D502F0200205F080552A4303D0EC
:104F3800636F0BB1204698472668D4F89020B36871
:104F480002F0280203F0400353EA0205204621D06C
:104F5800FFF798FEB3685F0617D5226802F10803C9
:104F680053E8003F23F04003083242E800310029AB
:104F7800F3D1D4F8800040B1724B8363FEF7AFF8E9
:104F880030B1D4F88000836B7DE72046FFF731FF0E
:104F9800BDE8F081FFF72DFFC4F89050F8E7E06E08
:104FA800012840F08980CE0640F18680D00640F185
:104FB800838010221A629A6851064BD5D4F8802053
:104FC80011684A6892B2002AE2D0B4F85C009042B4
:104FD800DED9A4F85E200A6892062FD453E8002F81
:104FE80022F4807243E800210029F7D103F1080276
:104FF80052E8002F22F0010203F1080040E80021E6
:105008000029F3D103F1080252E8002F22F04002F0
:1050180003F1080040E800210029F3D12022C4F858
:105028008C20E16653E8002F22F0100243E80021AB
:105038000029F7D1D4F88000FEF71CF80223236773
:10504800B4F85E30B4F85C10C91A89B22046FFF78C
:10505800FFFE9DE7B4F85E20B4F85E00B4F85C107B
:1050680080B292B2002893D0891A89B200298FD0D1
:1050780053E8002F22F4907243E800200028F7D16B
:10508800314D03F1080252E8002F2A4003F10806C7
:1050980046E800200028F4D12022C4F88C2060675C
:1050A800E06653E8002F22F0100243E800200028B1
:1050B800F7D102232367C9E7CF0209D56E0207D5C6
:1050C8004FF4801220461A62BDE8F04100F0A0BDFE
:1050D80008060BD502F0800005F40005284305D02A
:1050E800A36F002B3FF454AF2046CCE64F0611D5F2
:1050F80056060FD553E8002F22F0400243E800215E
:105108000029F7D12023C4F88830A1672046FCF78E
:1051180025FE3DE70D0206D5500004D52046BDE822
:10512800F04100F077BDCB017FF532AF002ABFF622
:105138002FAF2046BDE8F04100F06BBD0100001024
:1051480020010004454E0008FEFFFFEFD0F88C2038
:10515800B0F86010222A08B5036855D15B6A826DE1
:105168000B401370836D01338365B0F85E30013BEB
:105178009BB2A0F85E30B0F85E309BB2002B42D1F3
:10518800026852E8003F23F4907342E80031036854
:105198000029F5D103F1080252E8002F22F001029C
:1051A80003F1080C4CE800210029F3D12022C0F8B3
:1051B8008C20184A41679342016705D1C26E012AC3
:1051C8000ED0FCF7D9FD1EE05A681102F6D553E857
:1051D800002F22F0806243E800210029F7D1EDE793
:1051E8000022C26653E8002F22F0100243E8002193
:1051F8000029F7D1DA69B0F85C10D20644BF102252
:105208001A62FFF725FE08BD9A6942F008029A6102
:10521800F9E700BF00800040D0F88C20B0F860109B
:10522800222A08B5036852D15A6A1140826D22F8C1
:10523800021B8265B0F85E20013A92B2A0F85E20A7
:10524800B0F85E2092B2002A40D153E8002F22F431
:10525800907243E800210029F7D103F1080252E8CF
:10526800002F22F0010203F1080C4CE8002100296C
:10527800F3D12022C0F88C20174A41679342016776
:1052880005D1C26E012A0ED0FCF776FD1EE05A68E1
:105298001102F6D553E8002F22F0806243E800217E
:1052A8000029F7D1EDE70022C26653E8002F22F06B
:1052B800100243E800210029F7D1DA69B0F85C1040
:1052C800D20644BF10221A62FFF7C2FD08BD9A69D0
:1052D80042F008029A61F9E7008000402DE9F84F92
:1052E8000368B0F86060D3F81CB01F689D68D0F8F8
:1052F8008C20222A044640F0B980B0F8683043B1C7
:10530800DFF87491DFF874A14FF000081BF0200F4C
:1053180020D1B4F85E309BB2D3B1B4F868209A4279
:1053280016D9226802F1080353E8003F23F080539E
:10533800083242E8003122680029F2D1504B6367F5
:1053480052E8003F43F0200342E800310029F7D13A
:10535800BDE8F88F2368A26D5B6A33401370A36DB4
:105368000133A365B4F85E30013B9BB2A4F85E300C
:105378002368D3F81CB01BF0070F2ED01BF0010FC9
:1053880009D0F90507D501221A62D4F8902042F015
:105398000102C4F890201BF0020F09D0EA0707D5D4
:1053A80002221A62D4F8902042F00402C4F8902035
:1053B8001BF0040F09D0E80707D504221A62D4F8B5
:1053C800903043F00203C4F89030D4F8903023B101
:1053D8002046FFF70EFDC4F89080B4F85E309BB20B
:1053E800002B93D1226852E8003F23F4807342E8EF
:1053F800003123680029F5D103F1080252E8002F93
:1054080002EA090203F1080040E800210029F3D16B
:1054180020225345C4F88C20616721670AD05A6856
:10542800110207D553E8002F22F0806243E80021DB
:105438000029F7D1E26E012A14D10022E26653E86E
:10544800002F22F0100243E800210029F7D1DA6981
:10545800B4F85C10D20644BF10221A622046FFF747
:10546800F7FC53E72046FCF787FC4FE79A6942F0C0
:1054780008029A616CE700BFFEFFFFEF0080004062
:10548800555100082DE9F84F0368B0F86060D3F86B
:105498001CB01F689D68D0F88C20222A044640F072
:1054A800B780B0F8683043B1DFF87091DFF870A1C9
:1054B8004FF000081BF0200F20D1B4F85E309BB2EB
:1054C800D3B1B4F868209A4216D9226802F10803C9
:1054D80053E8003F23F08053083242E80031226845
:1054E8000029F2D14F4B636752E8003F43F0200395
:1054F80042E800310029F7D1BDE8F88F2368A26D92
:10550800596A314022F8021BA265B4F85E20013ABC
:1055180092B2A4F85E20D3F81CB01BF0070F2ED06F
:105528001BF0010F09D0F90507D501221A62D4F83A
:10553800902042F00102C4F890201BF0020F09D01D
:10554800EA0707D502221A62D4F8902042F0040232
:10555800C4F890201BF0040F09D0E80707D50422EF
:105568001A62D4F8903043F00203C4F89030D4F8AB
:10557800903023B12046FFF73CFCC4F89080B4F883
:105588005E309BB2002B95D1226852E8003F23F48D
:10559800807342E8003123680029F5D103F108023D
:1055A80052E8002F02EA090203F1080040E800214E
:1055B8000029F3D120225345C4F88C206167216764
:1055C8000AD05A68110207D553E8002F22F08062EA
:1055D80043E800210029F7D1E26E012A14D1002204
:1055E800E26653E8002F22F0100243E80021002968
:1055F800F7D1DA69B4F85C10D20644BF10221A62F7
:105608002046FFF725FC55E72046FCF7B5FB51E798
:105618009A6942F008029A616EE700BFFEFFFFEF49
:10562800008000402152000838B50446036821690B
:10563800A2681D68C0690A4361690A437749024341
:1056480029400A431A605A68E16822F440520A4322
:105658005A60734AA16993421CBF226A11439A682F
:1056680022F06E4222F430620A439A60DA6A616A72
:1056780022F00F020A43DA626A4A934219D14FF0C4
:10568800B043694AD3F8883003F0030343F4403346
:10569800934200F0B480B3F1031F24D0013A93423F
:1056A80040F0B580B0F5004F40F08F80FEF7E0F88D
:1056B8006EE05E4A93421CD14FF0B0435C49D3F888
:1056C800883003F00C0343F440228A4200F09780AC
:1056D80006D8002B7CD0574B9A42E3D0012026E015
:1056E800B2F10C1FFAD1B0F5004F53D04FF400407F
:1056F80075E04B4A9342F1D14FF0B043D3F888306C
:1057080003F44063B3F5006F18D006D85BB1B3F566
:10571800806FE3D1FEF7ACF807E0B3F5406FDDD159
:105728004FF400400BE0FEF79BFC40B900204FF01F
:105738000113A3660023C4E91D3338BD3E486568DC
:105748003E4B626A05EB450133F81220B0FBF2F3D9
:105758009942C3D8B3EB053FC0D800231946FBF7DD
:105768001FFA090241EA10616B080002C0182A46B4
:105778004FF0000341F10001FBF712FA304BA0F59E
:1057880040729A42AAD82368D860CFE7FEF768FC2F
:105798000028CBD06168294B626A33F81220B0FB2D
:1057A800F2F24B0803EB42034FF6EF72B3FBF1F34F
:1057B800A3F11001914291D823F00F02216892B20F
:1057C800C3F342031343CB60B0E7FEF751F804E09C
:1057D800B0F5004FDAD0FEF743FC0028A6D0636886
:1057E800616A164A32F81120B0FBF2F000EB530060
:1057F800B0FBF3F04FF6EF73A0F11002C1E7B0F57C
:10580800004F0D48EBD1C5E7FEF73AFCC0E7B0F50D
:10581800004FF9D0FEF734FCDFE700BFF369FFCF94
:1058280000800040003801400200030000440040AE
:1058380008000C0004000C000024F400C8F1000863
:10584800FFFC0F00836ADA0710B506D50168C46A41
:105858004A6822F4003222434A609C0706D5016850
:10586800046B4A6822F4803222434A60590706D5FD
:105878000168446B4A6822F4802222434A601A076E
:1058880006D50168846B4A6822F4004222434A60C4
:10589800DC0606D50168C46B8A6822F4805222436C
:1058A8008A60990606D50168046C8A6822F4005259
:1058B80022438A605A060FD50168446C4A6822F46C
:1058C80080122243B4F5801F4A6005D14A68846C6F
:1058D80022F4C00222434A601B0606D50268C16C46
:1058E800536823F400230B43536010BD2DE9F8439C
:1058F800DDF8209005460F46164698462A68D36973
:1059080037EA03030CBF01230023B34201D0002070
:1059180029E0B9F1FF3FF2D0FBF7E4FFA0EB080064
:1059280048452C6802D8B9F1000F1ED154E8003F51
:1059380023F4D07344E80032002AF7D104F10803B5
:1059480053E8003F23F0010304F1080141E8003265
:10595800002AF3D12023C5F88830C5F88C300023FD
:1059680085F884300320BDE8F88323685A07C5D535
:10597800E3691B05C2D54FF40063236254E8003F76
:1059880023F4D07344E80032002AF7D104F1080365
:1059980053E8003F23F0010304F1080141E8003215
:1059A800002AF3D12023C5F88830C5F88C30C5F813
:1059B8009030D4E773B504460026C0F89060FBF732
:1059C80091FF23681B681A07054619D423681B68CA
:1059D8005B070AD56FF07E43009300222B464FF4F5
:1059E80080012046FFF782FFB0B900202023C4F8C9
:1059F800883084F88400C4F88C30E06620670CE0B6
:105A08006FF07E430093324603464FF40011204660
:105A1800FFF76CFF0028D9D0032002B070BD10B585
:105A2800044650B3D0F888301BB980F88430FCF7AE
:105A3800ABF822682423C4F88830136823F00103E4
:105A480013602046FFF7F0FD012816D0A36A13B1B2
:105A58002046FFF7F7FE23685A6822F490425A60FE
:105A68009A6822F02A029A601A6842F001022046D7
:105A78001A60BDE81040FFF79DBF012010BD00006F
:105A880030B581658168A0F85C200023B1F5805F9E
:105A9800A0F85E20436735D10369002B40F2FF135D
:105AA80018BFFF23A0F860300023C0F890302223ED
:105AB800C0F88C30016801F1080353E8003F43F057
:105AC8000103083141E800340368002CF2D1456E27
:105AD80084680169B5F1005F32D1B0F86850954229
:105AE8002ED8B4F5805F244A03D1244C002908BF7E
:105AF80022464267B1B153E8002F42F4807243E86E
:105B08000021F7E729B90369002B14BF7F23FF237E
:105B1800C8E7B1F1805FC5D10369002B14BF3F23EB
:105B28007F23BFE703F1080252E8002F42F08052BA
:105B380003F1080040E800210029F3D1002030BD1E
:105B4800B4F5805F0E4A03D10E4C002908BF2246E7
:105B5800426741B153E8002F42F4907243E80021B4
:105B68000029F7D1EAE753E8002F42F0200243E882
:105B780000210029F7D1E1E7E55200088D5400081B
:105B88005551000821520008D0F88C30202B30B431
:105B980015D1B9B1B2B100230468C3660A4B9C425F
:105BA8000AD063681B0207D554E8003F43F08063BE
:105BB80044E80035002DF7D130BCFFF761BF022063
:105BC80030BC70470120FBE700800040436E30B5D1
:105BD8002BB90123A0F86A30A0F8683030BD0368FB
:105BE800094D9A689968094C490FC2F342626B5C87
:105BF800615CDB00B3FBF1F3A0F86A30AB5CA25C3C
:105C0800DB00B3FBF2F3E7E7E8F10008E0F1000896
:105C18007047704770471FB504AB03E9060090F85A
:105C28008430012B04463AD0012380F884302423A1
:105C3800C0F8883003681A6822F001021A609A686E
:105C480022F440120A439A6071B95A68BDF80C00F0
:105C58009DF80E1022F0100202435A605A6822F092
:105C68007F4242EA01625A601A6842F001021A60F1
:105C7800FBF738FE6FF07E42034600924FF4800136
:105C880000222046FFF732FE38B92023C4F88830B6
:105C9800002384F8843004B010BD0320F8E7022004
:105CA800F9E790F88430012B0FD0012380F8843075
:105CB800016851E8002F42F0020241E80023002B5E
:105CC800F6D180F88430184670470220704710B526
:105CD80090F88430012B044617D02423C0F888306C
:105CE80003681A68196821F00101196042F000522E
:105CF8004FF0005141661A60FFF768FF2023C0F893
:105D08008830002084F8840010BD0220FCE770B5BC
:105D180090F88430012B044617D005682423C0F876
:105D280088302E682B6823F001032B60AB6823F0C2
:105D380060431943A960FFF749FF20232E60C0F88C
:105D48008830002084F8840070BD0220FCE7000041
:105D580038B5084D052455F8043B2BB9013C14F01F
:105D6800FF04F8D1204638BDDB6898470028F5D0F5
:105D7800F9E700BFAC050020034BD870034B1B6844
:105D88001B6C03B11847704794050020900500204C
:105D9800034B1874034B1B685B6C03B118477047BF
:105DA8009405002090050020F0B5314D314B95F950
:105DB8000420314E91B00C46012795F905108DF855
:105DC800047002288DF809208DF80A1010D18DF87A
:105DD8000800D8711C7202F063FD337803B114B166
:105DE80001A803F0C1F9254B059A1A6011B0F0BD5E
:105DF80059714FF480711A71D9801C7233788DF8FB
:105E0800087053BB1F2306A88DF81C208DF8183086
:105E180002F024FF20238DF8183006A82B798DF87E
:105E28001C3002F01BFF22238DF8183006A86B796E
:105E38008DF81C3002F012FF21238DF8183006A8C7
:105E48006B798DF81C3002F009FF29238DF8183082
:105E580006A80B4B079302F001FF02F021FD012376
:105E680006A88DF818308DF81C3002F0F7FEB4E75C
:105E780094050020AC000020700400206405002078
:105E8800000400017FB5092301A88DF8043003F050
:105E98006BF90038044B059A1A6018BF012040427C
:105EA80007B05DF804FB00BF6405002070B5044628
:105EB8000B46144962784A700020A2780A7208706A
:105EC8001A884A729A788A72DB780B746368CB6096
:105ED8000D4B1B68DA6A2AB1237803F0FB030A2BFF
:105EE80000D09047094E002556F8043B1BB15B6A69
:105EF8000BB1204698470135EBB2052B6DB2F3D1B3
:105F080070BD00BF7C00002090050020AC0500207B
:105F180070B5044611480123037063784370A37871
:105F28008372E368C360E378037623694376237951
:105F380043720B4B1B689B6A03B19847094E0025B7
:105F480056F8043B1BB19B690BB1204698470135B5
:105F5800EBB2052B6DB2F3D170BD00BF90000020ED
:105F680090050020AC050020014B1868704700BF61
:105F78006405002000B58BB0012368468DF8003019
:105F880002F046FD38B99DF80400003818BF01201A
:105F98000BB05DF804FB0020FAE7000008B501F03B
:105FA80037FE40B9FFF7E6FF012806D0054B197AFE
:105FB800D879FFF7F9FE012008BDBDE80840FFF7D2
:105FC800C7BE00BFAC0000202DE9F04186B00546F1
:105FD8000E46174601F01CFE002873D101F030FE72
:105FE800044640B9FFF7C6FF01280AD03D4B197A8D
:105FF800D879FFF7D9FE6FF00204204606B0BDE855
:10600800F081DFF8E48088F80860003E18BF0126B8
:106018008DF80460354E687833798DF8123069460A
:1060280002F094FC00283FD08DF804400394ADF8AA
:1060380010406FF0060495E803002D4B83E8030039
:10604800337988F80A30394601A803F091F9294BC9
:10605800059A1A6011283FD801A353F820F000BF11
:10606800D3600008CD600008E1600008E160000826
:10607800E1600008E1600008E1600008FF5F0008D7
:10608800E1600008E1600008E1600008C7600008FE
:10609800E1600008E1600008CD600008CD600008FC
:1060A800CD600008E76000082B788DF808306B7821
:1060B800ADF810306B6803934FF0FF34BBE76FF017
:1060C80005049AE76FF0010497E70B4B00221A705A
:1060D800E31D18BF144690E74FF0FF348DE76FF0CB
:1060E80004048AE7AC0000209000002094050020FA
:1060F800A0000020640500206305002037B501F0EA
:10610800A9FD134D052455F8043B4BB11A693AB162
:106118009B682BB1984718B155F8043C1B69984700
:10612800013C14F0FF04EED1FFF712FE68B9094DE7
:106138002B7853B1084BADF80040D978019422462A
:106148006846FFF741FF00B92C7003B030BD00BFAF
:10615800AC050020630500209405002030B58BB005
:10616800044601F055FD0546002835D1FFF702FF2A
:10617800012834D168468DF8005002F049FC40BB34
:106188009DF80430A34204D0012C22D0022C12D056
:1061980014B100200BB030BD002BFAD068468DF842
:1061A800044002F05BFDA0B90E4B1B681B6B002B73
:1061B800EFD09847EDE763B968468DF8044002F0E0
:1061C8004DFD30B9074B1B681B6B002BE1D02046F7
:1061D800EFE74FF0FF30DDE76FF00100DAE76FF02F
:1061E8000200D7E79005002010B504468AB018B918
:1061F8004FF0FF300AB010BD002368468DF800301C
:1062080002F006FC0028F3D19DF804302370F1E772
:106218007FB500220B4620498DF8072001220A701D
:1062280042784A700446002A33D102790A721A88E1
:106238004A729A788A72DB780B740369CB60C378E8
:10624800164D8DF80830037B8DF809308368039369
:106258002B68DB6A0BB102A898472B689B6B13B1BC
:10626800227E02B198470E4E052556F8043B1BB115
:10627800DB690BB120469847013D15F0FF05F4D1C5
:106288000DF10700FFF7B0FF637913B1054B012249
:106298001A7004B070BD00BF7C000020900500207B
:1062A800AC0500206305002010B504468AB018B973
:1062B8004FF0FF300AB010BD202368468DF800303B
:1062C80002F0A6FB0028F3D1024A9DF9043023709E
:1062D8001371EFE79405002000B58BB023230190DC
:1062E80068468DF8003002F0B9FC003818BF01206C
:1062F80040420BB05DF804FB70B5654C01468EB0AA
:106308001822204606F0C0F8624B00221A70FCF7EB
:106318000BF823784068012202FA03F1014004D106
:106328005D4B084608F09CF8FEE75C495C481A4655
:1063380002F0F8F818B14FF0FF300EB070BD272307
:1063480004A88DF8103002F089FC564E564D0028EE
:1063580070D1012333702B68DB690BB1002098479B
:10636800272304A88DF8103002F052FB059B93F800
:106378004820227093F8182193F81A316270A3709C
:10638800464BD3E9020105F06FFF05460028D2D13C
:10639800464E062304A88DF8103002F039FB059B01
:1063A800736104A802F05AFC022304A88DF8103087
:1063B800059602F02DFB0836032304A88DF810304B
:1063C800059602F025FB0F2606F014F8012304A811
:1063D8008DF814308DF8106002F040FC10230DEB9E
:1063E80003008DF810308DF8145002F037FC0423A8
:1063F8008DF8103004A8A3788DF8143002F02EFC24
:106408003A238DF8103004A86369059302F026FC3E
:1064180002A920788DF8086004F09CF8003818BFAD
:106428000120E0711420FFF757FFE07903F062F9CB
:10643800284682E728238DF810302B681B6943B162
:1064480004A802F0E5FA2B6805981B6940F2C451CC
:106458009847272304A88DF8103002F0FFFB50B9A5
:10646800012304A88DF8103002F0D2FA9DF81430F8
:10647800002B7FF46EAF3378002B7FF46CAF0522CE
:1064880004A88DF81020059302F0E8FB78E700BF18
:106498009405002063050020F0F10008680500203D
:1064A800800500207004002090050020D005002001
:1064B80037B500230D4601930446D0B900F0A8FB78
:1064C8000190019BD3B10F4A42F824300E4A9A62D8
:1064D8000E4A1268916B1963916C596392690C4961
:1064E800D9625A6128465B680A49F2229847002017
:1064F80006E001A900F092FB0028E2D04FF0FF303F
:1065080003B030BDAC050020B15D00089005002047
:106518008D5E000871040020194B07B51860194BEF
:10652800194A1A60194A5A60194A9A60194ADA606F
:10653800194B02681A6042685A6082689A60C26899
:10654800DA60164A1A6182695A61154BC26B5A6041
:10655800144A019119609A601946134ADA600020BA
:10656800FFF7A6FF48B901A800F056FB003818BF8E
:106578000120404203B05DF804FB4FF0FF30F9E71B
:106588009005002080050020195F000819620008A6
:106598002D660008B55E0008680500200DA50008F6
:1065A800C0050020815D0008995D000849B118B157
:1065B800012804D000207047034B0B60FAE7034B17
:1065C800FBE74FF0FF3070470004000101000102B3
:1065D80008B503F0ABF8002814BF6FF001000020E5
:1065E80008BD08B502F084F9002814BF6FF0010057
:1065F800002008BD10B504468AB018B94FF0FF3026
:106608000AB010BD212368468DF8003002F000FA68
:106618000028F3D1024A9DF9043023705371EFE743
:10662800940500202DE9F0412F4D304F00232B70A9
:1066380043786B703B689B6A8AB004460BB1284666
:106648009847DFF8AC80002658F8043B1BB11B6A5A
:106658000BB1204698470136F3B2052B76B2F3D139
:106668002378052B2FD00B2B35D0012B25D1214C8E
:10667800062368468DF8003002F0CAF90199E079DE
:1066880005F038FE10B91C4B019A5A611B48FFF7F8
:106698000BFE1B48FFF7AEFF6B788BB9A371194B44
:1066A8005878FFF75BFD3B685B6A0BB11148984768
:1066B8006B7813B9E07905F0AFFE0AB0BDE8F08158
:1066C800FF23A371EFE7104B01225A74227A9A74C0
:1066D800627ADA74F1E76378002BEED00AB0BDE88D
:1066E800F041FFF7CFBB00BF9000002090050020CD
:1066F800AC050020AC000020D0050020B000002030
:10670800B1000020940500207C00002030B58BB03B
:10671800FFF767FF0446F0B903F0FCFE831C1DD0A9
:10672800F8B9134D2B685B69DBB1272368468DF8F0
:10673800003002F06DF92B6801985B694FF4B9617C
:10674800984703F0F9FE78B92CB9094B1B68DB6947
:106758000BB10120984720460BB030BD6FF00704FD
:10676800EFE74FF0FF34ECE74FF0FF34F3E700BFFB
:1067780090050020014B1878704700BF04060020E0
:10678800014B5878704700BF04060020704700008E
:10679800044B9A7A0AB101225A70034B5B6903B120
:1067A8001847704704060020B800002073B5224C33
:1067B8006378002B33D008F03BF966680546FFF78D
:1067C800D3FB0644AE4214D2A37A93B1E0228DF8EB
:1067D80000208DF80130217AE36801930122684690
:1067E800FFF7F2FB08B1073010D100236370A372E2
:1067F800656094F83430EBB1002384F834300F4BE3
:106808005B6BBBB102B0BDE87040184740F2DC5189
:106818000B4808F0D9F90A4808F09CF9E8E794F819
:106828003520002AE5D094F8360084F83530FFF793
:1068380095FCDEE702B070BD04060020B800002019
:10684800E805002037B5104D104CC8B1C1B16272CF
:10685800012300222860E16023700D480D4B00924F
:106868004FF0FF3108F0CAF800250B482582202296
:10687800294605F01DFE6570A574A58603B030BDD8
:1068880000232B602370EFE7000600200406002099
:10689800E805002099670008180600202DE9F04750
:1068A8008E4C23788CB0002B56D0C2780AB9837BE3
:1068B80013B1238A01332382437B002B4CD0E02A77
:1068C8004AD10023A372876897F80080B8F1220F95
:1068D80027D8B8F1220F30D8DFE818F04100FB00C4
:1068E80052005A0061006E0075008E009D00B400D1
:1068F800C7002F002F002F002F002F002F002F0080
:106908002F002F002F002F002F002F002F002F0007
:106918002F002F002F002F002F002F00C900D000BC
:10692800D400B8F17E0F00F0CC80B8F17F0F00F0F2
:10693800DF80B8F17D0F00F0AB80A57A002D00F064
:106948005B81674C637A3BB94FF47A71204608F053
:106958003BF9204608F0FEF80CB0BDE8F087E36884
:1069680001220021A2721970A37AE1689818A07216
:106978000620C854A37AE1689818A072CA54DCE7C4
:10698800584B9B6A002BD8D0012102209847D4E7A6
:106998007B7884F83630012384F83530CDE704233A
:1069A8008DF804307B78003B18BF012301A88DF8CF
:1069B800083002F053F9C0E77878003818BF012092
:1069C80002F098FEB9E7484E0FCE01AD0FC50FCEC5
:1069D8000FC596E8070085E807007B780A2BACD836
:1069E800424A12685268002AA7D00CA901EB830317
:1069F80053F82C0C9047A0E77878431E012B9CD8BD
:106A08003A4B01381B6818BF012020729B68002B85
:106A180093D0984791E7E26801230821A372117087
:106A2800627A057BA17AAA4228BF2A46934284D279
:106A380085685A1CEB5CE56801334E1CA6726B54E2
:106A4800D3B2EDE7E3680122A27209221A70A37A91
:106A5800E268218A581CA072D154A27A238AE1687C
:106A68001B0A501CA0728B5467E7238265E7052335
:106A78008DF8043001A802F077FB5EE7194BDB6A5A
:106A880098475AE7194B78781B686075DB68BEE74A
:106A9800037B072B7FF451AF06238DF80430B7F83A
:106AA8000130ADF808307B793A791B0443EA0223B8
:106AB800FA781343642253430393BB798DF810305B
:106AC800D8E73B2201A88DF804208DF8083002F0A1
:106AD800C5F8012384F834302FE700BF04060020EE
:106AE800E8050020B80000204CF00008000600204F
:106AF8002A2301A88DF8043001F08AFF94F80A903F
:106B0800E6689DF808009DF809509DF80A709DF800
:106B18000BC09DF80D309DF80E209DF80F109DF8C4
:106B28000CE009F1010A84F80AA006F80980354E3C
:106B380094F80A903668D4F80C8009F1010A84F8B0
:106B48000AA096F803A008F809A094F80A90D4F8C7
:106B58000C8009F1010A84F80AA096F802A008F846
:106B680009A094F80A90D4F80C8009F1010A84F875
:106B78000AA096F801A008F809A094F80A9009F16B
:106B8800010A84F80AA096F80080E66806F80980E9
:106B980094F80A80E66808F1010984F80A9006F872
:106BA80008C094F80AC0E6680CF1010884F80A8065
:106BB80006F80C70A77AE66807F1010C84F80AC099
:106BC800F555A57AE6686F1CA7727055A07AE56836
:106BD800461CA6722954A17AE0684D1CA57242543D
:106BE800A27AE168501CA0728B54A37AE268591CFF
:106BF800A17202F803E0A0E6034807F05DFF6570A4
:106C0800AAE600BF00060020E80500207047000043
:106C180000487047B8000020002070474FF0FF3050
:106C280070470000044B054A93F81831022B18BF2F
:106C3800062382F890347047A80C00206C120020BC
:106C4800034BD3F8483313B15B6903B11847704756
:106C58006C120020034A137843F004031370FFF703
:106C6800EFBF00BF500600201FB50A4B8DF8090082
:106C780093F87C208DF80A2093F88C2093F848002C
:106C88000D3202A98DF8082003F064FCC0B205B0EB
:106C98005DF804FBA80C002008B5074807F00CFFB6
:106CA800064B93F81A2412B1012283F81924BDE87F
:106CB8000840FFF7C5BF00BF6C1600206C1200200B
:106CC80010B50C4CD4F8403343F08003C4F840337B
:106CD80094F81A3413B10020FFF7DEFF94F89134CA
:106CE80023F0120343F0120384F89134BDE81040F6
:106CF800FFF798BF6C1200202DE9F041DFF8AC8057
:106D080098F81831022B06460D4602D0284BDB6A4C
:106D1800984702F0A6FD044628B1022002F097FD2C
:106D2800002002F099FD98F81831012B17D102F0D4
:106D38009AFD074630B1002002F08AFD002002F0DB
:106D48008CFD3C4602F091FD48B1002002F081FD27
:106D5800002002F083FDBDE8F041FFF763BF002C7F
:106D6800F9D1144C94F8902494F81A34BAB90BB1A8
:106D780084F84164304602F017FFD8F82C0007F079
:106D880061FED4F8B4339842E5D30B4807F094FE7B
:106D980094F8913443F0100384F89134DBE70BB195
:106DA80084F84154284602F0FFFEF1E7A80C0020C1
:106DB8006CF900086C12002004160020074A10B570
:106DC800137843F002031370FFF73AFFBDE8104051
:106DD800034B01220021022007F042BB500600208D
:106DE80039F20008074A10B5137843F00803137006
:106DF800FFF726FFBDE81040034B012200210220C7
:106E080007F02EBB5006002049F200082DE9F0419A
:106E18000F4616461D46804607F00AFE0B4A0C4CE4
:106E28001378278123F0110343F01103C4E9000804
:106E3800137066812573FFF703FFBDE8F041054B2A
:106E480001220021022007F00BBB00BF50060020E2
:106E58003C06002059F2000813B507F0E9FD0D4B78
:106E68006C461860204607F037FD94E803000A4A8C
:106E78000A4B83E80300137843F020031370FFF7ED
:106E8800DFFE074B01220021022002B0BDE81040BE
:106E980007F0E6BA4C06002050060020A415002092
:106EA80066F200082DE9F04192B0064602F0D9FCDE
:106EB800002840F05881AD4D95F81831012B09D0C4
:106EC8002B6BAB4C93B194F80431BBB1042B6FD04E
:106ED800032003E002F0C7FC18B10F2012B0BDE890
:106EE800F08102F0C2FC0028EAD0F6E7B5F82031BC
:106EF800D4F81C24013B53432B63E4E79D4803F07B
:106F080060FA002840F0128194F80C3123802B6B32
:106F18000C930DF1180895F839308DF83830404643
:106F280095F81C318DF83A3007F0FCFCD5F828317B
:106F3800009302AF98E80600D5F82431384607F0E8
:106F480088FC97E803000FAB83E80300EB6A0D9316
:106F580000238DF844302388ADF8463095F8303159
:106F680001228DF839201BB98DF844208DF839306D
:106F7800814B0093814B95F84800A3F179020CA945
:106F880003F05DFBC0B10B28A8D1D4F8941499B1D3
:106F9800002EA3D0D4F84033794843F02003C4F836
:106FA800403307F011FE764807F0D4FD002095E73E
:106FB800704803F03AFAA4E795F8487095F96930F3
:106FC80095F9392095F87D106E4E384603F044FB4C
:106FD800009641B2EB6C95F850203846183603F00D
:106FE800DFFA0096EB6C95F8502095F9701095F83B
:106FF800480003F0D5FAD4F8C413AB6DD4F8DC23F9
:107008000B44C4F8B033EB6D1344C4F8B43394F8AC
:107018000431042B07D02B6E0B44C4F8B0336B6ECD
:107028001344C4F8B4330023089395F83031002B87
:1070380040D100238DF8133095F839308DF8213080
:1070480095F838308DF82230D5F880300993D5F886
:1070580084300A932388ADF82C3095F8303194F8B1
:107068001B648DF82E3095F84800474B8DF820604A
:107078000DF1130208A903F0A7FA012384F841349B
:1070880095F8393084F842349DF8133084F8433445
:10709800D4F81C34C4F85064C4F84834C4F85834DC
:1070A80002F0E5FBC8B1D4F81C0402F0F2FBA0B171
:1070B800102013E708A802F0A7FC60B995F9390079
:1070C80094F837629DF82070FFF7CEFD3E44B04239
:1070D800AFD2082002E7132000E795F81831012BFA
:1070E80001D102F0D8FB02F0C5FB0023059394F808
:1070F800043195F9395094F81B649BB1042B7FF443
:10710800E7AE05A802F0B4FE58BB94F8183413B1E2
:10711800059B013B0593174B05983246E9B202F0EF
:107128000DFF02E0134802F0DDFE08B11120D5E69C
:10713800D4F8403394F80C11218043F00203C4F8CA
:10714800403394F8183411480133DBB284F818340A
:1071580084F845340E4B00259B6AC4F89854984728
:1071680024E71220BAE60E20B8E600BFA80C0020DB
:107178006C12002074130020D80C00200017002087
:10718800D415002024160020881600206E12002036
:107198006CF9000873B5134D134E0096EB6C95F817
:1071A800502095F9781095F8480003F0F9F995F80A
:1071B8003031337595F8480040F2012306F13C025E
:1071C8003146738203F0F8F950B196F83C3086F8EE
:1071D8008230064B00205B6B9847F37C86F8A8301A
:1071E80002B070BDA80C0020541600206CF90008ED
:1071F800F8B5324C94F81831012B05460ED0022B05
:107208004ED0002B57D138B9D4E91B0104F17403CF
:1072180083E803000020F8BD012806D102F02CFB0A
:107228000028F8D184F81851F5E7022843D1244EF4
:1072380084F8180106F5747CBCE80F0006F57A7727
:107248000FC79CE8030094F8E92094F8003187E818
:10725800030086F8FB53D2B1022B18D1D4F80431BD
:107268006367C6F8EC3394F87D3094F8082186F803
:10727800F83394F88C3084F8782086F8F93396F847
:107288001B2486F8E82340F20133A6F8FA330023DA
:1072980086F81A340B4BDB6A9847FFF77BFFB9E790
:1072A80048B9074B84F81801062283F89024054B47
:1072B800DB6A9847AEE70320ADE700BFA80C0020C3
:1072C8006C1200206CF90008F0B5504C504EB4F820
:1072D800DC202287D4E92D0194F8B12084F86920B4
:1072E80004F16C0282E80300D4E92F0104F174026E
:1072F80082E80300B4F8C420A4F87C2091B0D4F844
:10730800CC20D4F8C810C4F884200025D4F8D020A4
:10731800C4F888200123A4F82031C4F8801084F828
:107328003051A56284F81B5184F83A5084F81D51F5
:1073380084F81E51C4F83451C6F89854A6F8185465
:1073480086F81A54A4F838518DF8183004F50973E2
:10735800039304F50A7394F84800049303A92D4B8A
:1073680084F84551C4E94F55A4F84651059303F0F4
:10737800FFF8E36EC6F8D43394F87D3086F8E0332E
:1073880094F88C3086F8E1334FF48073A6F8E23332
:1073980086F8D05394F8303186F8E43306F57477DC
:1073A8000FCF06F57A740FC497E8030040F2012363
:1073B80084E80300A6F8FA33D6F8483386F81B5455
:1073C800CDE901551BB15A685B6901920293124BD2
:1073D8000793A3F148020892A3F1140209920F4AF5
:1073E8000B9229330A93A2F19C030C93A2F1980300
:1073F8000D93131D0E9301A902F14C0307A802F582
:1074080099620F9302F022FA11B0F0BDA80C002087
:107418006C12002054060020D41600208C0D002089
:10742800F8B50D4F0D4E0C4607F046FB3B6B9847E1
:107438000B4A96F84800214603F0BEF850B1094DB2
:10744800706D95F8243485F86A347B6B9847E37C33
:1074580085F89034F8BD00BF6CF90008A80C00202E
:10746800901600206C1200200F4890F81B3480F80A
:10747800B8330E4B93F8692080F8BB2393F87D202E
:1074880080F8C82393F88C2080F8C92393F830310A
:1074980080F8CC330022A0F8CA2300F56E7100F5FD
:1074A8006070FFF7BDBF00BF6C120020A80C002061
:1074B800114890F89034EBB190F81B3480F8D03331
:1074C8000E4BDA6EC0F8D42393F87D2080F8E023C1
:1074D80093F88C2080F8E12393F8303180F8E43376
:1074E8004FF48072A0F8E22300F5747100F566701D
:1074F800FFF796BF704700BF6C120020A80C002051
:1075080070B5344C2421204604F0D4FF636A9842B5
:1075180018BF60624FF01C012F4814BF01250025D9
:1075280004F0C8FF636C984218BF60644FF4807120
:107538002A4818BF45F0020504F0BCFFD4F84831CA
:10754800984218BFC4F848014FF0D401244818BF26
:1075580045F0040504F0AEFFD4F82032984218BF75
:10756800C4F820024FF000011E4818BF45F0080576
:1075780004F0A0FFD4F82432984218BFC4F82402BB
:107588004FF46071184818BF45F0100504F092FFD9
:10759800D4F8A835984218BFC4F8A8054FF01401CC
:1075A800124818BF45F0200504F084FFD4F8C03510
:1075B80098420F4B18BFC4F8C005D3F8483318BF1A
:1075C80045F040052BB11B691BB12846BDE870404A
:1075D800184770BDA80C0020D00C0020F00C00202B
:1075E800F40D0020CC0E0020D00E002054120020F4
:1075F8006C1200202DE9F04F8FB04FF00009012BDD
:1076080006460F4690468DF80D90ADF8109002D8BA
:107618004C46BC4202D30FB0BDE8F08F305D02F09B
:1076280033FA2044B842F6DC335D651C023BEDB208
:10763800112BF0D801A252F823F000BF8D76000874
:10764800B7760008B5770008DD7700085B78000892
:1076580081780008E77800080F7900089579000814
:107668001F7600081F760008E97900081F760008D1
:107678001F760008917A0008B97A0008F17A0008A4
:10768800257B0008052002F0A7FA70B1052100202B
:1076980002F068FA725DBA4BE51C0234E4B283F872
:1076A8005C24325D83F85D24EDB22C46B1E70023FB
:1076B8008DF80E308DF80F308DF814308DF81830A5
:1076C800B9F1000F6DD1AF4C4FF0050994F87C204B
:1076D8008DF831206B1E94F839208DF8332033440F
:1076E80094F838200B938DF8342094F81A3194F8D4
:1076F80068208DF83520D4F82C218DF832300A9284
:1077080073B37B1C5B1BDBB28DF8303006AB019387
:1077180005AB009394F848000DF10F030DF10E022C
:107728000AA902F05DFF8DF80D0000F00700072898
:1077380013D194F939209DF90E3084F839309A42E2
:107748009DF80F3084F83830B8BF01229DF8143006
:10775800B8BF84F81D2184F868304FF0000A09E0AA
:107768000523D1E701220DF10D01032002F0A4F851
:107778000AF1010A5FFA8AF29DF81830B3FBF9F1B1
:107788009142EFD82B44DDB26B1EDBB29F420BD97E
:10779800F25C032A9AD0AF4288BF1D464FF0010918
:1077A80083E70534E5B2F9E71D46F7E7735D7549E8
:1077B80003F00F03012281F81B31023402FA03F3AC
:1077C800A1F82031E4B2002204A9042002F074F8E0
:1077D80025466AE707238DF80D30735DC3F302125F
:1077E80003F00F038DF82830E31CDBB28DF8292055
:1077F800F25C231DDBB2651DF35C0234E4B21B04AA
:1078080043EA0223325D5F4C13436422534394F8E6
:1078180048000B930AA902F0F2FE00F00703072BB9
:10782800EDB28DF80D000CD19DF8283084F8703039
:1078380084F878300B9BE36663679DF8293084F8F9
:1078480069308DF81000012204A9052002F034F8EF
:107858002BE74B4BD3F8483363B11B6853B19847B8
:1078680008F03F038DF810008DF81130022204A9AA
:107878000620EBE7FF20F3E703238DF80D30735D57
:107888008DF81C300AAB0693E31CDBB2A51DF25C35
:10789800231DDBB206A9F35C1B0443EA0223A21CE6
:1078A800D2B20534B25C134364225343E4B20A9360
:1078B80000230B93335D8DF83030324B93F848003A
:1078C80002F0A3FEC3B20028EDB28DF80D30FFF62A
:1078D800ECAE8DF81030012204A90720B6E7735DDD
:1078E80003F00F03012B4FF47A7238BF012353437F
:1078F800244A0234936503F57A73D365E4B200220F
:1079080004A9082062E7735D1E4DC3F340128DF889
:10791800152095F84800C3F3001205A903F00F03DA
:107928008DF814208DF8163002F075FE02340130FF
:10793800E4B23FF44DAFBDF81430134AA5F87C30DB
:107948009DF816309DF814A0D05CF8F73BFF022391
:10795800C5F880000AA995F848008DF828308DF8F8
:107968002AA002F0F7FD95F93930069040B2984206
:10797800B8BF184685F83900002204A9092025E770
:107988006C120020A80C002073F2000803238DF865
:107998000D30735D8DF82830E31CDBB2651DF25C99
:1079A800231DDBB20234F35CE4B21B0443EA022376
:1079B800325D1343642253430B93644B0AA993F833
:1079C800480002F02EFEC3B20028EDB28DF80D304B
:1079D800FFF66BAE8DF81030012204A90A2035E7B6
:1079E800092002F0F9F8DFF868B1002849D0092128
:1079F800002002F0B7F80023ADF81E30A31CDBB25C
:107A0800F25CE31CDBB216F803A0735D4FEA0A4A86
:107A18004AEA022A4AEA030A231DDBB2A51D0534F5
:107A2800F35CE4B24AEA036A335D4FF47A72534373
:107A38000AAC1B122046ADF81C3006F04DFF454B32
:107A480053440693DBF83C3300930DF1180A9AE887
:107A58000600DBF8383308A806F0FBFE099B009304
:107A680094E80600089B504606F0D8FE9AE8030002
:107A780006F00AFF01F00AFF0123EDB28BF8383453
:107A880013E68BF8380410E60C2002F0A5F800285D
:107A98003FF40BAE0C21002002F064F82C4B93F855
:107AA8009034043B012B7FF600AE01F0EBFEFCE5C1
:107AB800A31CDBB2725DF15CE31CDBB2651DF35CF9
:107AC8000434E4B21B04305D43EA01231343642108
:107AD800594300F00F0001F0D6FEEDB28DF810000A
:107AE800012204A91120B1E60D2002F075F8002842
:107AF8003FF4DBAD0D21002002F034F8A31CDBB20B
:107B0800154AF05C735D1268251D0334E4B243EA3C
:107B18000020315DEDB201F0B8FEC6E5725DA31C30
:107B2800251D0334DBB2E4B2F15C335D1B0443EA88
:107B3800012313436420584301F0A9FEEDB28DF8E8
:107B48001000012204A9132080E600BFA80C002021
:107B58006C120020803DD5123C0600200E4B93F895
:107B68009124920703D593F88F24012A08D90B4949
:107B780091F81A2122B18A6A501C18BF01328A6210
:107B88000022A3F8182483F81A24D3F8402322F0FB
:107B98000202C3F8402370476C120020A80C002092
:107BA80070B5184C1848194D06F086FFD4F84033C4
:107BB800D4F89804D5F8906023F02003C4F8403333
:107BC80038B106F03FFF864203D2002385F83A30E9
:107BD80070BD0120FFF766F90028F9D00B28F7D00F
:107BE80095F8393084F84234092094F8183484F828
:107BF800453484F8410401F0D7FFBDE87040FFF731
:107C0800ADBF00BF6C120020D4150020A80C0020C6
:107C1800094BD3F84023012A0AD008490978C90733
:107C280008D43AB993F89204013818BF0120704774
:107C380000207047012070476C1200205006002079
:107C4800034BD3F84003431E58425841704700BFC6
:107C58006C1200202DE9F04FA9B0EFF3108272B634
:107C6800DFF8F0B20021DBF80030CBF8001082F327
:107C78001088B94C002B00F0E180DAB29B06039221
:107C880064D5B64D95F81831022B02D0B44BDB6A97
:107C98009847EFF3108872B6B24F06F0C9FE3E68F7
:107CA800D4F8B013361A3144AF4806F08DFFAE4809
:107CB80006F050FFD4F8B413AC48314406F084FF02
:107CC800AA4806F047FF88F3108894F81A34002B66
:107CD80000F06B81152312A995F848008DF84830FB
:107CE80002F038FCD4F8B4130F900144A04806F011
:107CF8006BFF9F4806F02EFF3B6894F81B24EB624D
:107D08000DAF38468DF870201D9306F00BFED5F8A0
:107D18002831009306AE97E80600D5F8243130469E
:107D280006F097FD96E803001FAB83E80300D4F83C
:107D38001C341E9395F8303195F84800003B18BF65
:107D480001231CA98DF8713002F00DFC039BDF069E
:107D580048D5824DDFF81CA2D5F8E42004929BF8A0
:107D68000020BAF90A809AF90C90A4F88C840023B0
:107D780063F300020A9384F84434A4F8223484F8A4
:107D88002534C4F82834A4F82C3484F82E34C4F8E4
:107D9800303484F82034C4F8343484F83834C4F8DF
:107DA8003C346F4B8BF8002094F89024DB6A84F8FD
:107DB8008E9484F88F24DAF80470BAF8086098472B
:107DC80094F88F3413B9694806F076FE3146384680
:107DD80001F045FD8346002800F0EA80A4F87E847F
:107DE80084F88094039B19071AD55C4B93F81831D3
:107DF800022B02D05A4BDB6A98470220FEF712FF8B
:107E080084F8410401F0D0FE94F81A3413B1012328
:107E180084F8193494F8913443F0100384F89134B9
:107E2800039B5A0703D506210520FEF765FF039B30
:107E38009B0703D504210320FEF75EFF01F02DFD0B
:107E480094F89124D7065FD5002384F89234D4F8A7
:107E580040331E0644BF23F08203C4F8403312F0B7
:107E6800050F00F0FB820B2001F0B6FE002800F0A1
:107E7800F58294F89134DD0700F1F082580740F15B
:107E88000783D4F8403323F00203C4F84033D4F80E
:107E9800402382BB94F8915415F001011EBF2B4674
:107EA80062F3000384F8913494F891345E0744BF78
:107EB8006FF3820384F89134012384F8923421B15A
:107EC800D4F844332C481B6898476D070BD52B48CA
:107ED80001F08EFE01F0BCFE28B194F8913443F015
:107EE800040384F8913401F0C6FC94F891346FF3DC
:107EF800041384F89134012384F8923494F891346B
:107F080043F0200384F8913494F8913418070AD583
:107F18006FF3C3031A4984F89134D4F84433A1F1B8
:107F28002400DB68984794F8913499070AD56FF3D1
:107F38004103134984F89134D4F84433A1F16C0017
:107F48005B68984794F89034022B1BD1FFF722F90D
:107F580018E000BF500600206C120020A80C00207A
:107F68006CF900084C060020EC15002004160020CF
:107F78006C1600203C060020AC160020C01600201D
:107F8800F816002094F891349A0640F1C4826FF3F1
:107F9800451384F89134D4F84033002B40F0BB8269
:107FA80029B0BDE8F04FFFF7ABBA84F84134A3E637
:107FB80095F81831012B0CD101F055FC804668B1B9
:107FC800584601F045FC584601F047FC042384F864
:107FD8008F347EB9012384F821344FE101F045FC48
:107FE8000028F6D0404601F034FC404601F036FC4B
:107FF8000523ECE73B7805935B09013B062B00F270
:108008001782DFE813F007001502950015029200A9
:1080180015020602102EDDD995F830311297F6B206
:108028008DF84C60002BD5D11CA804F055F912AA84
:108038001CA9FF2002F09EF89DF85830C3F30303F3
:1080480007468DF82C3095F8480095F87D308DF866
:108058002D3007220BA902F090FA002F5DD10028DD
:108068005BD09DF853309DF852201599C5F8E4105F
:108078001B0443EA02239DF8512002201343C5F84C
:10808800E03004F037F99DF8583095F8480085F845
:108098002E71C3F30212C3F3030385F8703085F819
:1080A80078309DF8593085F86920012B38BF0123B5
:1080B8004FF47A725343AB651344EB650DF15A03E1
:1080C8004FF001081093113E94F81B348DF83C30A2
:1080D8000FA985F868808DF8446002F056FA0223EB
:1080E800404685F8303101F077FD18B141463846F1
:1080F80001F038FD94F88F34012B00F2A78194F831
:108108001A34002B40F09A8194F8913443F010030C
:1081180084F89134FEF786FD64E6012001F05CFDE9
:108128000028E7D001210720E2E7012384F8203462
:1081380095F87D308DF82E3094F824348DF82D3054
:1081480095F88C3095F848000D330BA98DF82C3034
:1081580002F000FAA6F10D031BB2099023EAE373BB
:1081680000B283423FF736AF0B2E7FF633AFBA4BE0
:1081780025931CA8FF231C978DF874608DF8983000
:1081880002F0C4F8074600287FF424AF95F81831A8
:10819800012B13D101F067FB002872D0384601F09B
:1081A80057FB384601F059FB04239DF87C101E98B4
:1081B80084F88F34C1F3001101F06EFB9DF87C3018
:1081C8001E99C4F8341413F00F0203D09DF89000E0
:1081D800002862D19DF89800002861D0002A7FF419
:1081E800F9AE9DF89020002A14BF4FF003084FF015
:1081F800020800220A92D5F8EC2095F8E90091428D
:1082080051D100284FD0D5F80C1195F8EAB009687B
:108218000A9195F81811022902D1032184F88F14C4
:10822800B8F1030F7FF4D6AE13F0600F7FF4D2AE2F
:108238000492012795F82E31BBF1000F36D0BBF11F
:10824800010F13D1012B33D16FF0090646FA08F656
:1082580006F00106C6F10206F6B2BDF87E100AAABB
:10826800304601F011FE38B3072823D0012384F8E3
:1082780021340A9BC4F83034C4F86C34FEF720FD6E
:10828800B0E501F0F2FA002898D0384601F0E1FA9A
:10829800384601F0E3FA052387E74FF00008A8E71E
:1082A8004FF00108A5E74FF0010BC3E70426D4E718
:1082B8000326D2E70823DAE71CAB009304990A9B4C
:1082C8003246584601F0A2FE20B1022814BF0B2303
:1082D8000A2380E60A9BC4F83034C4F86C349DF84D
:1082E8007C3084F82104C3F3401384F82E3484F8D6
:1082F800443494F88F3484F82274012B9EBF0122F1
:10830800A86285F81E21012FC4F8280484F82C04DB
:1083180084F8410438D1022284F8202495F83A20C0
:10832800002A4AD19DF87C20D60646D4012B94F821
:1083380040149DF87C2005D8012901D1900601D56B
:1083480001F04CFBB8F1020F94F88F3443D0B8F128
:10835800030F0AD09DF87C10B8F1010F4A4601F0CE
:108368000F0120A83BD0FFF745F99DF8903084F81D
:108378002334259BC4F828349DF8983084F82C348D
:10838800012384F82D3430E0059A02F0E002A02A97
:108398001BD195F82E11012285F83A2009B92799A1
:1083A8006963012B84F8202407D9D5F89020C4F8F4
:1083B8003C24DAF80020C4F8982495F81821002AFB
:1083C800B4D1012284F82524B0E7002285F83A20A8
:1083D80084F82024A6E79DF8981025984A46FFF7C8
:1083E80009F99DF8903084F823349DF89020E02A0C
:1083F80008D195F81F312BB984F82324C4F8283400
:10840800A4F82C3494F8913443F0020384F891349E
:1084180070E6114D013EB2B2791C284604F034F8DA
:108428000323A4F82034C4F8285484F82C64E9E71A
:10843800012384F82134FEF743FC5BE694F84434C6
:10844800002B3FF461AE0020FEF726FC94F88F3431
:10845800022B3FF45FAE57E6A414002094F8913441
:10846800590715D5012001F0B7FB60B1012001F0D3
:108478008BFB08B984F81804D4F8403323F00203BE
:10848800C4F8403304E0062001F0A6FB0028F3D12D
:1084980094F89134DA077FF5FAAC94F840240AB1DD
:1084A800032A18D11D4A94F8181492F868209142AA
:1084B80005D29B0723D594F88F34012B1FD8184871
:1084C80006F0FAFAD4F8403323F02003C4F8403316
:1084D800FFF744FBDBE4012A11D194F81924002AA0
:1084E8003FF4D5AC0D4A94F8181492F868209142DC
:1084F800E5D29F0703D594F84434002BDFD194F8D4
:10850800913400206FF3041384F8913484F819042B
:10851800FFF746FBBBE429B0BDE8F08FA80C0020AC
:10852800D41500202DE9F04F89468DB090460746B6
:10853800002800F08F81002900F08C810368002B4F
:1085480000F088814368002B00F084818368002B49
:1085580000F08081C368002B00F07C81104601F098
:10856800F5FF002800F07881BD4CBE4D384601F07B
:10857800AFFA40F2C4520021204603F099FF40F2BE
:108588001C520021284603F093FFB74BC4F82C3146
:1085980004F50973089304F50A7300264046099305
:1085A80008A9B24B84F848800A9384F8186184F8C3
:1085B8008C608DF82C6001F0DBFF0F2306A994F87E
:1085C80048008DF8183001F0C5FF801B18BF012046
:1085D8004FF00A0B84F81C0106A994F848008DF89E
:1085E80018B001F0B7FF4FF0060A84F8DC0006A9BE
:1085F80094F848008DF818A001F0ACFF102384F817
:10860800DD0006A994F848008DF8183001F0A2FFA3
:108618001123C4F89C0006A994F848008DF8183076
:1086280001F098FF1223C4F8A00006A994F84800A6
:108638008DF8183001F08EFF1323C4F8A40006A9A2
:1086480094F848008DF8183001F084FF1423C4F81A
:10865800A80006A994F848008DF8183001F07AFFB0
:108668001623C4F8AC0006A994F848008DF8183011
:1086780001F070FF172384F8B10006A994F84800A8
:108688008DF8183001F066FF18230DEB0301C4F8CC
:10869800B400C4F8BC0094F848008DF8183001F014
:1086A80059FFC0B21D2384F8B80084F8C00006A999
:1086B80094F848008DF8183001F04CFF1E2384F818
:1086C800C40006A994F848008DF8183001F042FF5C
:1086D8001F2384F8C50006A994F848008DF81830BF
:1086E80001F038FF2023C4F8C80006A994F8480010
:1086F8008DF8183001F02EFF0B23C4F8CC0006A922
:1087080094F848008DF8183001F024FF0C2306A9CE
:10871800A4F8D00094F848008DF8183001F01AFF3A
:10872800D4F89C306365D4F8A030A365D4F8A4309D
:10873800E365D4F8A83023664FF00108D4F8AC30CC
:108748000590A4F8D200636684F8B080C4F894B0A9
:1087580084F898A0C4F84CB084F850A084F86880D5
:1087680084F81F81C5F84893FEF7AEFDC5F8447339
:10877800C4E90B663E4B84F8198185F89164C5F805
:10878800408332464FF0FF31009605F55A7006F0E7
:1087980035F9384B009632464FF0FF3105F56070D9
:1087A80006F02CF9344B009632464FF0FF3105F5B0
:1087B800667006F023F902AF304B009632464FF050
:1087C800FF3105F5806006F019F9384606F0AAF879
:1087D80097E8030004F5927383E80300284B294FB8
:1087E8001E60294BC5F84C33284BC5F85433284B29
:1087F800C5F85C33274BC5F85033274BC5F85833B9
:1088080005F553703B68984704F5A67003F080FBA4
:1088180020B1112630460DB0BDE8F08F204601F09A
:1088280003FB0028F5D101F039F8B8B91B4801F06D
:108838004DFB06460028ECD17B69984703F002FE01
:10884800BB6D94F819019847FB6A9847012385F88E
:108858009234DFE70326DDE70926DBE71326D9E7AD
:10886800A80C00206C12002000040001540600200F
:10887800A97B000871740008B9740008A16C00088D
:10888800500600206CF90008616E0008156E00089B
:108898005D6C0008ED6D0008C56D0008900D0020A6
:1088A80008B5034B0020C3F84003FEF7BBF908BD29
:1088B8006C12002010B5FFF7ABF90A4C60B90A4BEF
:1088C80093F81831022B02D1084BDB6A9847012331
:1088D800C4F84033002010BDD4F84003013818BF55
:1088E8000120F8E76C120020A80C00206CF90008A1
:1088F80038B5124C204606F0DFF804F1180006F0EF
:10890800DBF804F1300006F0D7F804F1980006F01F
:10891800D3F800F0AFFF0A4B0025DB6A984744F80C
:10892800285CFEF7EDFD0749074840F2C45203F002
:10893800ABFD012344F8283C284638BDD415002057
:108948006CF90008A80C0020E406002070B52E4B36
:108958008AB0054693F8DD008DF8090093F8DC002D
:108968008DF80A0029489A6A90F81804039200269C
:108978008DF80B0004960C46002940D00692D3F8D7
:10898800882007921A8F93F81A118DF8151052BA89
:10899800ADF8202093F87C2093F848308DF82430E7
:1089A80003AB8DF822008DF8232000930DF10A0205
:1089B8000DF10B030DF1090105A88DF8146000F005
:1089C800D7FE9DF90900FEF74FF9607004A801F081
:1089D8001BF8B0B9049A0F2A0DD863789A420AD8BE
:1089E8001544AB42A3EB02012CBF002001202170EB
:1089F800C0000AB070BD002323700820F9E70320E7
:108A0800F7E71320F5E700BFA80C00206C12002040
:108A18001FB50446002800F010810378412B00F2AE
:108A28000781DFE813F0420049004D00510055006E
:108A380059005E0005010501050105010501050153
:108A480005010501650069006D0078007F0082005E
:108A580085008A0088008C00900093009600990099
:108A68009C009F00AE00B200BA00B600BE00C10074
:108A7800C500CE00CA00CC000501D20005010501E1
:108A880005010501050105010501050105010501AE
:108A980005010501050105010501DA00DE00E20016
:108AA800E700EB00EF00F300FC00664B93F8183189
:108AB8002371002004B010BD624B93F83031F7E702
:108AC800406803F0C3FBF4E7406803F005FCF0E7F7
:108AD8005C4B93F81A31EBE75A4BD3F8E0306360FC
:108AE800E7E7584B011D93F8300103F00DFCE0E770
:108AF800544B93F81931DBE7524B93F88C30D7E796
:108B08001C238DF808304F4B02A993F8480001F058
:108B180021FD6060CDE74C4B043493E8030084E802
:108B28000300C6E7494B0434F7E7494B0434F4E73C
:108B3800484B0434F1E71A23E3E71923E1E7414BF3
:108B480093F86830B4E73F4B5B6DC8E73D4B9B6DCE
:108B5800C5E73C4BDB6DC2E73A4B1B6EBFE7394BB1
:108B68005B6EBCE702238DF80830364B02A993F8F8
:108B78007C2093F848008DF80A2001F0EBFC207166
:108B880097E7304B93F8DD3092E72E4B93F8393066
:108B98008EE72C4B93F8DC308AE72A4B93F8383071
:108BA80086E7284BDB6C9AE7264B93F850307FE733
:108BB800244BD3F8843063607BE7224B8FE7264B46
:108BC8008DE7204BD3F8CC30F5E71E4BD3F82C318A
:108BD800436001F04DFDA0606BE71A4BD3F890306D
:108BE8007DE7184B93F81F3162E7164BB3F88830CE
:108BF800A3805EE7134BB3F88A30F9E7114BB3F85B
:108C0800D030F5E70F4BB3F8D230F1E70D4B93F8BE
:108C180048200AB1062A12D1B3F8A035E8E7094B73
:108C280093F848200AB1062A09D1D3F8A43556E7A3
:108C380004B0BDE8104000F021BE03203AE7182038
:108C480038E700BFA80C0020140D00205C0D0020A0
:108C58001C0D0020640D0020E40600207FB50446AA
:108C680010B9032004B070BDA34DD5F840339A075E
:108C780000F16F820278412A00F26882DFE812F080
:108C88004200470055005B005F0064006900760001
:108C9800810087008D00930099009F00A500AB001C
:108CA800B5006602BA00DC00EF00160138012901A0
:108CB80042014B014F01530157015B0166025F01FD
:108CC800710199018701AB01B101B801BD01C20170
:108CD800660228026602660266026602660266028A
:108CE800660266026602660266026602660266023C
:108CF80066026602340239023E02430248024D020D
:108D080052025C020079FEF773FA30B1AAE70379E0
:108D1800022BA6D0794A82F8303195F8913443F085
:108D2800200385F8913400209CE7406803F080FA1E
:108D38000028F2D095E7406803F0BEFAF8E76F4BD9
:108D4800027983F81A21E8E76C4B4268C3F8E020FF
:108D5800E3E76A4E416896F8300103F0CBFA002841
:108D68007FF47FAF6368C6F8E430D6E7416800292E
:108D78003FF477AF002001F0DDF90028CDD01120B5
:108D880070E7416800293FF46CAF0120F3E74168C0
:108D980000293FF466AF0820EDE7416800293FF459
:108DA80060AF0920E7E7416800293FF45AAF0C207B
:108DB800E1E7416800293FF454AF0D20DBE7416843
:108DC80000293FF44EAF0E20D5E7416800293FF453
:108DD80048AF0F20CFE74A4C484B007983F8190178
:108DE800A36D9847E36A984797E7444B027983F85D
:108DF8008C2092E7414E037A8DF8043096F84800AB
:108E080096F87D308DF80530072201A901F0B5FBF1
:108E180000283FF426AF636896F8480001930022C3
:108E280001A901F0AAFB00283FF41BAF6C36D4E976
:108E3800010186E8030070E7304E037A8DF80430AC
:108E480096F8480096F87D308DF80530072201A97C
:108E580001F093FB00283FF404AFB436E7E7274E50
:108E6800037A8DF8043096F8480096F87D308DF82E
:108E78000530072201A901F080FB00283FF4F1AE7C
:108E8800D4E9010106F1740383E8030096F8183168
:108E9800022B7FF442AF96F83031002B3FF43DAF00
:108EA800174BDB6A9847FEF775F936E7134E037AD6
:108EB8008DF8043096F8480096F87D308DF8053026
:108EC800072201A901F059FB00283FF4CAAEBC36BD
:108ED800ADE74368029301238DF80C30074B02A9D4
:108EE80093F8480001F056FB00287FF416AFB8E667
:108EF800436802930023EFE76C120020A80C0020BF
:108F08006CF9000803795A1E0E2A3FF6AAAE934A56
:108F180082F8683001E7914B42685A65FDE68F4B4D
:108F280042689A65F9E68D4B4268DA65F5E68B4B3F
:108F380042681A66F1E6894B42685A66EDE6874C44
:108F4800037994F848008DF80430062201A901F04D
:108F580014FB00283FF485AE9DF8043084F8DD301A
:108F6800DBE67E4C03798DF8043094F8480094F8D9
:108F78007C308DF80630052201A901F0FEFA0028A0
:108F88003FF46FAE9DF8043084F83930C5E6734C71
:108F9800037994F848008DF804300A2201A901F0F9
:108FA800ECFA00283FF45DAE9DF8043084F8DC301C
:108FB800B3E66A4C037994F848008DF80430092226
:108FC80001A901F0DAFA00283FF44BAE9DF804300D
:108FD80084F83830A1E6614B4268C3F89420DA641B
:108FE8009BE65E4B027983F8982083F8502094E63C
:108FF8005A4B4268C3F884208FE6584B4268C3F83E
:10900800CC208AE6012B40F0A480554C2421204630
:1090180003F050FA636A984201D0172022E61C2117
:1090280004F1280003F046FA636C9842F5D14FF436
:10903800807104F1480003F03DFAD4F848319842B1
:10904800EBD1D42104F5A67003F034FAD4F8203219
:109058009842E2D1002104F5097003F02BFAD4F804
:1090680024329842D9D14FF4607104F50A7003F0A4
:1090780021FAD4F8A8359842CFD1142104F2AC5083
:1090880003F018FAD4F8C0359842C6D1334E2146B9
:10909800304640F2C45203F0F7F9204640F2C45279
:1090A800002103F005FA95F81B3485F8E833736F4F
:1090B800C5F8EC3396F87D3085F8F83340F2012393
:1090C800A5F8FA33274B96F819019B6D984724E6C3
:1090D8008379012B3FF6C5AD204B42684068C3F841
:1090E8002C2100F0BDFE48E61C4B4268C3F89020D6
:1090F80013E61A4B027983F81F210EE6174B828874
:10910800A3F8882009E6154B8288A3F88A2004E68C
:10911800124B8288A3F8D020FFE5104B8288A3F871
:10912800D220FAE50D4B93F848200AB1062A12D14D
:10913800A288A3F8A025F0E5084B93F848200AB1C7
:10914800062A08D16268C3F8A425E6E500F098FB72
:10915800DBE5012086E5182084E500BFA80C002087
:10916800E40600206CF900082DE9F04387B00023DD
:10917800ADF800300646002800F0EE800361FEF7E7
:1091880047FD20B10124204607B0BDE8F08300F078
:1091980065FD0028F6D100F05BFD014618B96F485F
:1091A800142203F085F96E4D95F89134012243F0AD
:1091B800040385F8552485F8913433788DF8043004
:1091C8000021013B8DF80520ADF806100C2B00F2AC
:1091D800BB80DFE803F007B9B9B97982B9B990B9AA
:1091E800AD9AA900D5F8407317F02007CAD196F8B0
:1091F8000480B8F1020F46D1DFF868815A4CFEF7B7
:1092080063F896F9051098F848003A4601F00FFA05
:1092180088F83900B37988F83830384607238DF84C
:109228000530FDF7E5FFFF2304F58670A5F80C313E
:10923800C5F8084185F8047103F04EF804F58A7002
:1092480003F004F83846FDF72DFE0446002839D00F
:1092580096F9051098F84800012201F0E8F988F815
:109268003900D5F894343361002C71D000F0F0FC4B
:10927800002888D195F8913485F81A0460F38203A0
:1092880085F891347FE7B8F1010F4FF00204E8D177
:10929800DFF8D0908DF8144099F8480089F81D71CE
:1092A80002A901F065F9337989F830318DF8057034
:1092B8008DF80680FDF7C4FC95F8913443F010034F
:1092C80085F891340024CCE700226946022000F09A
:1092D800F3FA0028F6D01324C3E7244BB288DB6BDB
:1092E80096F90C10B0689847D5F8403343F002035C
:1092F800C5F84033E6E702A90D2000F053FB00282B
:10930800E0D0002269460D20E1E7164B93F81831AA
:10931800D3B9347904F0070000F0ABFA8DF80040B7
:10932800012269461020D2E7002269461220CEE7C2
:109338008DF8072000F08EFA044638B900F087FA55
:10934800204600F089FABDE702248AE7012488E76D
:1093580001A800F0D1FB16E7032414E7C01600208B
:109368006C120020A80C00206E1200206CF9000876
:109378002DE9F04F99B08046059118B9032019B02E
:10938800BDE8F08F00230361FEF742FC0446002885
:1093980040F0A58046460FCE0EAD0FC514225248A8
:1093A80098F800A0B8F80C7098F90EB04F4E214606
:1093B80003F07EF84E4B012283F8412496F83021C1
:1093C800022A25460BD196F81821022A07D196F8C9
:1093D8001E2122B9BAF1010F38BF4FF0010ABAF1C4
:1093E800010F2BD0BAF1030F2AD0BAF1000F33D1F5
:1093F80002229DF83C30DDF84090029362F3471555
:10940800012496F87C108DF8321002220CA996F8E7
:1094180048008DF8302001F09DF896F81A3196F83A
:1094280030C196F81D1140B2002B63D0BCF1010F7A
:1094380057D1002955D1002C61D153E00422D8E737
:109448000023DDF83C90BDF840709DF942B00293CE
:1094580065F01F050124D4E74FF0000BD946CDF87D
:1094680008B0CEE74FF0010084F81A04D2E005F204
:109478009A420BA900F0D4FA002800F015811320B5
:10948800049B33871A4B002283F81A2423E105F240
:109498009A452A460BA900F0C3FA0028EFD10B9B86
:1094A80084F82801C4F82C5184F83031FCE0B9F173
:1094B800000F00F0F980002A00F0F6804946E01C11
:1094C80002F0E2FF94F8373201332380ECE01220F7
:1094D800D6E70220D4E70720D4E71320D2E70120FB
:1094E8004DE7FCB90220F6E0AC160020A80C0020DD
:1094F8006C120020002CF5D05845B8BF584696F895
:109508007C308DF82000052296F848008DF822302E
:1095180008A901F032F800283FF430AF9DF8203058
:1095280086F839306F4A704BD2F89804D3F89040D7
:1095380038B105F087FA6C4B84423CBF002283F8AF
:109548003A20198F1A8F93F830010491996A09917A
:1095580052BA0028BFD093F81B0100B9186393F8DA
:109568001801ADF85820013893F87C2093F81A4177
:109578001491D0F1000BD3F888108DF85B204BEBD9
:10958800000B93F8482093F83A0093F868308DF868
:109598005A3009AB0093554B03904FF001008DF8FA
:1095A8004C0015918DF85C20A3F12F01A3F1300236
:1095B80013A88DF84D4000F0DBF8039B4FEA0B1B16
:1095C8004BEA431B00264BEA801B4BEAC413B14508
:1095D800444C039308BF37463A46494604F59C7005
:1095E800CDE90A669B46268084F81A6402F04CFF8F
:1095F800E9B2A570C5F34215FAB2042D3A4E039BA1
:1096080084F837223FF42EAF072D3FF450AF022DD8
:109618007FF45FAF364D84F80D110420029984F869
:109628000401FF2084F80C0184F8281184F814310F
:10963800D6F8E410C4F8085105F59B730AA8C4F8D5
:10964800101184F83021C4F82C3100F011FC0028E6
:109658007FF43DAF0A9BA4F844040BA8A4F8163184
:10966800C4F84C3400F0D0F900287FF408AF0B9B05
:10967800D3B196F93900FDF7F7FA94F83732002B91
:109688003FF405AF0B9B0F2B3FF6F1AE05F58B7240
:109698000BA90F2000F0C4F900287FF4F0AE0B9B53
:1096A80063F3030B84F814B10598FDF7FBFB00285E
:1096B8007FF4E6AE099B86F83A00B36200F080F9C1
:1096C80000287FF40AAF94F8913484F840A443F05A
:1096D800010384F89134034BD3F89434C8F810305C
:1096E8004DE600BF6C120020A80C0020100D0020D1
:1096F8006E12002037B50B4D8DF8040004460F227A
:1097080095F8480001A900F038FF40B1064A85F8ED
:109718001C4192F8913443F0200382F8913403B04D
:1097280030BD00BFA80C00206C12002010B5FFF758
:10973800C1F8044688B90A4805F0BEF9094805F099
:10974800BBF9094805F0B8F900F094F8FDF7BCFD3D
:10975800064BDB6A9847204610BD0124FBE700BF93
:10976800D4150020EC150020041600206CF9000820
:109778002DE9F04F8BB047780093149B90F90C803B
:1097880090F90D6090F80EB08A4641681960044659
:109798009146002F58D002238DF8103004A9C37BBE
:1097A800007C8DF8123000F0D5FEB4F808C061894D
:1097B80043B26068984545466144B8BF1D46604558
:1097C80034BF00270127884209D30A218DF81010D9
:1097D800207C019304A900F0BDFE019B46B2B4F8B9
:1097E80008C0608961680CEB400E714519D3A1EB84
:1097F8000C01B1FBF0FC00FB1C1191B9984503DC8E
:109808002378CBB94FF0010B21238DF81030207C41
:10981800E37B8DF8115004A98DF8123000F09AFE00
:1098280045B2009B8AF80050384689F8006083F8F2
:1098380000B00BB0BDE8F08F0223207C8DF82430F7
:1098480006A900F095FEDDE74546EAE77047704750
:109858007047704700207047704770477047002076
:109868007047002070470020704700207047002094
:109878007047704770477047022070470220704752
:1098880002207047704700207047704770470020DB
:1098980070470020704770477047704710B5054CF7
:1098A8004FF403722046002102F002FE0020C4E9B2
:1098B800000010BD881700202DE9F8438146904626
:1098C80000293CD01F4C2023224604F1100012F836
:1098D800017F6FBB8242FAD11B4E3368013403B952
:1098E8003460736803B11C6000252560C4F80880E3
:1098F80074601FFA88F284F80490601D02F0C4FDB9
:10990800B9F1110F4FF0000398BF104D6373D6F8EB
:10991800083298BF25FA09F503F1010398BF05F04D
:10992800010543442573C6F808323846BDE8F88374
:10993800013B13F0FF030446C6D10227F5E70127D0
:10994800F3E700BF8F1700208817002020070200C8
:1099580010B518B3124A1368984204D1036813600B
:10996800002305E00B46002BFAD019688842F9D18C
:109978005168884208BF53600BB101681960D2F87A
:1099880008328168013B00245B1A04602146C2F852
:109998000832102202F08CFD204610BD0120FCE7A1
:1099A80088170020054B1B6813B11A798242FAD137
:1099B800002B0B600CBF0320002070478817002085
:1099C80010B5054B186800B910BD037B04680BB9C6
:1099D800FFF7BEFF2046F6E78817002038B5084B8A
:1099E800084C186800B938BD03790568112B05D8EB
:1099F80024FA03F3DB0701D5FFF7AAFF2846F1E7AE
:109A0800881700202007020028B1044BD3F8083239
:109A18000360002070470120704700BF88170020AE
:109A28002DE9F04107460E46154642B339B3154BAA
:109A38001C6800232CB93046FFF7E6FF0020BDE87C
:109A4800F081A268F91A0132914215D32279EA54B9
:109A5800581C22895FFA80F8611D55FA80F002F0DF
:109A680013FDA368246898445FFA88F3E2E7204668
:109A78002568FFF76DFF2C46002CF8D1DBE70120A5
:109A8800DDE700BF881700200238C0B211289ABF4E
:109A9800014B185C0020704783F2000830B50B4B6F
:109AA80093F820200446084672B100211C3305783B
:109AB800A54208D001319842CDB214BF0430103805
:109AC800AA42F4D8002030BD1046FCE794190020C3
:109AD80010B5084C00232060142204F10C00FF216B
:109AE80084F82030C4E9010002F0E2FC012384F884
:109AF800213010BD9419002010B50E4A92F820109C
:109B0800042915D8936804781C7044785C70C4786C
:109B1800807898700131DC7082F8201002F11C0105
:109B28008B4214BF043302F10C039360012010BD73
:109B38000020FCE794190020094B93F8200068B135
:109B48005A6803F11C018A4200F1FF3014BF043245
:109B580003F10C0283F820005A600120704700BF0F
:109B68009419002010B5074B93F8202004460846A6
:109B780032B15968FFF792FF10B101234470837026
:109B880010BD00BF9419002008B5064B93F820209B
:109B98002AB15968FFF782FF08B1407808BD012053
:109BA800FCE700BF9419002030B50A4A92F820104B
:109BB800536882F8210061B1916801241C32DD7874
:109BC800587005B99C70934214BF0433103B9942F6
:109BD800F5D130BD9419002008B5044B5968FFF73A
:109BE8005DFF003818BF012008BD00BF9419002090
:109BF800F7B50422154E044600210DEB020096F835
:109C0800207002F055FC0025EBB29F4201D803B04A
:109C1800F0BD7368197821705A786270987838B1F5
:109C2800336820469B689847FFF786FF0135EBE7C6
:109C3800DB788DF804108DF805208DF80730FFF7D4
:109C48007BFF01A8FFF758FFF0E700BF9419002039
:109C5800014B93F82000704794190020034B93F8A8
:109C68002000042894BF0020012070479419002088
:109C78001FB50024CDE90244C41F8DF800408DF8BB
:109C880001100C0AADF80420090C120C8DF8031011
:109C98008DF806208DF8073002461B0A0121684618
:109CA8008DF802408DF8083002F05DFA002818BFE0
:109CB8000E2004B010BD2DE9F04188B090460D4645
:109CC8000F9A0746002847D000240121CDE9044413
:109CD8008DF810109DF838108DF81510ADF8163065
:109CE800190CCDE900441B0ECDE902448DF819305A
:109CF800ADF81A20130C120E07948DF818108DF871
:109D08001C308DF81D20E3B21E01002DF6B203DCD5
:109D1800002008B0BDE8F081013310218DF81F3014
:109D280042466B460DEB010002F0B3F90346A8B9B1
:109D3800102D28463E44A8BF10206946327811F8F5
:109D480001CB013382EA0C02984206F8012BF5DCBC
:109D5800103D2DB20134D6E70920DAE70E20D8E706
:109D68000138032815D8DFE800F002080C100A4B68
:109D78001B681B690B6000207047074B1B685B69F9
:109D8800F8E7054B1B689B69F4E7034B1B68DB6925
:109D9800F0E70520704700BFB81900202DE9F04111
:109DA800C4B00C464A9E17461D468046B8B3B1F566
:109DB800807F36D84FF488720021684602F078FB1D
:109DC800492300934FF48073ADF804302B0C8DF8C1
:109DD8000830330CADF80650ADF80A608DF80C3039
:109DE80022460023414604A82D0E360E8DF80E306B
:109DF8008DF809508DF80D608DF80F4002F044FB86
:109E080004F110014B9A3B4689B2684602F02BF9DF
:109E180010B1012818BF0E2044B0BDE8F081092018
:109E2800FAE70D20F8E7000010B590B10A4C282297
:109E38000021206002F03CFB2368084A1A600020D9
:109E48004FF0FF32C3E90302C3E90522C3E9072241
:109E580010BD0820FCE700BFB8190020000101016F
:109E6800024B1B6818600020704700BFB81900201B
:109E780030B1044B1B68DB68013303600020704776
:109E880009207047B819002013B500230C46019328
:109E9800CAB101A9FFF764FF18B9019B591C02D187
:109EA800146002B010BD99B2611A002901DD5C1876
:109EB800F6E702D113600720F3E71B0C1B0403F538
:109EC80080331C44ECE70920EBE7000028B1044B81
:109ED8001B681C334362002070470920704700BF8D
:109EE800B81900201FB5044600B3002303A8039344
:109EF80002F090F9104ABDF80C30126820469380A1
:109F0800E38200F05EFA98B904F11803009321681F
:109F18000123132202F09CF860B9204600F051FAA0
:109F2800003818BF0120000104B010BD0920FBE76C
:109F38001020F9E70E20F7E7B8190020F0B505461C
:109F480087B01C4613B9092007B0F0BD2E4E336800
:109F5800DB68834255D894F82020002A0CBF0822D9
:109F68000922834205D3204600F05FFA68B1102029
:109F7800EAE7002301900093A36894F82810606A28
:109F8800FFF799FE0028EED0DEE723792168B4F8C0
:109F980008C0A768043B9AB20029D4D0B2F5807FE4
:109FA8002DD8ADF80EC08DF817304FEA174C04F1D4
:109FB8002C033F0E8DF8117000932F0C08234FF0DF
:109FC800490EADF80C008DF814708DF816002F0EA0
:109FD8000DEB0300CDF808E08DF810C0ADF8125075
:109FE8008DF8157002F034F808B10E20ACE7204661
:109FF80000F01BFA0028BAD13368DD60A4E70D2011
:10A00800A2E70620A0E700BFB81900202DE9FF410C
:10A018000A9D80460F4616461C46002D5AD000233E
:10A0280003A910460393FFF79BFE18B1062004B05E
:10A03800BDE8F081039B9C4201D80133F6D1284644
:10A0480000F064F9002847D1264B1A78424503D01E
:10A058001A79424542D10120AA68BA4240D103EB9D
:10A068008002EB6A92F801802979CDE9004304392E
:10A07800927828683B4689B2FFF790FE0028D6D12F
:10A0880095F820300194002B4FF00103009314BF82
:10A098004246082295F82810686A3B46FFF70BFEEF
:10A0A8000028C4D1013E032EC1D8DFE806F002071C
:10A0B8000B0F0D4B1B681C611C62B8E70A4B1B6831
:10A0C8005C61F9E7084B1B689C61F5E7064B1B6868
:10A0D800DC61ACE70920AAE70F20A8E70B20A6E778
:10A0E8000220A4E7F0000020B81900201FB50B29B2
:10A0F8004FF00003CDE90033CDE902330A4607D01B
:10A108000C2914D00A2910D00A2005B05DF804FBE8
:10A11800012802D120238DF800300021684602F082
:10A1280022F8002818BF0E20EFE73023F3E70B21B1
:10A13800F4E7000038B5054602F010F8044610B1FF
:10A148000E24204638BD002DFBD1094B1B680B217E
:10A158009878FFF7CBFF0028F2D10C21FFF7C6FF54
:10A168000028EDD10A21FFF7C1FF0028E9D0E7E771
:10A17800B81900202DE9F04380468FB00C461746E9
:10A18800002A6BD0002969D0002529461D2206A87F
:10A19800059504F097FE8DF81350344D2B680DF19A
:10A1A80014099E88CDF804900DF1130302933B79AE
:10A1B80000933B6832462146404601F0F0FF0028F4
:10A1C8004ED138683A79494602F05EF9384600F0CF
:10A1D8004FF8002846D13C7AFA79BB79240444EA3E
:10A1E80002241C432B689A6894423DD99C609DF8D0
:10A1F80013000B21FFF77AFF034658BB0C21FFF72A
:10A2080075FF034630BB0A21FFF770FF034608BB02
:10A218007B7ABA7AFF7A3F0447EA02271F433A4615
:10A22800334621460920FFF723FD034690B93346FC
:10A238003A4621460820FFF71BFD034650B92A6815
:10A248009DF8131091700021D1604FF0FF31C2E9E1
:10A258000411916118460FB0BDE8F0830923F9E7AE
:10A268000E23F7E70F23F5E70323F3E7B8190020D8
:10A2780010B50446002845D00168002942D011F8DD
:10A28800013B43710322063002F0FEF82046032208
:10A2980050F8091B043102F0F7F82168CB79E36024
:10A2A8000A7A43EA0223E3604A7A43EA0243E36014
:10A2B8008A7A43EA0263E360CB7A23740B7B637484
:10A2C8002379212B1AD110220D3104F1120002F04A
:10A2D800DBF81D222168501C8B5C6362085C43EA32
:10A2E8000023901C6362085C033243EA0043636204
:10A2F8008A5C43EA02636362002010BD112B03DC11
:10A308000D22E7E70220F8E70120F6E710B504463A
:10A31800002854D00168002951D00B7843714B783C
:10A3280083608A7843EA02238360CA7843EA024357
:10A3380083600A7943EA026383604B7903738B79FC
:10A34800C381CA7943EA0223027BC38102F00F0268
:10A358000831103002F098F8237B002203F00F0335
:10A3680084F8202084F82820227903F10800111AA3
:10A3780004290DDD21680933043AD21A085C84F8EF
:10A388002000D2B2606A84F82820194402F07CF8D0
:10A39800237922681A44002012F8043CE36212F878
:10A3A800031C43EA0123E36212F8021C43EA014357
:10A3B800E36212F8012C43EA0263E36210BD022053
:10A3C800FCE710B5044660B3036853B30279162A54
:10A3D80029D942791A700146082251F8060B013032
:10A3E80002F05CF82146082251F80E0B093002F001
:10A3F80055F82368E28A5A74E38A22681B0A937420
:10A408002368A269DA74A36922681B0A1375236892
:10A41800628B5A752368E27E9A7517232371002090
:10A4280010BD0120FCE70220FAE738B504460028F1
:10A4380063D00168002960D0037B90F8282003F0DE
:10A448000F03002A57D10833207904321344984265
:10A4580055D363790B702368A2685A70A368226881
:10A468001B0A937023686289DA702368E27A1A718A
:10A478002368227B5A712368E2899A71E3892268EA
:10A488001B0A2146D371227B51F8100B02F00F02F0
:10A49800083001F0F9FF237B94F8282003F00F031C
:10A4A80003F108052AB1226894F82010515503F1E8
:10A4B8000905206894F82820616A284401F0E4FF1F
:10A4C80094F828302268E16A2B44D1545A1CE16A76
:10A4D800206892B2090A81549A1C2168E08D92B2D0
:10A4E8008854DA1C216894F82F0092B204338854F7
:10A4F8002371002038BD0933A6E70120FAE70220BE
:10A50800F8E70000024B1A8810431880704700BF14
:10A51800BC19002008B5074B1B883BB1FEF7CAF9E8
:10A52800002814BF6FF00200002008BD6FF0010082
:10A53800FBE700BFBC19002010B5034B00241C80AA
:10A54800FEF7AEF9204610BDBC190020B0FA80F025
:10A558004009704782B018B9084602B000F0CAB87E
:10A56800002002B0704710B9084600F077B970476C
:10A5780010B9084600F08EB97047034608461146E0
:10A588000BB900F0E5B90020704710B9084600F093
:10A598006DBD704710B9084600F006BA0020704734
:10A5A80010B40446084611461A46019B14B910BC5B
:10A5B80000F014BA10BC70470346084611460BB9A0
:10A5C80000F03EBA0020704710B404460846114611
:10A5D8001A4614B910BC00F0ABBA002010BC704782
:10A5E80030B40546084611461A46DDE902341DB95D
:10A5F800029430BC00F02ABB002030BC704710B970
:10A60800084600F0DBBB0020704710B9084600F090
:10A618006BBD0020704710B9084600F0EABB002067
:10A62800704710B9084600F0E7BB002070470346A2
:10A63800084611460BB900F001BC0020704710B461
:10A648000446084611461A46019B14B910BC00F08E
:10A65800F7BB092010BC704710B4044608461146E1
:10A668001A4614B910BC00F061BDC8B210BC7047DE
:10A678000048704701000102064B10B51B6A0446EA
:10A68800984730B10448054B204498428CBF0020BD
:10A69800012010BD6CF9000840C220C980B92A0009
:10A6A800F0B5114B85B00C4610491F56054601F010
:10A6B8004BF80F4BE4B25E6A072D4FF00103CDE96A
:10A6C800024301460AD105220023CDE900234FF4B5
:10A6D8007A727A431846B04705B0F0BD08220020C8
:10A6E800CDE900203A46F5E750F3000830F30008BA
:10A6F8006CF900081FB5002300930378013B372B42
:10A7080021D8DFE803F01C242020201E2020202050
:10A718004143454E2055585B5E6164206C1E6E7344
:10A72800787A20207D8126202020202020202020AB
:10A738002020202083858A2020838A208C90C3783B
:10A748000BB102230093009805B05DF804FB8378F1
:10A75800F6E743788DF8043005238DF805308378C3
:10A76800003B18BF01235B008DF8063010238DF8DD
:10A778000730304B1B6801A803F55872CDE9022356
:10A7880000F0C2FF0090DEE74023DBE72023D9E793
:10A79800827890F9013012B9274AD35CD2E7274A68
:10A7A800FBE7827890F90130002AF8D1244AF4E7CF
:10A7B80040F6B833C6E74FF47A73C3E74FF4FA6349
:10A7C800C0E741F28833BDE741F27073BAE71D482C
:10A7D8004FF47A7101F03CFE00F5FA60D2E71A4BAB
:10A7E800B0E7144B1B6803F55873ABE7114B1B68B4
:10A7F80003F55B73A6E71023A4E70E4B1B68A1E7DC
:10A808004FF0834300939EE7104BFBE7104B99E70B
:10A8180040F21113ADF8003095E7032392E790F961
:10A8280001300C4AB9E70C4990F9010000F08CFF9F
:10A83800A8E700BFC419002025F3000815F3000895
:10A848001DF3000818FCFFFF00EA06379A99094033
:10A8580040F7093750F3000830F3000837B50B4BC1
:10A8680002781B680C2101FB02335B7A03EB43047B
:10A87800074B1D6803690093C3684278816805EB3C
:10A88800C40000F0DDFC03B030BD00BFC4190020D7
:10A89800C019002070B586B0027B6423ADF8003083
:10A8A800012A4FF00003CDE90133CDE903338DF8D8
:10A8B80002308DF8143030D0022A39D05ABB0368E0
:10A8C8004BB343683BB31F4D80682B601E4B182267
:10A8D8006946186001F0D8FD1C4B2C6893E8070006
:10A8E8000C3384E8070093E8070004F10C060323FF
:10A8F80086E80700A4F86C33012204F55B7104F5BF
:10A90800587000F08EFC2B684FF6B072A3F87823CD
:10A918000522C3F87C2306B070BD0A490868436065
:10A92800036100F55B7100F5587000F07AFCF2E7FE
:10A93800044B1B68B3F86023B3F86C130A43A3F8FD
:10A948006023E8E7C4190020C019002078F0000847
:10A9580008B503460A2924D8DFE801F00623232393
:10A96800230B161B23212100BDE808400068FFF7D0
:10A9780083BE90F900009978052271B900F011FCA6
:10A98800003818BF012008BD052293F900000021F6
:10A99800F4E790F900005978EEE70221EEE7072284
:10A9A800F3E70020EFE7000008B502791AB1012AA1
:10A9B8000BD0002008BD084B01681B68012203F575
:10A9C800587000F02EFC0120F4E7034B01681B6867
:10A9D80003F55B70F5E700BFC4190020F7B505283B
:10A9E800144D1C46A8BF052058700E462946174628
:10A9F80000F0AAFE94F90130A070072B13D1322081
:10AA080000F0A2FD0C4BDB6D0546984704F10C02E3
:10AA180008340346019200943A463146284600F02D
:10AA280098FD03B0F0BD054A55F82310D05C00F03E
:10AA380083FDE7E730F300086CF9000850F30008DD
:10AA48002DE9F04F344F90F901607B68D0F80490FD
:10AA58008BB00446884698470546002859D1E37CC0
:10AA680073B92E4A2378126803EB4303990002EB6B
:10AA78008303D3F80490B9F1000F01D152F8019083
:10AA8800274B484613F906B0FB689847A37C2289F0
:10AA9800D7F818A00993072E28D100230121CDE962
:10AAA8000223204A0693CDE90431CDE90733052175
:10AAB800CDE900214FF47A7202FB0BF24CF25031CF
:10AAC8001846D047637C13B3174B995D7B6D0D31E6
:10AAD800C9B228469847E07C3246494600F046FE0F
:10AAE80088F8006001200BB0BDE8F08F0021012537
:10AAF8000823CDE90013CDE90715CDE90511CDE906
:10AB080003110292A1782B465A462846D9E7074BEB
:10AB1800DBE70020E7E700BF6CF90008C419002054
:10AB280050F30008854501001DF3000825F30008CF
:10AB38002DE9F04F8DB090F90130DFF8FCA0DFF877
:10AB4800FC90CDE90A123E4A12F903B00278DAF80D
:10AB580000300C2505FB02333A4A5B7A126803EB96
:10AB6800430302EBC303044693F9021090F9020071
:10AB780000F0E5FD3449064694F9010000F0E4FDD3
:10AB8800A26861688046304600F00BFD2178DAF84B
:10AB98000020D9F80C306943074650589847D9F82F
:10ABA8001C309C4694F901300025072B4FF47A633A
:10ABB800CDE90753CDE905552DD10123CDE903533F
:10ABC8000523CDE901534FF47A7303FB0BF300938C
:10ABD8003946434646F2A81228466746B8472378BE
:10ABE800DAF800200C214B4394F90110D05800F0FA
:10ABF800DFFDA18994F90100FFF752FD0B9B217B32
:10AC08001860D9F85430284698470A9B01201E70CE
:10AC18000DB0BDE8F08F01200823CDE90350CDE940
:10AC280001032A46CDF800B0654643463946A84791
:10AC380001200546D3E700BFC41900206CF90008BD
:10AC480050F30008C019002030F300082DE9F04F38
:10AC58008FB0002405468A46914698460494ADF87C
:10AC68001440ADF8024007264FF0010B2B7AA3429F
:10AC780006D9686804A9204400F0F6FB00285ED1D4
:10AC880002238DF8083002A86B7A8DF80A30FFF796
:10AC980031FDAB7A8DF81D309DF811308DF81E30DE
:10ACA8009DF812308DF81F309DF810308DF8203047
:10ACB800EB7A8DF821302B7B8DF822306B7B8DF869
:10ACC800233010238DF81C608DF824303A4E8DF80F
:10ACD8002C000DF102030A9305238DF82D303368FB
:10ACE8000C930723ADF834302B6806930DF112024C
:10ACF80004AB0DF1110106A800F0D0FB07280546AA
:10AD08000BD130680C22002100F5587001F0D0FBFF
:10AD18003368BDF80220A3F860239DF811308AF843
:10AD280000309DF8123089F800309DF8103088F80E
:10AD38000030189B28461C700FB0BDE8F08F9DF8B6
:10AD48001330BDF81470ADF802702044C4B2F3B9E2
:10AD580017B3194A00201168072602464FF00C0C59
:10AD6800062B1BD10CFB00FE51F80EE0BEF1000FC4
:10AD780004D00BFA00F23A4397B2012201301028AE
:10AD8800EED1002A3FF472AFADF802706EE75A1E9A
:10AD9800042A01D9062BDCD0062667E747FA00FE0D
:10ADA8001EF0010FEAD00CFB00FE51F80EE0BEF1D8
:10ADB800000F08BF0626E1E7C419002038B505468C
:10ADC8004068FFF759FC0522841D002195F9000011
:10ADD800E4B200F0E6F908B904F0FD0495F90100C1
:10ADE8000722002100F0DDF908B904F0FB04204631
:10ADF80038BD00207047000010B503780F2B0446BB
:10AE080018D84068FFF738FC22780B4902EB420259
:10AE18000968831C01EB820051F82220DBB21AB9C1
:10AE280003F0FD0358B210BD032B06BF62684260F1
:10AE38000223F7E70020F6E7C41900200220704734
:10AE48002DE9F04FDFF838810446D8F8000099B0B2
:10AE58008946174600211E460122032300F5587033
:10AE6800CDE90611CDE908118DF814108DF81510EB
:10AE7800ADF8163000F0B7F938B9D8F80020B2F8B4
:10AE8800603343F00303A2F86033D8F80020637AF4
:10AE98008DF8283002F55871CDE90B12394A94F92A
:10AEA800083012680D920DF116020F922268109266
:10AEB80062681192D4E90301A27A8DF84820012230
:10AEC8008DF8492013AA82E803001025227DE18A23
:10AED8008DF8293018468DF85420ADF83850FFF712
:10AEE800DFFB0AAB17930DF115031690009331465B
:10AEF800019705AB06AA10A800F0C2FB064698BB4E
:10AF08009DF81410204F013901F0A2FA1F4B1B695C
:10AF18000393C4B24FF00C0B04F160036B44D8F8F0
:10AF2800000013F848AC9DF814300BFB0AFC013400
:10AF38003946B4FBF3F203FB1244D0F87C33B0F982
:10AF4800782350F80C00DDF80CC0E4B2E04728B1D3
:10AF580089F800A0304619B0BDE8F08F013D15F022
:10AF6800FF05D9D10D26F5E70C2801BFD8F8002038
:10AF7800B2F8603343F00303A2F86033EAE700BF96
:10AF8800C4190020C0190020400D03006CF9000806
:10AF9800F8B50679012E054648D90F2E48D803681A
:10AFA800187A40F303000522002140B200F0F9F8B6
:10AFB8002B680446187A40F303100522002140B29A
:10AFC80000F0EFF8B8B1B4FA84F4640929680B7A90
:10AFD800086843F3030243F303135BB252B29A4285
:10AFE800C8BF0124FFF748FB80F00103DBB224B19E
:10AFF8000533D8B2F8BD0124E8E7DBB90E4F29685C
:10B008003B6806EB460003EB80000C2201F03CFA9B
:10B018003A680C2303FB062320465C72B2F86013DF
:10B028000123B3400B43A2F86033E3E70620E1E7CE
:10B038000320DFE70420DDE7C419002010B40178FD
:10B0480001290ED9084B18680C234B43C418002259
:10B05800C250C4E9012200F5587010BC102200F05B
:10B06800A9B8002010BC7047C41900202DE9F04190
:10B0780086B050238DF81430037A102B074630D150
:10B088004368DD7B6DBB0224A8466426062C14D8D1
:10B098007A68535D03932A44517843EA0123039362
:10B0A800927843EA02437343CDE9033863B96846AB
:10B0B8008DF80040FFF7C2FF0DE0CDF80C808DF849
:10B0C8001480CDF81080F2E703AB01A801938DF846
:10B0D8000840FFF75DFF0134E4B2102C05F10305C9
:10B0E800D4D106B0BDE8F0811FB5026803791168B4
:10B0F80049B901A88DF80430FFF7A0FF78B1032003
:10B1080005B05DF804FB02A802928DF80C30FFF739
:10B118003FFF042805D0052805D00028EFD00020DF
:10B12800EEE70220ECE70120EAE70000C90020B9B9
:10B13800034B0B449856C0B27047024BF9E700BF67
:10B14800D5F2000895F20008F0B59A42069D03DB97
:10B158009DF914309A4220DD0020F0BD03EB430333
:10B1680031F814C005EB830300264CFA06F7FF07F5
:10B1780007D51F7A07F00F0E964502DCB2EB171FB2
:10B188000DDD0136102E03F10C03EED10134E4B2CB
:10B198002301DBB29842E1D8DEE70024F8E701207A
:10B1A800DBE7884204DB9042CCBF002001207047D7
:10B1B8000020704710B51409B4EB111F03464FEA7D
:10B1C80011100ED391420CD202B201F00F0133F8E4
:10B1D8001240012000FA01F124EA010123F81210BB
:10B1E80010BD0020FCE7F0B528B100EB41050127B0
:10B1F8000020914200D3F0BD002435F802CB23464D
:10B2080007FA04F636EA0C0608BF013304F1010414
:10B2180008BFDBB2102CF3D118440131C0B2C9B257
:10B22800E7E710B500B149B910BD31F8134020F86F
:10B2380013400133DCB2A242F7D8F5E70023F9E75F
:10B2480082B030B504880493D2B9B3F5616F15D3D1
:10B2580049F6AF2542F21072AB4298BF4FF47A72AA
:10B26800944238BF14466143BDE83040C3688B42FE
:10B278008CBF5B1A0023C36002B070476422EFE7FB
:10B28800012C38BF0124EEE72DE9F04F8FB01546A9
:10B29800199F03939DF8603007930C46804603F08E
:10B2A800C7FB6A4A0590A7F5F633303BB3FBF2F3C8
:10B2B800534303F5F63B0493182313FB05430BF1A3
:10B2C800300B069300254FF0FF3A069B9C4207D1AE
:10B2D800002D14BF50464FF0FF300FB0BDE8F08F7F
:10B2E800BDF96830ADF824300999199738460897A0
:10B2F80003F02EFB2688B8F1000F5FD1B7F5616F18
:10B308005AD349F6AF2242F21073974298BF4FF4CE
:10B318007A739E4238BF1E46642E59D1DFF83091A9
:10B32800A060A1680CA803F035FB0D9B0093DDE934
:10B3380008120C9B0AA803F08CFA039A0A9B0AB914
:10B34800079A2AB122694A4502D1424A93420ED944
:10B35800414BC4F80C909F4209D90023ADF82C301A
:10B368000B99CDF828B0584603F0F2FAA06060684F
:10B3780008B9C4F80C90C4F81090B8F1000F04D0C4
:10B3880003F060FBE3680344E360D4E903329342CB
:10B39800059B88BFE26063601B9BE1687343994229
:10B3A80004D20398E8B9B8F1000F1AD001231D445C
:10B3B8002375EDB2183488E76423AAE7039B0BB919
:10B3C800234BE360012EDFF8889038BF0126CEE7D3
:10B3D800B6F57A7F0ABFDFF88490DFF88490A06022
:10B3E8009FE700209342207506D85B1A9A4505F11D
:10B3F800010528BF9A46EDB2B8F1000FDAD1642EE4
:10B40800184AADF82C801DD049F6B023B6F57A7FDE
:10B4180018BF1346974281BF049A02F5A83202F575
:10B42800C0729B180A931A9B00930AAE96E806000E
:10B43800199B304603F00DFA96E8030003F088FAEA
:10B448008246B7E74FF46163E4E700BF805101002B
:10B4580040771B007F5101002FEC010080A81201EA
:10B46800002E930230EC01000378032B14D14378AB
:10B4780003F00F021B098A704B7083788B80C278A7
:10B4880043EA02238B800379C3F3021203F00F030C
:10B49800CA700B7005207047002070472DE9F347EC
:10B4A8009A464379057990F907609146044690F9E0
:10B4B80006208846D3B190F90870002D37D00F2A9E
:10B4C8001BD194F909200F2E27D194F90A00072DD2
:10B4D80002D1002F08BF012788F8002089F8000052
:10B4E80028468AF8007002B0BDE8F08790F90B7022
:10B4F80090F9092090F90A60DFE7A369019394F9AC
:10B508001530009394F914302169207BFFF71CFE55
:10B518000028D8D105F0FD05D5E794F91D00B04203
:10B52800D5DC94F91C30B34203DA05F0FB0530464C
:10B53800D2E73046CBE70000024B03FA00F0B0FB3D
:10B54800F1F0704740420F004FF4FA53B3FBF0F0AC
:10B55800704730B54FF47A750C1F6A4300FB04221C
:10B5680052001EBF00F1FF341219B2FBF0F29142F3
:10B5780038BF1146039A1160820048431CBF01304E
:10B5880040084FF47A71121A01FB1323002BCABF2B
:10B5980003F2E73393FBF1F1B3FBF1F1049B19607C
:10B5A80030BD38B5400014460D46F5F70BF9014695
:10B5B8002846F5F755F82146F5F752F8F4F744FF11
:10B5C80003F0AEFCF5F720F840B238BD2DE9F74F8F
:10B5D800019300239C469E46048A1E01F6B2B4429B
:10B5E80046D906EB46054FEA4309AD0000244768F3
:10B5F80037F809702741FF0729D5876807EB050A3F
:10B608007F5927B3077837B9476927B137F80970E1
:10B618002741FF071BD59AF8087090F901B047F346
:10B6280003084FFA88F8D84511DC47F303177FB2AF
:10B638005F450CDB9AF8097007EB4708C76807EB0A
:10B64800C8073F7D5FB90CF1010C5FFA8CFC01342F
:10B65800102C05F10C05CAD10133DBB2BCE70EF1A1
:10B66800010706EB040801F80E805FFA87FEEEE793
:10B67800019B82F800E083F800C003B0BDE8F08FBA
:10B688002DE9FF4704464068DDE90C671D468A46F8
:10B69800914603F0D7F923681B1A3B604FF0000866
:10B6A8000123337085F80080636813B123688342EF
:10B6B80024D8D4F81CC0CAF80080A3699CF800E01C
:10B6C8000393D4E9030101AB83E80300237D0093CE
:10B6D800DCF80C10237A627A7046FFF7D5FD334602
:10B6E80038602A46E0694946FFF770FF2B782BB18E
:10B6F800C7F80080002004B0BDE8F0873378002B3D
:10B708000CBF0C200B20F6E737B590F9002090F914
:10B718000250954204460FD0013A52B295420BD0DE
:10B72800A368019394F9013000936168E0782B468F
:10B73800FFF70AFD0028EFD0104603B030BD88425D
:10B74800B8BF08467047000051F82000054B9842E2
:10B7580005D0054BC31A5842584140007047012094
:10B76800704700BF90D0030020A1070005281FB52F
:10B778000ED80C4B53F820300093CDE901120A4B38
:10B7880001220021022002F06BFE05B05DF804FBE7
:10B79800CDE90012054B01220021022002F060FED3
:10B7A800F3E700BFC4F3000858F3000877F3000874
:10B7B80007B5054BCDE9000101220021022002F066
:10B7C8004FFE03B05DF804FB93F3000810B5102298
:10B7D80004460021F13000F06BFE0021C4F814117A
:10B7E8002046F022BDE8104000F062BE024608463E
:10B7F800102100F0A5B92DE9F0430446D0F8140152
:10B8080085B00E46154604F2011988B3C0F1100838
:10B818009045474628BF1746BAB2484400F034FE60
:10B82800D4F814313B440F2BC4F814312DD9A84552
:10B838002BD204F1F00304F5807113F8012F187C62
:10B848008B4282EA00021A70F7D104F1F108102243
:10B858004146684600F018FE22466946684600F0F0
:10B86800F1F910226946404600F00EFE3E44ED1BF9
:10B8780004F5807804F1F107102D09D8AAB23146F1
:10B88800484600F001FEC4F8145105B0BDE8F08345
:10B8980004F1F003711E13F8012F11F8010F43454D
:10B8A80082EA00021A70F6D110223946684600F082
:10B8B800EBFD22466946684600F0C4F91022694645
:10B8C800384600F0E1FD1036103DD5E7F0B589B0F7
:10B8D8000C46102200210546684600F0E9FD224684
:10B8E8006946684600F0AEF99DF90030002B6A46BB
:10B8F8004FF0000143DA137812F8010F01315B00B1
:10B9080043EAD0130F2902F8013CF4D19DF80F3017
:10B918005B0083F08703D4F81401DBB210288DF89C
:10B928000F303BD104F58073694604F5887013F82D
:10B93800016F11F8012B984282EA06021A70F6D1BB
:10B9480004F1F00304F5807113F8012F187C8B4281
:10B9580082EA00021A70F7D110220DEB020004F1FE
:10B96800F10100F091FD2246294604A800F06AF989
:10B9780010220021684600F09BFD09B0F0BD137845
:10B9880012F8010F01315B0043EAD0130F2902F8C6
:10B99800013CF4D19DF80F305B00BCE79DF9003005
:10B9A800002B6A464FF0000137DA137812F8016F5E
:10B9B80001315B0043EAD6130F2902F8013CF4D1A8
:10B9C8009DF80F305B0083F08703471CDBB28DF8CE
:10B9D8000F30102F04EB0003C0F10F064FF0800268
:10B9E80088BF002600F5817083F8012100213246C6
:10B9F80020443E4403F066FAC4F8146104F58073E9
:10BA0800694604F5887013F8016F11F8012B984204
:10BA180082EA06021A70F6D192E7137812F8016FDB
:10BA280001315B0043EAD6130F2902F8013CF4D137
:10BA38009DF80F305B00C8E70A780378534003701D
:10BA48004A784378534043708A78837853408370A8
:10BA5800CA78C3785340C3700A7903795340037195
:10BA68004A794379534043718A7983795340837182
:10BA7800CA79C3795340C3710A7A037A534003726F
:10BA88004A7A437A534043728A7A837A534083725C
:10BA9800CA7AC37A5340C3720A7B037B5340037349
:10BAA8004A7B437B534043738A7B837B5340837336
:10BAB800CA7BC37B5340C373704710B50B781478A7
:10BAC8006340037054784B786340437094788B7864
:10BAD80063408370D478CB786340C37014790B7952
:10BAE8006340037154794B796340437194798B793E
:10BAF80063408371D479CB796340C371147A0B7A2C
:10BB080063400372547A4B7A634043728B7A947A17
:10BB180063408372D47ACB7A6340C372147B0B7B05
:10BB280063400373547B4B7B63404373947B8B7BF1
:10BB380063408373CB7BD27B5340C37310BD00003B
:10BB4800A1F11003DBB2102B2DE9F047044604D80D
:10BB58003A4820FA03F3DB0705D4002382F8F030D3
:10BB6800FF20BDE8F087561E254615F8013B06F86C
:10BB7800013F631B0B4413F0FF00F6D101F11C03D6
:10BB88009B005FFA83FCC3F30313013BDFF8B0901B
:10BB980082F8F030884653184FF0010EB8FBF1FADE
:10BBA80001FB1A8A1AF0FF0A13F8047C13F8036CD5
:10BBB80013F8025C13F8014C30D119F806A019F8F3
:10BBC800056019F8045019F807404FEADE1707EB2B
:10BBD80047078EEA0A0A07EBC7074FEA4E0EFFB27D
:10BBE8005FFA8EFE87EA0E0E574692F800A087EAA3
:10BBF8000A071F7057787E405E70967875409D7072
:10BC0800D57808F104085FFA88F86C40C445DC7000
:10BC180002F1040203F10403C0D8A2E71829E4D909
:10BC2800BAF1100FE1D1DFF818A01AF807701AF866
:10BC380006601AF805501AF80440D6E70101010019
:10BC4800DCF500082DE9F04FA3B092F8F0301D9113
:10BC58001B920193002B00F0538101461EA8FFF7A9
:10BC68002CFF1B9BA74CA84DA84E10330293002312
:10BC780003939DF87C0004909DF886000590205C55
:10BC880006909DF87B000790205C089004989DF82A
:10BC980081C0205C099014F80C000A909DF880007F
:10BCA8000B909DF885009DF878809DF87DE09DF8C3
:10BCB80082A09DF887900C909DF87A00029B1C93B7
:10BCC80014F80A2014F8093014F8081014F80E7043
:10BCD8000D90205C0E909DF87F000F90205C1090D6
:10BCE8000B98205C11900C98205C12909DF88400B1
:10BCF80013909DF8790014909DF87E001590205CB3
:10BD080016909DF883001790205C18901398205C7B
:10BD180019901498205C1A900398013003900298A7
:10BD2800DDF804B0103002909DF80C00834536D839
:10BD38008DF878108DF87A2009990E9A8DF87C1074
:10BD48008DF882201199069A8DF880108DF87E2042
:10BD58001999169A8DF884108DF886200A99189AE0
:10BD68008DF87D108DF887201299109A8DF87B3008
:10BD78001B9B8DF881108DF883201A99089A1D98BD
:10BD88008DF885108DF87F201EA903EB0B128DF816
:10BD98007970FFF792FE002023B0BDE8F08F15F808
:10BDA80008B082EA03008BEA000016F80EB080EAB9
:10BDB8000B008DF8780015F80E004B40434016F83C
:10BDC8000A0043408DF8793081EA070315F80A1014
:10BDD800594016F80930594016F808308DF87A108D
:10BDE8007A40534015F8092053408DF87B30089A63
:10BDF800069B5340049AAA5C534016F80C20534003
:10BE08008DF87C30DDE908325A4015F80C30534083
:10BE1800059AB25C53408DF87D30DDE909325A400D
:10BE2800059BEB5C5340079AB25C53408DF87E301B
:10BE3800069B0A9A5340049AB25C5A40079BEB5CF3
:10BE48005A408DF87F200E9B109A53400B9AAA5C9B
:10BE580053400C9AB25C53408DF88030DDE91032C3
:10BE68005A400C9BEB5C53400D9AB25C53408DF8E2
:10BE78008130DDE911325A400D9BEB5C53400F9A3B
:10BE8800B25C53408DF88230129A0E9B53400B9A45
:10BE9800B25C5A400F9BEB5C1C995A408DF883208A
:10BEA800169B189A5340139AAA5C5340149AB25C92
:10BEB80053408DF88430DDE918325A40149BEB5C0E
:10BEC8005340159AB25C53408DF88530DDE919323C
:10BED8005A40159BEB5C5340179AB25C53408DF85F
:10BEE80086301A9A169B5340139AB25C5340179A9D
:10BEF800AA5C1EA853408DF88730FFF79DFDB8E671
:10BF0800FF2049E7DCF50008DCF40008DCF3000852
:10BF180008B538B1044A05491060D82200F0B4FACF
:10BF2800002008BD0220FCE7C81900200CFB00080F
:10BF38000A4B1A6870B5002302F1180503EB0314C5
:10BF48002E5D864204D1183422440A60002070BD58
:10BF580001330B2BF2D10320F9E700BFC8190020E9
:10BF68002DE9F041CCB00646DDF8488117461C465D
:10BF78000D4631B3B8F1000F23D006A8FFF726FC11
:10BF8800204601A9FFF7D4FF0446B0B9019906A8D5
:10BF98000131FFF72BFC26B11022314606A8FFF726
:10BFA8002AFC3A46294606A8FFF725FC06A902A856
:10BFB800FFF78CFC029BC8F8003020464CB0BDE867
:10BFC800F0810224F9E7000030B595B013A90446C2
:10BFD800FFF7AEFF002830D11B4B0C2101FB00F20C
:10BFE800D5189A5CA2422AD1139B1A7C1092DA7B4C
:10BFF8000F929A7B0E925A7B0D921A7B0C92DA7AE8
:10C008000B929A7A0A925A7A09921A7A0892DA79EB
:10C0180007929A7906925A7905921A790492DA78EF
:10C0280003929A7802925B7801930022AB6800939E
:10C038001146064B022002F013FA15B030BD01304C
:10C048000B28CBD1F9E700BF54F80008DCF600084C
:10C0580010B40B2B019C03D8019410BCFFF780BFD0
:10C06800032010BC704730B50D4685B01446014614
:10C0780068B103AA002000922A460390FFF770FFD8
:10C0880018B90398001B18BF012005B030BD022065
:10C09800FBE72DE9F0430D46BFB0144699468046AC
:10C0A80020B31BB311F00F0122D1F02201A800F038
:10C0B800FFF920466946FFF73BFF044648B9009858
:10C0C80001AA10210130FFF73BFD2E46AF1BFFB23E
:10C0D8001EB920463FB0BDE8F08301AA09EB07016D
:10C0E80008EB0700FFF7AEFD103EEFE70224F0E78C
:10C0F8000524EEE7F0B5184E3468024685B00846C8
:10C10800002304F1180103EB03154F5D97421ED17C
:10C118000D2A05F1190513D10023CDE90033CDE926
:10C1280002330C2210216B46FFF7B3FF0446306838
:10C1380010226946284400F0A7F9204605B0F0BD52
:10C1480001461022601900F09FF90024F5E7013339
:10C158000B2BD8D10324F0E7C819002009B1FFF749
:10C16800C9BF022070471FB51446A0B10C2A01D1DF
:10C178000B2912D10023CDE90033CDE902330A4659
:10C188006B461021FFF785FF18B969462046FFF76F
:10C19800B1FF04B010BD0220FBE70320F9E7F8B5B2
:10C1A8001E46DDE907479DF818505BB354B34FB3FB
:10C1B800212D29D819462A46204600F065F9012282
:10C1C800631C691EB018FFF764FFF8B9E37ADB094E
:10C1D8003B70EBB96319204613F8012C13F8021CC5
:10C1E800120642EA014213F8041C0A4313F8031C1E
:10C1F800012342EA0122291FFFF735FF003818BF43
:10C208000120F8BD0220FCE70520FAE70720F8E73F
:10C218000420F6E710B5044628B1044B5B6998473B
:10C228002060002010BD0220FCE700BF6CF9000868
:10C2380008B5014630B1044B0822186800F024F90B
:10C24800002008BD0220FCE7C819002008B530B15D
:10C25800044B0822196800F017F9002008BD0220D5
:10C26800FCE700BFC81900207FB5124E0023044622
:10C2780002A801930D46FFF7E9FF33685B69019354
:10C288006CB102AA082312F8011B41B9013B13F053
:10C29800FF03F8D102A8A04702A8FFF7C9FF35B1EC
:10C2A800019B23B901A8A8473368019A5A61002065
:10C2B80004B070BDC819002008B5014638B1054B57
:10C2C80018680822104400F0DFF8002008BD02209A
:10C2D800FCE700BFC819002008B538B1044B19683D
:10C2E8000822114400F0D0F8002008BD0220FCE725
:10C2F800C8190020034B1B6802280CBF196159613B
:10C3080000207047C819002049B1064B1B68D3E9C3
:10C318000423022808BF13460B6000207047022040
:10C32800704700BFC819002030B58FB000240546FB
:10C338000CA80994FFF78AFF9DF8373007939DF8FA
:10C34800363006939DF8353005939DF834300493C4
:10C358009DF8333003939DF8323002939DF83130C5
:10C3680001939DF830300093224621461E4B02204F
:10C3780002F076F80AA8FFF7AFFF9DF82F30079371
:10C388009DF82E3006939DF82D3005939DF82C309E
:10C3980004939DF82B3003939DF82A3002939DF85F
:10C3A800293001939DF82830009322460F4B2146EF
:10C3B800022002F055F809A92846FFF7A5FF9DF8C5
:10C3C800243003939DF8253002939DF8263001937D
:10C3D8009DF8273000932246054B2146022002F0A3
:10C3E8003FF80FB030BD00BF38F7000876F70008F7
:10C3F800B4F7000808B50020FFF7E6FD0120FFF7B5
:10C40800E3FD0920FFF7E0FD0820FFF7DDFD002030
:10C41800FFF78AFF002008BD10B504460B20FFF780
:10C42800D3FD0C20FFF7D0FD0920FFF7CDFD082034
:10C43800FFF7CAFD0A20FFF7C7FD2046FFF774FF84
:10C44800002010BD014B1860704700BFF8000020A5
:10C458000B4A30B514680B4D43F2390305FB04331E
:10C468001360091A6FF00042B3FBF2F2C2EBC2721A
:10C4780001319B1A93FBF1F201FB1233184430BDD2
:10C48800F80000206D4EC64101380A44914200D19F
:10C49800704711F8013B00F8013FF7E710440A44E0
:10C4A800914200D1704711F8013B00F8013DF7E7D0
:10C4B80002F008BD30B530B10A4D01444FF0FF33EA
:10C4C800814201D1D84330BD10F8012B53400822D6
:10C4D80043F30004013A2C4092B284EA5303002A41
:10C4E800F6D1EDE72083B8ED01207047054B4FF4F6
:10C4F80000529A62044B1B6813B15B6803B118477A
:10C50800704700BF00040048581A0020054B4FF43C
:10C5180080529A62044B1B6813B1DB6803B1184759
:10C52800704700BF00040048581A002001207047D7
:10C538000120704701F03EB901F02CB910B501F0A7
:10C548000FFE0E21044640F61F1001F023F9204685
:10C55800012101F0EFFDBDE8104001F0CDBA000067
:10C5680070B50C4E01EB40030D46B3654FF6FF71F5
:10C57800002304461A46084601F054FB96F8560074
:10C58800002101F0D7FD29462046BDE8704001F0A2
:10C598008BBA00BFFC19002010B5044601F0A0FEBC
:10C5A80001281CD101F0A4FE34B11248214602F042
:10C5B8000BFB104802F0CEFA0F4C104B00214FF441
:10C5C8008052A1659A6194F8560001F0B3FD637832
:10C5D8006BB16FF07F40BDE8104001F049BA00230D
:10C5E80040F262211A46084601F01CFBDCE7A0680D
:10C5F8008001F0E7CC190020FC1900200004004855
:10C60800002001F0B5B9000008B501F0BDF8043804
:10C61800C0B2032896BF024B0020185C08BD00BFBB
:10C6280036F9000808B501F0B0FD033008BD01F087
:10C638003FB901F0FFB808B501F0F6FC08BD0000ED
:10C6480038B50D46144601F053FB284601F088FD25
:10C658000E21054640F61F1001F09CF828460121DE
:10C66800074D01F067FD01F047FA4FF47A71614315
:10C67800284602F0A9FA2846BDE8384002F06ABA0E
:10C68800E419002001F034BB08B5084B002193F8E9
:10C69800560001F04FFD00234FF4C0711A460846BA
:10C6A80001F0C0FABDE8084001F01ABAFC190020F0
:10C6B80010B5044601F014FE01281CD101F018FE43
:10C6C80034B11248214602F07FFA104802F042FACB
:10C6D8000F4C104B00214FF48052A1659A6194F8D9
:10C6E800560001F027FD63786BB16FF07F40BDE81D
:10C6F800104001F073B9002340F262211A4608463F
:10C7080001F090FADCE7A0688001F0E7CC1900207E
:10C71800FC1900200004004808B54FF0040001F09F
:10C728000DF9BDE808400220F5F7E4B808B5002384
:10C738001A461946184601F075FABDE8084001F096
:10C7480063B900001D4B73B51D4D186000241D48CA
:10C758006C70C5E90144AC6501F08EFAAC8101F05A
:10C76800F9F92146204601F041FC21460422012026
:10C7780001F0F2FA144E154D4FF6FF71234622468A
:10C78800084601F04FFAFFF7C7FF2246104B009406
:10C798004FF0FF31304602F031F90E4B009422463B
:10C7A8004FF0FF31284602F029F9304602F084F9AB
:10C7B800284602B0BDE8704002F07EB9581A002041
:10C7C800FC19002081D70008E4190020CC190020AA
:10C7D800F5C4000815C500080128084805D1084B0C
:10C7E800C17719700E3001F09DBB437D012B03D139
:10C7F800034B81751970F5E7704700BFFC190020DD
:10C80800FC0000200D4B10B5044618735873012026
:10C8180000F016F85CB134214FF4E86000F0BAFF7C
:10C828004421BDE8104040F2417000F0B3BF14212C
:10C838004FF4E86000F0AEFF2421F2E7FC19002075
:10C8480038B5114C0546207001F057FD052D04D868
:10C85800DFE805F0090B03171709032001F066FA52
:10C868000023637338BD0020F8E7012001F05EFA69
:10C87800207B637B8342F5D06073BDE83840FFF7C7
:10C88800C1BF0220EAE700BFFC1900202DE9F043F0
:10C898001E4687B000230546CDE901330C461746EE
:10C8A80001F01DFD032D5BD8DFE815F07A00C1000B
:10C8B8000C010400A27C082A69D8A16801A801F02B
:10C8C800D5FE2168002962D042F210729142E37CC1
:10C8D800874D50D80322AA7385F83820E96385F874
:10C8E80044304FF002086368A17DDB002B820423EB
:10C8F800AB74A37CDB00EB7402294FF000032B75AB
:10C90800637D02D0227D022A46D103F10F02D2B202
:10C91800012A01D9012B3AD1764B774A1968039439
:10C928004FF0010903A88DF8149001F0D5FC70BBF5
:10C93800287685F817906875FFF762FE4046FFF77E
:10C948007FFF6E4801F082FA6D4801F0EBFA01A80A
:10C9580000F080FF208A00F051FFA08900F096FFC8
:10C96800384601F0FDFB624C84F8560001F0BCFC2F
:10C97800666000200DE04FF00008E963890885F83B
:10C988000E8085F8388085F844302964ABE74FF08D
:10C99800FF3007B0BDE8F083EB7529766A75CBE701
:10C9A8002368002BF3D0A27C082AF0D8504DA16848
:10C9B80001A801F05BFE002385F838302268EA639D
:10C9C800E27C85F84420A269AB732A646268D200CD
:10C9D8002A820422AA74A27C2B75D200EA74A27D52
:10C9E800022A02D0237D022B1CD1627D02F10F03A3
:10C9F800DBB2012B01D9012AC9D13E4B3E4A196845
:10CA080003944FF0010803A88DF8148001F064FC2A
:10CA18000028BCD1287685F817806875FFF7F0FDE7
:10CA280000208CE7617DE9752A766B75F6E7304D55
:10CA3800012185F83810227885F85020637885F828
:10CA48005130A37885F85230E3788B4202D0022B1C
:10CA580003D03BB985F8533004E00B3A012A29D8B2
:10CA680085F853104FF0010885F80E80A388AB8332
:10CA7800A379AB77E37985F82030237A85F82130DC
:10CA8800FFF7BEFD4046FFF7DBFE1C4801F0DEF96C
:10CA98001B4801F047FA95F85130062B40F68900FB
:10CAA8000AD100F087FE00F0FB0140F6890000F093
:10CAB80071FE55E70023CDE700F07CFE40F004014D
:10CAC800C9B2F2E72368013BB3F57A7FBFF45FAFE1
:10CAD8000320FFF7B5FE0648022380F838302368A4
:10CAE8008364162380F84C30383001F0AFF937E70B
:10CAF800FC190020581A0020E4190020341A0020DC
:10CB08000A1A0020F0B51E4687B00023CDE901338C
:10CB1800144607460D4601F0E2FB002C724C16BF86
:10CB2800012300230026637027B1012F7AD000204B
:10CB380007B0F0BDAB68002B00F0D280EB68002B8B
:10CB480000F0CE80AA7F082A00F2CA80296901A8CD
:10CB580001F08CFD2868003818BF012000F0D6FFCE
:10CB680084F83870AB68E36395F8203084F8443073
:10CB7800686801F057FBA77384F84500EB68DB0091
:10CB88002382EB7FA374AB7FDB00E37495F821303D
:10CB9800237595F82230002B3ED12A7D95F8241074
:10CBA800A275022995F8232001D0022B36D102F173
:10CBB8000F03DBB2012B02D9012A40F09180002338
:10CBC8008DF81430494B4A4A1968049503A801F0B6
:10CBD80083FB002840F0848001232076E37560758C
:10CBE800FFF70EFD0020FFF72BFE424801F02EF95B
:10CBF800414801F097F901A800F02CFEA88B00F03D
:10CC0800FDFD288B00F042FE4FF4FA53AA687343E7
:10CC1800B3FBF2F3A3608AE7FF22BFE7E275217650
:10CC28006375DDE72B8E002B5AD095F83230A86A51
:10CC3800012B0CBF2F7DFF27003818BF012000F003
:10CC480065FFF0B200F06EFF012184F8381095F806
:10CC58002C2084F8502095F82D3084F8513095F820
:10CC68002E3084F8523095F82F308B4202D0022BA8
:10CC780003D03BB984F8533004E00B3A012A27D893
:10CC880084F853102B8EA38395F83230A3770126AE
:10CC9800AB8E2384A673E777FFF7B2FC3046FFF725
:10CCA800CFFD144801F0D2F8134801F03BF994F88D
:10CCB8002130B34240F236700CD100F07BFD00F019
:10CCC800FB0140F2367000F065FD4FF6FF73A1E7F7
:10CCD8000023CFE700F06EFD40F00401C9B2F0E791
:10CCE8004FF0FF3024E700BFFC190020581A00203D
:10CCF800CC190020341A00200A1A00202DE9F04F20
:10CD080085B082460E9DBDF840809DF844709DF820
:10CD18004890019193461E4601F0E1FABAF1010FDD
:10CD2800524C54D0BAF1040F00F09180BAF1000FC0
:10CD38003AD10B22304684F8442084F838A0E563C1
:10CD480001F070FA4FEAC803B9F1000F238241F6E7
:10CD5800040363820CBF0123F223E37587F0010704
:10CD68000123237684F84500C4F840B084F80EA067
:10CD780084F814A06775FFF743FC5046FFF760FD81
:10CD880004F1380001F062F804F10E0001F0CAF86D
:10CD9800374A1068516802AB03C302A800F05AFD75
:10CDA80040F2FF1000F02AFD019801F0D9F90E2198
:10CDB80084F8560040F61F1000F0ECFC94F856007A
:10CDC80001F092FA169B636005B0BDE8F08F29491F
:10CDD80084F838A0EAB2895D84F8502076BB0B3D10
:10CDE800012D8CBF00250125053A012A04D8B8F188
:10CDF8000C0F38BF4FF00C081F4B9DF83C201B78D8
:10CE080084F85350E37701259DF8543084F8511085
:10CE180084F8522084F82130A573A4F81C80A777E1
:10CE280084F82090FFF7ECFB2846FFF709FD13482C
:10CE380001F00CF8124801F075F8B5E7012E04D19D
:10CE4800A5F10C035D425D41CEE70025CCE75046D5
:10CE5800FFF7F6FC022384F8383004F13800162373
:10CE6800A56484F84C3000F0F1FF9DE7FC19002020
:10CE780090F0000868F90008FC000020341A00202F
:10CE88000A1A00202DE9F04F87B0DFF8B4B29DF8F8
:10CE980064A09DF84C90029314469DF854309DF878
:10CEA8005020BDF84880039205468BF801A0BDF8D4
:10CEB800446001930F4601F012FABAF1000F18BF4F
:10CEC8004FF00008DFF87CA2039AB9F1000F08BF01
:10CED800FF22012D8AF8002000F0C880052D48D0D7
:10CEE800002D40F0C080284600F010FE0B22384686
:10CEF8008BF844208BF83850CBF83C4001F092F97D
:10CF0800019B8BF8450041F60402002BABF8122078
:10CF18009AF800208BF816200CBF0122F2228BF819
:10CF28001720F600012289F001098BF818208BF8E8
:10CF38000E50ABF810608BF814508BF81590FFF773
:10CF48005FFB2846FFF77CFC0BF1380000F07EFF02
:10CF58000BF10E0000F0E6FF7B490868496804AA57
:10CF680003C204A800F076FC40F2FF1000F046FC73
:10CF780071E0012000F0CAFD09224FF000098BF88A
:10CF8800442038464FF44872CBF840208BF838904C
:10CF9800CBF83C4001F046F94FF48052ABF8122030
:10CFA8009AF800208BF845008BF8162028460122B5
:10CFB800F6008BF817208BF80E90ABF81060ABF8E2
:10CFC80014908BF81890FFF73BFC0BF1380000F039
:10CFD8003DFF0BF10E0000F0A5FF5B498868C968AA
:10CFE80004AA03C204A800F035FC40F2FF1000F0C8
:10CFF80005FC40F6B80000F0DDFB00F0EF0140F65C
:10D00800B80000F0C7FB042140F6B90000F0C2FBED
:10D0180040F69B0000F0CEFB00F0E30141F0080170
:10D0280040F69B0000F0B6FB40F2D16000F0C2FB76
:10D0380040F01801C9B240F2D16000F0ABFB40F2F9
:10D04800AC6000F0B7FB00F08F0141F0500140F2F6
:10D05800AC6000F09FFB4FF4FA5202FB08F2B2FBFF
:10D06800F4F2CBF8082007B0BDE8F08F002000F0FC
:10D078004DFD36498BF83850E2B2C95D8BF8502027
:10D08800002F4DD10B3C012C8CBF00240124053A04
:10D09800012A02D80C2E38BF0C26029B9AF80020D1
:10D0A8008BF852308BF85340019B8BF81F200124DA
:10D0B8009DF860208BF821208BF851108BF82030D8
:10D0C8008BF80E40ABF81C608BF81E90FFF798FAAF
:10D0D8002046FFF7B5FB1E4800F0B8FE1D4800F0DB
:10D0E80021FF5FFA88F000F01DFD40F6A30000F074
:10D0F80061FB00EA040140F6A30000F04BFB9BF83B
:10D108002120A24240F2367013D100F053FB00F008
:10D11800FB0140F2367000F03DFB4FF6FF72A0E7CE
:10D12800012F04D1A4F10C035C425C41AFE7002459
:10D13800ADE700F03FFB40F00401C9B2E9E700BFEA
:10D14800FC190020FC00002090F0000868F9000895
:10D15800341A00200A1A0020F0B58BB00D46044698
:10D1680017461E46FFF74CFA0020FFF769FB2046DA
:10D1780000F0BEFD00240123CDE9084303234FF44A
:10D18800167229462046CDE90644CDE90444CDE986
:10D198000244CDE900532346FFF774FE2046FFF70B
:10D1A80087FAFFF73FFAF4F7A5FB01F041FC0446C4
:10D1B800204601F047FCB04205D30124FFF720FACE
:10D1C80020460BB0F0BD00F02FFF8742F0DA0024B4
:10D1D800F4E70000F7B500230C4640F201211A4697
:10D1E8000646084600F01EFD644B654D4FF400529C
:10D1F8009A6195F85600012100F09CFF2B78012BCD
:10D2080040F6890013D195F85130062B0FD100F064
:10D21800D1FA00F0FB0140F6890000F0BBFA2B7848
:10D22800042B6CD8DFE803F0524B527F090000F062
:10D23800C1FA40F00401C9B2EDE7524A731E104624
:10D24800C6F101074FF0000CF9188C426FDC002280
:10D25800E7001346BA4271D19A0142EAC3125B0150
:10D2680083F020031343661C0355F6B20223464895
:10D27800AB73AE7600F056FE0021F12000F08AFA7A
:10D288000021F02000F086FAAB6C642B70D170217D
:10D29800F32000F07FFA1D21F22000F07BFAE10074
:10D2A8008C1CF420090A00F075FA04F0FE01F52040
:10D2B80000F070FA33486FF07F4231461DE0EC779A
:10D2C800314800F02FFE0022214615E001F008F851
:10D2D8000128074625D121460DF10702304601F005
:10D2E80004F80446A0B99DF807302748AB7500F04C
:10D2F80019FE9DF807102246304600F065FB696864
:10D30800224801F061FC214801F024FC002006E0DD
:10D318001F4B3A460021022001F0A2F8032003B077
:10D32800F0BDAC75CCE70223AB73AC76C8E713F855
:10D33800011FC943197002F801CB85E7D1106FEAC4
:10D34800020C715C0CF0070C013241FA0CF101F08F
:10D3580001014FEAE20C4B40D14310F80CE001F018
:10D36800070103FA01F141EA0E0100F80C1071E718
:10D37800E121F32000F00EFA04218DE700040048B3
:10D38800FC1900205C1A00200A1A0020E419002069
:10D39800D8F80008F0B5BDF814409DF818709DF84D
:10D3A8001CE09DF8205040B1012814D00122002330
:10D3B80098180138B0FBF2F0F0BD87F00107E300E0
:10D3C80003EBC70318330EEB450503EBC5034FF416
:10D3D8007A714B43ECE7501F012803F1040302D88C
:10D3E8000C2C38BF0C24D1B9A2F10B0CBCF1010FE5
:10D3F8008CBF4FF0000C4FF0010C2801002F00EB00
:10D40800CE000CBF14250025A0EB8200062A4FEAA7
:10D4180082062844A2F102070DD8354610E00129FA
:10D4280006D1A2F10C00D0F1000C4CEB000CE4E7A3
:10D438004FF0000CE1E70830BCF1000FEDD0BD0063
:10D448000028ACBF2E182E1C701E90FBF5F003FBB5
:10D458000044094B062A5A5C8CBF0C340E340A2A45
:10D4680009D8A30001334FF47A71BB404B430349F9
:10D4780051F822209CE7FFDE68F900083CF9000813
:10D4880008B5094B012193F8560000F053FE4FF4FC
:10D49800D7602D2100F07EF900F033FBBDE808408D
:10D4A800024800F07BBA00BFFC190020FFFF0F0004
:10D4B80073B5A44CB4F854300025202B8DF80350D4
:10D4C800019500F01B8114D8082B0DD87BB1013BC6
:10D4D800072B0CD8DFE813F042005B000B00CD00EF
:10D4E8000B000B000B00FD00102B00F0008102B0B8
:10D4F80070BDB3F5807F00F0988011D8402B00F004
:10D508001081802BF3D1284600F032FA8E4B1B682D
:10D51800002BECD09B69002BE9D028469847E6E71A
:10D52800B3F5007FE3D1894B01222946022000F0A0
:10D5380097FF00F029F9042840F08580844B85483E
:10D548004FF400529A6201F0B7FA284600F010FA38
:10D558007D4B1B68002BCAD05B6814E07C4B7D4870
:10D568004FF400529A6201F0A7FA002000F000FA86
:10D5780000F0B8FE012801D100F0BDFE724B1B6817
:10D58800002BB4D01B68002BB1D09847AFE7704B85
:10D5980071484FF480529A6201F08EFA657895B915
:10D5A800284600F0E5F9294640F6021000F0F2F8A6
:10D5B80040F6441000F0FEF840F00201C9B240F60F
:10D5C800441000F0E7F8FF220DF1030163485E4DB7
:10D5D80000F05AFD624800F071FD2B68002B86D0E0
:10D5E8009E68002E83D094F82430012B08D194F93A
:10D5F800313094F930209DF803105848B04776E749
:10D60800E06B01A900F022FE019B9DF8031053482E
:10D618004FF47A7203F5FA7393FBF2F32A685BB25C
:10D62800956894F92920A84761E7284600F0A0F9F1
:10D63800454B1B68002B3FF45AAF9B69002B3FF406
:10D6480056AF01206AE700F09FF805287FF44FAF36
:10D658003F4B41484FF480529A6201F02DFA284618
:10D6680000F086F9384B1B68002B3FF440AFDB68AD
:10D6780089E700213B4B0122022000F0F1FEA16D59
:10D6880000293FF434AFC1F3074140F6031000F01E
:10D6980081F894F8591040F6041000F07BF894F8DB
:10D6A800581040F6051000F075F840F6021000F02A
:10D6B80081F840F00101C9B240F6021000F06AF8A2
:10D6C800002340F262211A460846A36500F0AAFA30
:10D6D8000DE7254B01220021022000F0C1FE00F0D9
:10D6E800FFFD01287FF403AF00F006FEFFE61F4BA5
:10D6F80001220021022000F0B3FEF8E6164801F0EE
:10D70800DBF9607808B900F033F90F4B1B68002B80
:10D718003FF4EDAEDB68002B3FF4E9AE9847144BBD
:10D72800E6E7144B01222946022000F099FE6078B2
:10D7380008B900F01DF9044B1B68002B3FF4D7AE65
:10D748001B6920E7FC190020581A0020EDF8000892
:10D7580000040048E4190020CC1900205C1A0020BD
:10D76800201A002001F900080AF9000814F9000835
:10D778001DF9000826F90008024BA3F85400FFF72A
:10D7880097BE00BFFC190020014B1878704700BFF6
:10D798006A1B002007B501238DF807100DF1070259
:10D7A80001460348F7F7BEF803B05DF804FB00BF75
:10D7B800C401002007B5012301460DF10702044802
:10D7C800F7F7E9F89DF8070003B05DF804FB00BF20
:10D7D800C401002010B50446F4F710FE01280CD14E
:10D7E80040F62310FFF7E6FF00F0F901214340F669
:10D7F8002310BDE81040FFF7CDBF10BD10B50C4B8E
:10D808001B7804469BB94FF4D760FFF7D3FFC4F3E6
:10D81800002100F0FE0001434FF4D760FFF7BAFF84
:10D82800E1B240F2B960BDE81040FFF7B3BF10BDE8
:10D83800691B002010B51346EFF3108472B60A4630
:10D8480001460348F7F76EF884F3108810BD00BF4F
:10D85800C401002008B5014608224FF4D860FFF73C
:10D86800E9FF002008BD000007B5074B1B7840BA48
:10D87800ADF804002BB9022201A940F2BC60FFF701
:10D88800D9FF03B05DF804FB691B002007B5074BFF
:10D898001B7840BAADF804002BB9022201A940F266
:10D8A800BE60FFF7C7FF03B05DF804FB691B0020EB
:10D8B80010B51346EFF3108472B60A4601460348C2
:10D8C800F7F769F884F3108810BD00BFC401002081
:10D8D80010B51346EFF3108472B60A4601460348A2
:10D8E800F7F74BF984F3108810BD00BFC40100207E
:10D8F8000A4601460020FFF7EBBF000010B51346AB
:10D90800EFF3108472B60A4601460348F7F768F940
:10D9180084F3108810BD00BFC401002010B5134661
:10D92800EFF3108472B60A4601460348F7F76EF81B
:10D9380084F3108810BD00BFC401002013B504464D
:10D948000020F4F735FD0220FFF744FF04F0070438
:10D9580001220DF1070184208DF80740FFF7DEFF53
:10D96800024B00221A7002B010BD00BF6A1B0020D3
:10D9780007B501228DF807000DF107018020FFF798
:10D98800CDFF9DF80730002B034B14BF0222012264
:10D998001A7003B05DF804FB6A1B002007B5094B39
:10D9A8008DF8060004221A70030C8DF80430032247
:10D9B800030A01A983208DF80530FFF7AFFF03B0F4
:10D9C8005DF804FB6A1B002010B51446FFF790FFB2
:10D9D8002046BDE81040FFF7E1BF000007B5094B3E
:10D9E8008DF8060005221A70030C8DF80430032206
:10D9F800030A01A982208DF80530FFF78FFF03B0D5
:10DA08005DF804FB6A1B002073B5002640F6E200AF
:10DA18000196FFF7CFFE00F0FE01054640F6E20052
:10DA2800FFF7B8FE40F6E500FFF7C4FE00F07F01FF
:10DA3800044640F6E500FFF7ADFE6FF07F40FFF7C4
:10DA4800CDFF04220DEB020140F61900FFF730FF6D
:10DA58003046FFF78DFF294640F6E200FFF79AFEB1
:10DA6800214640F6E500FFF795FE019802B070BD2B
:10DA780013B50C4B04460522972140F6AC001A70EA
:10DA8800FFF788FE230C8DF804300322230A01A92E
:10DA980082208DF805308DF80640FFF73FFF02B071
:10DAA80010BD00BF6A1B002007B5030C8DF80030BD
:10DAB800030A8DF801300B0C49BA8DF80200ADF855
:10DAC80004100622694694208DF80330FFF726FFDC
:10DAD800024B06221A7003B05DF804FB6A1B002093
:10DAE800002208B51146C520FFF718FF014B072291
:10DAF8001A7008BD6A1B002000221146D120FFF7CA
:10DB08000DBF00221146D220FFF708BF07B501223A
:10DB18008DF807000DF107019F20FFF7FFFE03B006
:10DB28005DF804FB07B501228DF807000DF1070128
:10DB3800A020FFF7F3FE9DF807103F2907D901F051
:10DB4800F8010131C9B240F20670FFF723FE03B0B5
:10DB58005DF804FB07B5F4F751FC431E58425841E1
:10DB68008DF8070001220DF107019620FFF7D6FE78
:10DB780003B05DF804FB07B500F07F008DF80700DF
:10DB880001220DF107018920FFF7C8FE03B05DF8F7
:10DB980004FB0000154B984207B51BD8144B98425C
:10DBA8001BD8144B98421BD8134B98421BD8134BC5
:10DBB80098428BBF6B2229226F232B238DF80420D8
:10DBC80001A9022298208DF80530FFF7A7FE03B0BF
:10DBD8005DF804FBE122E923F0E7D722DB23EDE738
:10DBE800C122C523EAE775228123E7E700E9A435C6
:10DBF80080F8A9328044E52D000B6B1B40FC5419BA
:10DC080007B58DF8062004228DF804008DF805105C
:10DC180095200DEB02018DF80730FFF77FFE03B06A
:10DC28005DF804FB07B552BAADF8042040BA0822E3
:10DC380049BAADF80000ADF802105BBA6946104663
:10DC4800ADF80630FFF76AFE03B05DF804FB07B5D0
:10DC58000B0C042200F0070049BA8DF80400ADF857
:10DC6800061097200DEB02018DF80530FFF756FEE0
:10DC780003B05DF804FB000010B508B1194B18603B
:10DC8800F3F73CFD0220FFF7A5FD0024164B2046C4
:10DC98001C70FFF76DFEF4F7AFFB012817D14FF4A6
:10DCA8002071FFF7D4FF40F611102146FFF772FDEF
:10DCB8004FF07F00FFF75FFF0E2140F61F10FFF7C0
:10DCC80069FDF4F741FB094B01221A7010BD1021C0
:10DCD80040F61110FFF75EFD102140F61210FFF715
:10DCE80059FDE9E75C1B0020601B00206A1B00202F
:10DCF80037B50C4D2B7804461BB9FFF74BFF0123B2
:10DD08002B700023084A6006E109F2F749FF042254
:10DD180000BA01900DEB02018620FFF7FFFD03B06A
:10DD280030BD00BF601B00200048E80107B5094B63
:10DD38008DF807000146187018B940F2AC60FFF77B
:10DD480029FD01220DF107018A20FFF7E7FD03B045
:10DD58005DF804FB691B0020012873B50C461646C4
:10DD680037D10020F4F74CFBA042B8BF44B20E28CC
:10DD780005461AD101231A4600210420FFF740FF67
:10DD88006FF010039C42B8BF1C46182140F6E7000C
:10DD9800FFF700FD022201A98E208DF804408DF8BE
:10DDA8000560FFF7BBFD02B070BD01230A28E4B28D
:10DDB8001A464FF0000105D11846FFF721FF03343A
:10DDC80064B2DDE70720C5F10E05FFF719FF2C4403
:10DDD800F6E740F6D800FFF7EDFC40F01E01C9B2A7
:10DDE80040F6D800FFF7D6FC0120F4F709FBA04263
:10DDF800B8BF44B2142805464FF001034FF00002A3
:10DE08000CD105210320FFF7FBFE023464B26FF04A
:10DE180008039C42B8BF1C463821B7E7112805D132
:10DE280003210220FFF7ECFE0534EFE70E2804D1AA
:10DE380002210846FFF7E4FEE9E7C5F116050721C8
:10DE480004202544FFF7DCFE6CB2E0E713B5314A45
:10DE58000446516810686B4603C32F4B20781B7823
:10DE6800834201D0FFF762FF2378032B27D8DFE82E
:10DE780003F00239283C6268284BB3FBF2F31A0C12
:10DE8800A1688DF800208DF802301A0A237B8DF8DE
:10DE98000330637B8DF801208DF80430204A00237D
:10DEA8004806C909F2F77CFE030C40BA8DF8053024
:10DEB800ADF80600082269468B20FFF72FFD02B057
:10DEC80010BD2269154BB3FBF2F31A0C8DF8002034
:10DED8008DF802301A0A237D8DF801208DF8033061
:10DEE8000422E8E7A3690093FAE762680B4BB3FBE7
:10DEF800F2F31A0C8DF800208DF802301A0A237BF1
:10DF08008DF80330637B8DF801208DF804300522ED
:10DF1800D1E700BFA0F00008691B00200000093D00
:10DF28000048E8011FB52E4A0446D1689068127C63
:10DF380001AB03C31A702B4B20781B78834201D0A6
:10DF4800FFF7F4FE2378032B26D8DFE803F0023826
:10DF58003302637AF12B21D14FF6FF70FFF784FC6F
:10DF680048F20500FFF792FC02236288A188ADF809
:10DF7800061052BAE188ADF804208DF80B30227AE9
:10DF8800A37A8DF80A20ADF808108DF80C30092214
:10DF980001A98C20FFF7C2FC04B010BDF22BE4D11C
:10DFA80041F60F50FFF760FC41F22100FFF76EFCCD
:10DFB8000623DAE7237B8DF804300122E8E7E389BA
:10DFC800094A5BBAADF80430237C13708DF806302B
:10DFD800637C8DF80730638AADF808300622D7E7EE
:10DFE800A0F00008691B0020681B002007B502226A
:10DFF8008DF804008DF805108F2001A9FFF78EFC1D
:10E0080003B05DF804FB000010B51346EFF310846D
:10E0180072B60A4601460348F6F730FD84F31088C5
:10E0280010BD00BFC401002007B5012201A91520B9
:10E03800FFF7EAFF9DF804004042401003B05DF886
:10E0480004FB000037B505460C46022201A913203F
:10E05800FFF7DAFF0A4B1B78012B0DD1094B1B7810
:10E06800012B09D140F20270FFF7A4FB9DF805309F
:10E078002870237003B030BD9DF80400F6E700BF98
:10E08800691B0020681B0020F7B50D4606460024D2
:10E098000DF10701284617468DF80740FFF7D2FF14
:10E0A8002A78BA4207D89DF807003146FFF726FCC0
:10E0B800204603B0F0BD0120FBE7000013B50322A2
:10E0C800044601A91420FFF79FFF184B1A78227005
:10E0D8004AB1012A17D014220021204600F0D0FAB4
:10E0E8000F2323700DE09DF8043023719DF805304F
:10E0F800A2605B425B10A3719DF806305B425B1027
:10E10800637102B010BD9DF804305B425B1023734D
:10E118009DF9053002339B1063739DF806305B420E
:10E128005B10A373024B1B682361EAE7691B00209D
:10E13800641B0020012908B5034608460ED1012BAF
:10E1480007D10420FFF746FB0220BDE80840F4F79A
:10E158002FB9022B14BF08460320F6E70120F4E785
:10E1680038B50446F4F746F950B102280CBF022529
:10E178000125284602222146FFF7EEFD284638BD34
:10E18800102CB4BF01250225F3E70A2070470000D0
:10E19800014B01201B6818475C1B0020014B022023
:10E1A8001B6818475C1B0020014B40201B68184760
:10E1B8005C1B002011B1012904D07047044B1B6877
:10E1C80080201847024B4FF480701B68F9E700BFA6
:10E1D8005C1B0020024B4FF400701B68184700BFFF
:10E1E8005C1B0020014B20201B6818475C1B00208B
:10E1F800014B04201B6818475C1B0020014B0820BA
:10E208001B6818475C1B0020014B10201B6818472F
:10E218005C1B0020024B4FF480401B68184700BF6E
:10E228005C1B002010B568B1074A002352F8334040
:10E23800844202EBC30101D9087910BD0133162BC2
:10E24800F4D1FEE71F20F8E7F8F9000873B51D4B75
:10E258000193044640F607000D46FFF7ABFAC0F3FA
:10E26800C10308336B4413F8042C00F0070301338F
:10E2780002FA03F3144AB2FBF3F2B2FBF4F00728F4
:10E288001ED84000042834BF042302234FF4D6606C
:10E2980002FB03F4FFF78EFA060240F2B160FFF7C3
:10E2A80089FA06F470663043030544BF6FEA0050EC
:10E2B8006FEA105063094343DB112B6002B070BD55
:10E2C8000123E3E704080A0C0048E8014FF0FF3097
:10E2D80070474FF0FF3070474FF0FF30704770477E
:10E2E800002070470020704770474FF0FF3070479C
:10E2F8004FF0FF30704770477047704770B5EFF3C5
:10E30800108672B6144B5C8A1A8A944213D1C4F5EB
:10E31800806292B2904206D3844218D901229A7040
:10E3280000221C805A825A8A0A800244C2F30902D7
:10E338005A8200200DE006D9C4F58065ADB2854249
:10E34800F1D88242E9E7121B92B28242EBD84FF031
:10E35800FF3086F3108870BD6C210020EFF3108128
:10E3680072B6034AD38A0133D38281F31088704787
:10E378006C210020EFF3108172B6034AD38A013B67
:10E38800D38281F3108870476C21002010B50848AB
:10E398001822002100F074F906484FF48062002129
:10E3A80000F06EF9044B05481B68BDE8104018479B
:10E3B8006C2100206B1D002018F1000831E50008D1
:10E3C800014B5860704700BF6C210020014B187248
:10E3D800704700BF6C21002073B5EFF3108572B64B
:10E3E8001C4CE08A00282FD1FFF7B8FF218A628AE7
:10E3F800914227D0A378012B12D1238820805B1A61
:10E408009BB20221A382A17063B9A3702382238ADD
:10E418009A428BBFD21AC3F58063A282A38201E01D
:10E42800002BF4D0268A0C4B1E4485F31088F3F792
:10E438004FFA0A4BA18ADB680193304602B0BDE867
:10E4480070401847FFF796FF85F31088002002B048
:10E4580070BD00BF6C2100206B1D002018F1000862
:10E4680008B4F0B586B00023ADF800302B4B0B9CF8
:10E478001D7A85424CD3D86881434CD15B681BB167
:10E4880012B1694602A898470CAB22464FF40071B6
:10E498002348019300F0F4FBFFF760FFBDF800305C
:10E4A80018440DF1020180B2FFF728FF01302AD08D
:10E4B8000023BDF80020BDF802601A480DF1080CD1
:10E4C8001F4699B216FA83F58A42ADB215D817B12C
:10E4D8003244ADF80220BDF80250019B22464FF4A9
:10E4E8000071284400F0CCFBFFF744FFFFF774FFEE
:10E4F80006B0BDE8F04001B070471CF8011B41555B
:10E5080001330127DDE7FFF735FF6FF00200EFE782
:10E518006FF00400ECE76FF00500E9E76C210020DC
:10E528006B1B00206B1D002013B5EFF3108472B62F
:10E53800204B9A78588A022A1DBF1A8A998A52183B
:10E54800002214BFC2F309029A7090421A8228D09E
:10E55800D98A012925D19978012913D119888A1ACC
:10E56800022192B2997000219A82198062B99A7038
:10E578001A821A8A90428BBF801AC2F580629882EA
:10E588009A8201E00029F4D0188A0B4A104484F3D7
:10E5980010880A4A998AD368019302B0BDE81040EE
:10E5A800184784F31088F3F797F902B0BDE81040D4
:10E5B800FFF7E0BE6C2100206B1D002018F1000859
:10E5C800024A00231360024A136070478821002022
:10E5D8008421002010B5EFF3108472B641B10129EF
:10E5E80003D1064A13680343136084F3108810BDEF
:10E5F800024A136823EA0003F6E700BF88210020D7
:10E6080010B5EFF3108472B641B1012903D1064A5F
:10E6180013680343136084F3108810BD024A13681B
:10E6280023EA0003F6E700BF8421002038B5EFF3A2
:10E63800108572B60A4B0B4C1B6833B12368984798
:10E648006368984785F3108838BD074B1B681BB172
:10E65800A3689847E368F4E7236998476369F0E794
:10E6680088210020B4F000088421002001380A44E1
:10E67800914200D1704711F8013B00F8013FF7E7DC
:10E6880000F020BC10B5EFF3108472B6064A136888
:10E6980003431360054A52F83130034342F83130DE
:10E6A80084F3108810BD00BFB02100208C21002009
:10E6B80070477047B0F5803F3ABF0004102300232D
:10E6C800B0F1807F3EBF08330002DBB2B0F1805F5B
:10E6D80038BF00014FEA1070054A38BF0433125C96
:10E6E80038BFDBB2C3F11F03981AC0B2704700BF2E
:10E6F800A8FA00082DE9F84F384D394ED5F80080B2
:10E70800DFF8E0B0DFF8E0A0DFF8E090D6F800C06E
:10E71800374FDBF80010374CDAF80020D9F8003012
:10E7280008EA00002860286800EA020E1EEA0C0FBA
:10E7380001D019421ED04FF0FF333B60FFF7B8FFFE
:10E74800EFF3108472B63368DBF80020DAF80010B3
:10E758000B4029680B4205D1D9F80030134201D18A
:10E76800F3F744F884F31088FFF7A3FFC5F8008097
:10E77800BDE8F88F236823680340134062681A4293
:10E7880004BF4FF0FF32626060681840FFF792FFE5
:10E7980062683860012303FA00F022EA000262602E
:10E7A800EFF3108172B63A689340326822EA0302A6
:10E7B8003260226822EA0303236081F310880E4A3C
:10E7C8003B6852F823309847D6F800C0DBF80010B1
:10E7D800DAF80020D9F80030A5E700BF00010020D2
:10E7E800B0210020AC21002004010020A821002035
:10E7F800A42100208C2100209421002010B511466E
:10E80800EFF3108472B6FFF755FF034B43F820105F
:10E8180084F3108810BD00BF9421002082B082B01C
:10E828000DF1080C0CE90600BDF8042003930B4415
:10E83800BDF810100A4491B212B2B2F57A7FA2BFA5
:10E84800A1F57A72013312B20360828002B002B07D
:10E85800704782B082B00DF1080C0CE90600BDF8D3
:10E8680004200393CB1ABDF81010521A91B212B2B9
:10E87800002ABEBF01F57A7203F1FF3312B20360BA
:10E88800828002B002B0704730B585B0114D6B463A
:10E8980083E8030000230293ADF80C3003A82B692A
:10E8A8009847009BBDF804400290181ABDF80C3038
:10E8B800E41AA3B224B2002CBEBF03F57A731CB2CB
:10E8C80000F1FF302B689847AB682046984705B0A1
:10E8D80030BD00BFD8F0000873B5114E00230546BF
:10E8E8000093ADF8043001A833699847F3680090A5
:10E8F8009847736804469847009B1844BDF804304D
:10E9080023449AB21BB2B3F57A7FA2BF0130A2F5B5
:10E918007A731BB228602846AB8002B070BD00BF76
:10E92800D8F0000837B500230093ADF80430074B42
:10E9380004461B6901A898476D46009095E80300B6
:10E9480084E80300204603B030BD00BFD8F00008BB
:10E9580037B50F4D02AB03E90300EB6898476B68C6
:10E9680004469847BDF80430009A1B1B99B21BB2A5
:10E97800002BA2EB0002BEBF01F57A7102F1FF3253
:10E988000BB24FF47A7000FB023003B030BD00BF09
:10E99800D8F000082DE9F0414FF47A75B1FBF5F590
:10E9A800C5EB4513DFF83C8005EB8303A1EBC303FC
:10E9B8009CB2D8F80C3006469847D8F80430074679
:10E9C8009847E31999B21BB2B3F57A7F2844A2BFDE
:10E9D800A1F57A7301301BB23060B3803046BDE8D0
:10E9E800F08100BFD8F00008024B00221A60024BE9
:10E9F8001B681847B4210020ECF00008F8B504465D
:10EA0800174608461E467CB173B1084B00255B6A61
:10EA180025609847069B60602581A572E6602361A2
:10EA2800E77265612846F8BD0120FCE7ECF00008B4
:10EA380010B5034CE3699847A36ABDE8104018472E
:10EA4800ECF0000870B5064DEB69064698476B6A0E
:10EA5800044630469847AB6A201ABDE8704018470C
:10EA6800ECF00008054B1B680BB918467047834249
:10EA780001D05B69F8E70120704700BFB42100208E
:10EA88002DE9F3410B4E336A044698470123B769D1
:10EA98002372D4F800800546B8472844804502D23E
:10EAA800B84728442060B3682068019302B0BDE8E5
:10EAB800F0411847ECF0000870B520B3EFF310866A
:10EAC80072B6124D2B680122827253B10022427233
:10EAD80098425C690ED102723CB120462C60FFF767
:10EAE800CFFF86F31088002070BD094BDB6898477C
:10EAF8002C60F6E71A465B69002BF2D09842F9D1F0
:10EB080043695361EDE70120EEE700BFB42100201F
:10EB1800ECF00008084B10B51A685369516911B92F
:10EB28005061416110BD046819688C4202D91A46C7
:10EB38005B69F3E71946F3E7B4210020044A136838
:10EB48000BB10021197243611060FFF799BF00BF34
:10EB5800B42100202DE9F041044600282DD0FFF70C
:10EB680081FF50BB657A45BBEFF3108872B6144E2F
:10EB78006768336A984787422CBF27602060114F27
:10EB8800A5724FF4807323813B684BB9336998476A
:10EB98002046FFF7D3FF88F310882846BDE8F081A8
:10EBA800B3699847236818443B6820601B689842FB
:10EBB8002046EED3FFF7AEFFEDE70125EDE700BFF6
:10EBC800ECF00008B421002010B5044608467CB1DA
:10EBD800084B5B6A984760602046FFF743FF40B1E7
:10EBE8002046FFF769FF2046BDE81040FFF7B2BF97
:10EBF800012010BDECF000082DE9F041EFF310877B
:10EC080072B61D4E1D4D736998473369044698477F
:10EC18002B684BB94FF000082B688BB9286828BBC4
:10EC280087F31088BDE8F081011B241A1A688A420C
:10EC38008CBF121900221A605B69002BF6D1E9E734
:10EC48001C681CB1B36998478442E7D22C68636991
:10EC58002B60A4F80880D4E9033098476389B3F59A
:10EC6800807FD9D12046FFF775FFD5E7037A002BBF
:10EC7800D6D1FFF705FFD3E7ECF00008B421002058
:10EC88002DE9F04F002997B081461E4640F31181C7
:10EC980004464F1E1378A4EB090023B90023237000
:10ECA80017B0BDE8F08FB842F8DA252B05D004F884
:10ECB800013B904608F10102ECE792F801E0AEF161
:10ECC800300102F10108AEF130034A424A41092BF2
:10ECD8002BD8414600250A20884611F8013BA3F1AC
:10ECE800300CBCF1090F1BD998F80030692B00F0E3
:10ECF8009E801DD8632B29D0642B00F09880582B58
:10ED08005AD0252B1AD198F80030002B00F09380A8
:10ED180004F8013BA4EB0903BB4280F28A80C9E7EF
:10ED280000FB0533A3F13005D6E74FF0FF35DBE7ED
:10ED3800752B7ED0782B41D0732B1CD0252304F85B
:10ED4800013BA4EB0903BB4273DADCE7002D05F1B4
:10ED5800FF3AD8BF4FF0000A52462046202100F063
:10ED6800B1F8A244002D56F8043B8AF80030D8BF09
:10ED780001252C449EE7504B56F804BBBBF1000F0D
:10ED880008BF9B465846F1F7F3F92A1A8542B8BFDF
:10ED98000022824620212046019200F093F8019A31
:10EDA80000232244534502DB02EB0A0482E71BF8E6
:10EDB8000310D1540133F5E742F040021021DFF887
:10EDC800FCB0DFF8FCA056F804CB12F0400F18BFD7
:10EDD800DA46BEF1300FCDF808A0A4EB09030CBF4A
:10EDE8004FF0300A4FF0200A9207A7EB0303604662
:10EDF800CDF80CA022D5002820DA4042013D4FF082
:10EE08002D0C05AA019200228246B0FBF1F001FB0D
:10EE180010AB029810F80BB0019800F801BB5145EF
:10EE2800019002F10102BAFBF1F0EDD910E042F0D5
:10EE380002020A21C3E708F1FF386BE7BCF1000FB3
:10EE480002D04FF0000CDCE730228DF814200122AC
:10EE5800BEF1300FA5EB020504D02020002D05F1EE
:10EE6800FF350ADCBCF1000F05D02D21013B04F869
:10EE7800011B3FF41FAF25440AE0013B04F8010BD6
:10EE8800ECD117E7039904F8011B013B3FF412AFDB
:10EE9800291B0029F6DC05A9114423442244A24277
:10EEA8003FF408AF11F8010D04F8010B9C42F6D1AC
:10EEB80000E70020F4E600BFB8FA0008E4FA00080A
:10EEC800BFFA000802440346934200D1704703F892
:10EED800011BF9E770B50D4D0D4C641BA4100026FD
:10EEE800A64209D10B4D0C4C00F09AF8641BA410F3
:10EEF8000026A64205D170BD55F8043B9847013657
:10EF0800EEE755F8043B98470136F2E7ECFB0008BA
:10EF1800ECFB0008ECFB0008F0FB00080000000018
:10EF28002DE9F041C1F30A57A7F2FF36132E024626
:10EF38000B460C460546804635DC002E17DA34A30E
:10EF4800D3E90023F1F722F900220023F1F752FB5D
:10EF580050B1002C57DA24F000442C430025AC4271
:10EF68002D4C08BF4FF0004423462A4624E02B4F7F
:10EF7800374101EA070C5CEA000C1DD024A3D3E951
:10EF88000023F1F703F900220023F1F733FB0028EF
:10EF9800EAD0002CBEBF4FF480133341E41824EAB2
:10EFA80007040025E0E7332E0ADDB6F5806F03D1AC
:10EFB800F1F7ECF802460B4610461946BDE8F08119
:10EFC800A7F213474FF0FF3C2CFA07F70742F3D09C
:10EFD8000FA3D3E90023F1F7D9F800220023F1F7B2
:10EFE80009FB0028C0D0002C0ADA142E01D1013404
:10EFF80006E0C6F134060123B3401D444545F6D367
:10F0080025EA0705B0E700252C46ADE7AFF30080F9
:10F018009C7500883CE4377E0000F0BFFFFF0F00BE
:10F02800F8B500BFF8BC08BC9E467047F8B500BFED
:08F03800F8BC08BC9E467047BD
:10F0400000000000010000000200000000000000BD
:10F050008813000010270000204E000030750000CB
:10F06000409C000050C3000060EA0000C0D40100D2
:10F0700080A903000053070000EA063700000000E3
:10F080005000000040F70937000000005000000069
:10F09000C194C10000000000B22700000000000081
:10F0A0000000000000000000000000000000000060
:10F0B00000000000851600089716000835160008A5
:10F0C0009B160008191600083116000825647325E0
:10F0D0003033643A00000000E9190008891A00087A
:10F0E000F9190008951A0008591A0008A11A000811
:10F0F00000000000091A0008C11900088D19000855
:10F10000451900089D190008B11900085119000897
:10F110005519000869190008111D0008391D00085B
:10F12000BD1C0008A91C0008A0860100400D0300BA
:10F13000801A060000350C0040420F0080841E003B
:10F1400000093D0000127A000024F40000366E0130
:10F150000048E801006CDC02000000000000000034
:10F16000000000000000000000000000000000009F
:10F17000000000000000000001000000020000008C
:10F180000300000004000000010000000300000074
:10F190000500000001000000010000000600000062
:10F1A0000A0000002000000002000000040000002F
:10F1B0000800000010000000400000008000000077
:10F1C000000100000002000001000200040006002F
:10F1D00008000A000C001000200040008000000120
:10F1E00008040204080101010101010307010000F4
:10F1F0006572726F723A20526567696F6E2069732B
:10F20000206E6F7420646566696E656420696E2087
:10F21000746865204D573A20736574206C6F726175
:10F2200077616E5F636F6E662E68206163636F72D5
:10F2300064696E676C790D0A004D41432072785401
:10F24000696D654F75740D0A004D41432074785403
:10F25000696D654F75740D0A004D41432072784405
:10F260006F6E650D0A004D4143207478446F6E65E2
:10F270000D0A00080A0C0D0E10121415181A1B1D89
:10F280001E212403050205010602020500000600F6
:10F29000000105040402020202020202020202024A
:10F2A0000202020203020202020202030403020239
:10F2B0000202020405040302020202050605040319
:10F2C00002020206070605040302020707070605F5
:10F2D0000403020707000000000000010201000013
:10F2E0000000000203020100000000030403020109
:10F2F00000000004050403020100000506050403E4
:10F3000002010006070605040302010707070605B8
:10F31000040302070700000B357DF2F2F23333736A
:10F3200073DEDEDEDE33337373F2F2F2F2000000DE
:10F3300048E8010048E8010048E8010048E8010009
:10F3400048E8010048E8010090D0030000000000F8
:10F350000C0B0A090807073252585F2573206F6E9D
:10F36000206672657120256420487A2061742044EB
:10F37000522025640D0A005258206F6E2066726577
:10F380007120256420487A2061742044522025642D
:10F390000D0A005458206F6E206672657120256436
:10F3A00020487A2061742044522025640D0A0031DF
:10F3B0000032004D756C74695F43004D756C746963
:10F3C0005F500000AFF30008B1F30008B9F3000884
:10F3D000B3F30008C1F30008BBF30008A584998DBE
:10F3E0000DBDB1545003A97D1962E69A459D408731
:10F3F00015EBC90BEC67FDEABFF7965BC21CAE6A62
:10F400005A41024F5CF434089373533F0C52655ECB
:10F4100028A10FB509369B3D2669CD9F1B9E742EF2
:10F420002DB2EEFBF64D61CE7B3E7197F568002C58
:10F43000601FC8EDBE46D94BDED4E84A6B2AE516FC
:10F44000C5D75594CF100681F044BAE3F3FEC08AC5
:10F45000ADBC4804DFC17563301A0E6D4C14352FF6
:10F46000E1A2CC3957F28247ACE72B95A098D17F27
:10F47000667EAB83CA29D33C79E21D763B564E1E8D
:10F48000DB0A6CE45D6EEFA6A8A4378B324359B754
:10F490008C64D2E0B4FA0725AF8EE918D5886F7274
:10F4A00024F1C751237C9C21DDDC86859042C4AACF
:10F4B000D8050112A35FF9D0915827B93813B33397
:10F4C000BB7089A7B622922049FF787A8FF88017FF
:10F4D000DA31C6B8C3B07711CBFCD63AC6F8EEF62F
:10F4E000FFD6DE916002CE56E7B54DEC8F1F89FA4C
:10F4F000EFB28EFB41B35F452353E49B75E13D4C76
:10F500006C7EF5836851D1F9E2AB622A0895469D7D
:10F5100030370A2F0E241BDFCD4E7FEA121D5834E0
:10F5200036DCB45BA476B77D52DD5E13A6B900C1AC
:10F5300040E379B6D48D67729498B085BBC54FED22
:10F54000869A66118AE904FEA078254BA25D8005A3
:10F550003F2170F16377AF4220E5FDBF811826C3DC
:10F56000BE35882E9355FC7AC8BA32E6C0199EA3E0
:10F5700044543B0B8CC76B28A7BC16ADDB647414DA
:10F58000920C48B89FBD43C43931D3F2D58B6EDAA3
:10F5900001B19C49D8ACF3CFCAF447106FF04A5C74
:10F5A00038577397CBA1E83E96610D0FE07C71CC84
:10F5B0009006F71CC26AAE6917993A27D9EB2B223D
:10F5C000D2A907332D3C15C987AA50A50359091A9A
:10F5D00065D784D082295A1E7BA86D2C637C777BEB
:10F5E000F26B6FC53001672BFED7AB76CA82C97D3F
:10F5F000FA5947F0ADD4A2AF9CA472C0B7FD9326D0
:10F60000363FF7CC34A5E5F171D8311504C723C3D3
:10F610001896059A071280E2EB27B27509832C1A17
:10F620001B6E5AA0523BD6B329E32F8453D100ED71
:10F6300020FCB15B6ACBBE394A4C58CFD0EFAAFB55
:10F64000434D338545F9027F503C9FA851A3408F1D
:10F65000929D38F5BCB6DA2110FFF3D2CD0C13EC35
:10F660005F974417C4A77E3D645D197360814FDCCA
:10F67000222A908846EEB814DE5E0BDBE0323A0AAE
:10F680004906245CC2D3AC629195E479E7C8376D32
:10F690008DD54EA96C56F4EA657AAE08BA78252E57
:10F6A0001CA6B4C6E8DD741F4BBD8B8A703EB566E0
:10F6B0004803F60E613557B986C11D9EE1F89811D1
:10F6C00069D98E949B1E87E9CE5528DF8CA1890DC0
:10F6D000BFE6426841992D0FB054BB162323232364
:10F6E000232320257320253032583A253032583ACA
:10F6F000253032583A253032583A253032583A259A
:10F700003032583A253032583A253032583A25307E
:10F7100032583A253032583A253032583A2530326C
:10F72000583A253032583A253032583A2530325836
:10F730003A253032580D0A00232323232323204463
:10F7400065764555493A2020202020202530325822
:10F750003A253032583A253032583A253032583A24
:10F76000253032583A253032583A253032583A2529
:10F770003032580D0A0023232323232320417070A5
:10F780004555493A202020202020253032583A255E
:10F790003032583A253032583A253032583A2530EE
:10F7A00032583A253032583A253032583A253032DC
:10F7B000580D0A0023232323232320446576416424
:10F7C00064723A2020202020253032583A253032E9
:10F7D000583A253032583A253032580D0A004170D7
:10F7E000704B65793A2020202020004E776B4B65C6
:10F7F000793A2020202020004E776B534B65793AD0
:10F800002020202000417070534B65793A20202041
:10F8100020004442496E744B65793A202020004D07
:10F8200043526F6F744B65793A2020004D434B452E
:10F830004B65793A20202020004D43417070534B96
:10F8400065795F303A004D434E776B534B65795F76
:10F85000303A0000000000004150505FDEF7000821
:10F86000010000004E574B5FEBF700080800000056
:10F870004E574B53F8F70008090000004150505311
:10F8800005F800080A0000004442495F12F8000829
:10F890000B0000004D4352541FF800080C000000FC
:10F8A0004D434B452CF800080D0000004D434B30F4
:10F8B00039F800080E0000004D41533039F80008B7
:10F8C0000F0000004D4E533046F8000810000000B5
:10F8D0005A45524F13F90008526164696F53656EBF
:10F8E00064204F76657273697A650D0A004952513A
:10F8F0005F52585F54585F54494D454F55540D0A57
:10F9000000505245204F4B0D0A0053594E43204F93
:10F910004B0D0A00484452204F4B0D0A00484452F8
:10F92000204B4F0D0A004952515F4352435F4552ED
:10F93000524F520D0A00020100030000841E000015
:10F94000093D0000127A000024F4000048E801009C
:10F9500090D0030020A1070000000000B1280000A3
:10F9600061510000C3A20000040506004DC7000855
:10F9700011C6000849C800088DC6000861D10008FA
:10F9800035C700088DCE000805CD0008F1C4000879
:10F990009DD30008DDD1000821C7000809C6000872
:10F9A000B9C6000891C6000849C600083FC600084D
:10F9B00041C500083DC500083BC6000837C6000821
:10F9C000E1C700080DC800082DC60008B9D400081A
:10F9D000A1C5000869C5000889D4000845C500080C
:10F9E0000DCB000895C80008D5E20008DBE200084E
:10F9F00035C5000839C50008C01200001F0000000E
:10FA0000A816000017000000841C00000F00000072
:10FA1000E42500001E000000B42D000016000000C8
:10FA2000083900000E0000002C4C00001D000000F2
:10FA3000685B000015000000747200000D000000FB
:10FA4000589800001C00000034B7000014000000AB
:10FA5000E8E400000C000000783101001B00000009
:10FA6000686E01001300000034CA01000B000000A2
:10FA7000286202001A00000040DB020012000000B1
:10FA80003C9303000A000000C0C2040019000000FB
:10FA900060B30500110000003820070009000000D5
:10FAA00020A107000000000004030202010101017F
:10FAB00000000000000000003C4E554C4C3E003061
:10FAC000313233343536373839616263646566679D
:10FAD00068696A6B6C6D6E6F70717273747576772E
:10FAE00078797A003031323334353637383941421B
:10FAF000434445464748494A4B4C4D4E4F5051525E
:0CFB0000535455565758595A0000000045
:10FB0C0000000000000000000000000000000000E9
:10FB1C000000000000000000002B7E151628AED25D
:10FB2C00A6ABF7158809CF4F3C012B7E151628AED6
:10FB3C00D2A6ABF7158809CF4F3C082B7E1516289B
:10FB4C00AED2A6ABF7158809CF4F3C092B7E151604
:10FB5C0028AED2A6ABF7158809CF4F3C0A0000009F
:10FB6C00000000000000000000000000000B00007E
:10FB7C0000000000000000000000000000000C006D
:10FB8C000000000000000000000000000000000D5C
:10FB9C000000000000000000000000000000000059
:10FBAC000E0000000000000000000000000000003B
:10FBBC00000F00000000000000000000000000002A
:10FBCC000000100000000000000000000000000019
:08FBDC00000000000000000021
:08FBE4009405FF7F0100000001
:04FBEC005D010008AF
:04FBF00039010008CF
:10FBF400000000002503002060EA0000000001006E
:10FC040000000000000000000000000004000000EC
:10FC1400401F0000F91700082918000841180008BF
:10FC2400AD1800088D1E000871210008111E00087F
:10FC3400ED21000800000000CD200008712000081C
:10FC4400F9200008D71D0008D31D0008D51D0008A1
:10FC54005D1E0008D91D0008E51D00089920000854
:10FC64000200000000093D00100000000000000038
:10FC7400D00500200000000000000000FF0000008C
:10FC840000000000D005002000000000000000007B
:10FC9400000000000000000000000000D00500206B
:10FCA4000000FF0000000000E00000004D680008B4
:10FCB4007D67000889670008B56700080000000038
:10FCC40000000000A568000895670008156C00088E
:10FCD4000000000000000000000000000000000020
:10FCE400000E0F0D0109081101000000FF000000C3
:08FCF400FFFFFFFFFFFFFFFF10
:0400000508002415B6
:00000001FF
